:020000040000FA
:040000006FD00400B9
:101000006F00907E00000000000000009020002093
:10101000AA220020A9BDF9F56C23002000000000E1
:10102000000000006C230020902000200000000041
:101030000000000090200020000000009020002010
:101040000000000090200020902000209020002030
:101050009020002090200020582F00209424002071
:101060000000000090200020902000201E2400207E
:1010700090200020D22300209020002090200020EB
:101080009020002090200020902000209020002020
:101090009020002001A04111B7170040985F3AC688
:1010A000945F3247E39CE6FE3245410182800111A4
:1010B00013078008F337078093F787083EC20100C3
:1010C0000100B7170040930570052380B70413068D
:1010D00080FA2380C7040100010083C6B70493F699
:1010E000F60DA385D704238007049246F3A6068055
:1010F0000100010093760502D5CEF336078093F602
:10110000860836C4010001002380B7042380C70489
:1011100001000100B70614007D89558D88C70100C4
:1011200001000100010023800704A246F3A6068007
:101130000100010073370780137787083AC6010062
:1011400001002380B7042380C704010001000100CF
:1011500001003727004093061005A303D7802380A2
:101160000704B247F3A70780010001009307800836
:10117000F3B7078093F787083ECE01000100B71749
:101180000040130770052380E704130780FA2380CB
:10119000E7040100010003C7B70413670708A3852C
:1011A000E70423800704F247F3A70780010001004A
:1011B0000561828093760504BDC6F336078093F6F9
:1011C000860836C8010001002380B7042380C704C5
:1011D00001000100B7061400938606047D89558D31
:1011E00088C7010001000100010023800704C246F6
:1011F000F3A6068001000100733707801377870884
:101200003ACA010001002380B7042380C70401000B
:1012100001003727004093062005A303D7802380D1
:101220000704D24781B773370780137787083ACC12
:10123000010001002380B7042380C70401000100DE
:1012400098471367070C98C723800704E24719BF24
:101250000111814601468145114506CE97000000E7
:10126000E780605893078008F3B7078093F78708F3
:101270003EC601000100B717004013077005238028
:10128000E704130780FA2380E7040100010003C785
:101290006704136717002383E70423800704B2471A
:1012A000F3A7078001000100F2400561828041112F
:1012B000814601468145114597000000E780A05214
:1012C00013078008F337078093F787083EC40100AF
:1012D0000100B7170040130670052380C70493066A
:1012E00080FA2380D70401000100FD552396B70240
:1012F00023800704A245F3A5058001000100733790
:101300000780137787083AC6010001002380C704CD
:101310002380D7040100010003C767041367170087
:101320002383E70423800704B247F3A70780010063
:10133000010001A0B1473305F50201007D1575FDDF
:101340008280411122C426C206C6AA8401446317C2
:101350009400B24022449244410182800504130566
:10136000803E420497000000E78000FD4180C5B741
:101370009305000273A04580824573901534924016
:101380002242B2424243D2436244F2440255925551
:101390002256B2564257D2576258F25806499649D9
:1013A000264AB64A464BD64B664CF64C065D965DD1
:1013B000265EB65E465FD65F09617300203041113C
:1013C000B7170040985F3AC6945F3247E39CE6FE49
:1013D000324541018280B71700401307000323887C
:1013E000E702854717170000232EF74873002030C7
:1013F000411122C42D6426C24AC006C637190040D6
:101400001304A4AAB704002023208900976000E0F9
:10141000E780A05F9C408297976000E0E780E05EF5
:10142000E5B737370040834747009146BD8B639E41
:10143000D702B73600401306F00F973500009385AA
:10144000E5209737000083D7673003C7A6001377DE
:10145000F70F1DE3B7E70400BC4F09468945171590
:1014600000000345A5F8829731A099466394D70000
:10147000834757007300203003C786001377F70FA8
:10148000E365F6FC13851700AE9717380000231F9D
:10149000A82A2380E70075B7B787004003C7670015
:1014A000098B6309071003C77700930600031377BE
:1014B0000703630DD708173800000348387C173638
:1014C00000001306A6780547B30606012380E60050
:1014D00083C577001737000013074779429793F5C4
:1014E000F50F2300B70003C58700973500009385EB
:1014F000E576C2951375F50F2380A5000347070015
:1015000089451377F703630CB70C63E7E50A6306B5
:10151000071A8545630CB7129737000083C7177603
:101520003307F600034707001377F70F19CB85073A
:1015300093F7F70F3D476363F71A17370000A30FC0
:10154000F772B787004009472383E700B787004059
:1015500083C77700E207E18763DE0704973700005F
:1015600083C7D771173700001307476E3E9785462C
:101570002300D700173700001307476F3E979306E5
:1015800000032300D700173700001307276D3E978D
:10159000A14685072300D70093F7F70F3D47636403
:1015A000F71417370000A30BF76CB7870040094703
:1015B0002383E70073002030930610026300D70EE8
:1015C000930620026305D70693060002E316D7F4BC
:1015D00003C727021377C70F13672700D5A803C7D0
:1015E00067001377070465CB03C7A702173800000D
:1015F00013084847173500001305853E13470708B1
:101600002385E70203C7A7021377370F1367870005
:101610002385E702814713070004B305F5008C41D9
:10162000B306F80091078CC2E399E7FEF5B503C74E
:10163000A702134707042385E70203C7A70213770E
:10164000C70F136727002385E702F9B503C76700B3
:101650001377070449C303C767021738000013084C
:101660002834173500001305652B1347070823831B
:10167000E70203C767021377370F136787002383D7
:10168000E702814713070004B305F5008C41B30658
:10169000F80091078CC2E399E7FEBDBD03C767025E
:1016A000134707042383E70203C767021377C70FB3
:1016B000136727002383E70285B503C76700137705
:1016C000070411CB03C727021377370F136787006F
:1016D0002381E70291B5238006003DBD97370000C6
:1016E000A38E0758B9BD97370000A389075875BD69
:1016F0002303048015472303E48001002302A48010
:10170000828083076480E3CE07FE23030480828007
:1017100083076480E3CE07FE03454480828083070D
:101720006480E3CE07FE2302A4808280411126C498
:101730004AC24EC006C61377F50BAD47AA892E895B
:101740009544630CF700194597000000E78080FA84
:1017500097000000E78020FB8D444E859700000035
:10176000E78040F9FD59FD1463983401B240A2446A
:101770001249824941018280135509011375F50F01
:1017800097000000E780E0F92209F1BF011126CCA3
:1017900006CEB704080097000000E780C0F61545A4
:1017A00097000000E78000F597000000E78080F6D2
:1017B00097000000E78000F62AC697000000E78047
:1017C00080F432459377150089EB13651500137586
:1017D000F50FF240E24405618280FD14E9F0014515
:1017E000CDBF397126DC4ADA4ED852D656D45AD2F9
:1017F0005ED006DE62CE66CCB7E700E07D5783AAF6
:10180000070022C603AA470023A0E71823A2E7186F
:10181000B7170040130770052380E704130780FA09
:101820002380E70483C74704930B75FFB684E20760
:1018300093FBFB0F8546AA892E8B32893724004003
:10184000E187015763FA76016308D50089461307DB
:1018500000026313D5000157D98F93F7F70FB71C18
:1018600000402382FC0411472303E4801305F00F9A
:1018700097000000E78000E8094C97000000E7802F
:1018800080E863657C15B7050700DA9537870700A0
:10189000795563FEE504B3879500636AF704370B57
:1018A0000800A94733EB65016395F90881E8814495
:1018B00097000000E78020E5268515A8DA85094510
:1018C00097000000E780C0E605090345F9FFFD1415
:1018D000050B97000000E780C0E481C49377FB0FFD
:1018E000E5F797000000E780A0EA69F17D55B7179A
:1018F0000040130770052380E704130780FA238054
:10190000E70403C74704418B2382E704F250B7E79B
:1019100000E023A0571123A24711E2543244525948
:10192000C259325AA25A125B825B724CE24C21615C
:101930008280A547639BF90685691309F00FB306FA
:101940009900B3742B01B6941349F9FFB37499004D
:10195000856B33796901416B9387F9FFB3F72701F1
:1019600099E363FC340193D94900C147E3E637FFAB
:101970003DBF0569C1697D19D9B71305800D63881D
:101980006901130500026384790113051008CA85F3
:1019900097000000E780C0D997000000E78040DF93
:1019A00031D54E99B38434416DBFDA852D4597000A
:1019B0000000E780E0D7CA94E30B99EE0509970091
:1019C0000000E78020D5A30FA9FEFDB79387F9FF9C
:1019D00093F7F70F636DFC0C83C71C0413073008E3
:1019E0006315F706370708006361EB06B3079B0032
:1019F000B706100063FBD704334BEB0089476399AC
:101A0000F9068980D549E38404EADA850945970017
:101A10000000E780E0D111090327C9FF9147232087
:101A2000E48003076480E34E07FE23033481FD173F
:101A3000EDFBFD14110B81C49377FB0FE9FF9700B9
:101A40000000E780E0D461F155B5B717004003C747
:101A50005704B70708001377070219E3B787070091
:101A60007955E376FBE833079B00E3F9E7F841B5E6
:101A70008547E380F9F0DA852D4597000000E7807F
:101A800020CB9389F4FFE38404E297000000E78011
:101A900060C893F7390091EB83260480032709007F
:101AA00093074900E396E6E03E89CE84D9BFB54767
:101AB0006399F9001305900B97000000E78080C33D
:101AC000FDB3B1471305B00AE388F9FE9947639760
:101AD000F904B7050800B365BB002D459700000069
:101AE000E78000C581448D4BA14997000000E78045
:101AF00060C263967401832704802320F900850463
:101B0000E39534FF8327048013172B0163550700E7
:101B10002312F90069BB2322F90051BB9D47639F43
:101B2000F90281451305B00497000000E78040C02A
:101B3000BD442320090023220900FD59970000001D
:101B4000E78040BD93F77400CA9703C70700FD14F0
:101B5000398D2380A700E39334FF91BBA14763979E
:101B6000F90697000000E780A0C28144630D0B00D6
:101B70008D479304C0036308FB00930400056304CE
:101B80008B01930440041375C507E30295D21945F0
:101B900097000000E78000B697000000E780A0B63D
:101BA000054597000000E780E0B426859700000017
:101BB000E78020B7094597000000E78080B69700CE
:101BC0000000E780E0BCE31405CE0DB39147639FAE
:101BD000F9001305600697000000E780A0B19700A8
:101BE0000000E78040B213059009F9B5E38109CC04
:101BF000F1547DB9BD6601471736000013068625EE
:101C0000938606A685458347060093F7F70F91C391
:101C100082800507E3F9E6FE97370000238CB722A0
:101C2000DDB77D166206618693178601E18763D46E
:101C3000070001458280931726003307F500AE9711
:101C400018439C4363E7E7007D16E37FF7FC7D556F
:101C5000828005458280FD15E205E18513978501A7
:101C6000618793F7F50F63480700FD15139725006B
:101C70002A97584365D713851700620561858280CE
:101C80003308B5021C4283A80600B335B502C297DB
:101C900033B50701AE98469585486367B5006394F0
:101CA000A50063E3070181480C43C6950CC388C2B5
:101CB0001CC2828081471397870161876343B70005
:101CC0008280139727002A97232007008507E5B70E
:101CD0008147014793968701E18663C5B6001335B6
:101CE0001700828093962700AA9694428507558F05
:101CF000D5B793D755408A07AA979C430545331516
:101D0000B5007D8D828017F3FFDFE702833D2A84D3
:101D100097000000E78060F405C5931725003E9406
:101D20000327C4FF814711EB7D1516053E9542053B
:101D3000418517F3FFDF6700033D05838507E5B79E
:101D40000145C5BF81471397870161876343C7007A
:101D5000828013972700B386E50094422A9785076F
:101D600014C3D5B77D1662066186014793178601B5
:101D7000E18763D50700133517008280931726008B
:101D8000B306F500AE9794429C437D16B58F5D8FE8
:101D9000F1BF8A05AA9501476363B500828083A6D7
:101DA000C5FFF11593D71600D98F9CC11397F60183
:101DB000E5B72A830148014701456343D700828084
:101DC000B387050183A80700B30706019C43C697A4
:101DD000AA976384F80033B517010507B308030118
:101DE000620723A0F80061871108C1BF2A83014759
:101DF0008147014563C3D70082803388E50083288B
:101E00000800330EE600032E0E003388A840330886
:101E1000C8416384080133B508018507B308E300AE
:101E2000E20723A00801E1871107E9B717F3FFDFF5
:101E3000E702232B0111B286B2842E86AA850A8579
:101E400097000000E780C0FA2A84A6850A859700DB
:101E50000000E78020E833348000060413351500C5
:101E6000018D056117F3FFDF6700E32917F3FFDF3B
:101E7000E702A3244111AA89AE8A328BB68402C23A
:101E800002C402C60144131C8401135C8C416349E3
:101E90009C02939B1400FD1B0549138CF4FFF15C1D
:101EA00033048901620461846340740792478E049D
:101EB000CE9423AEF4FE410117F3FFDF67006323E6
:101EC00013192400B30B2B01014A93172A00D6974C
:101ED00083A50B0088437800340050009700000071
:101EE000E78040DA050A93178A01E187F11BE35E78
:101EF000FCFC92474E9905042320F900A2473EC2FC
:101F0000B24702C63EC441B7131A8901135A8A4127
:101F1000131D240093178A01E18763CF970092472E
:101F20000A044E941CC0A24705091379F90F3EC25A
:101F3000B24702C63EC4ADB7B3079A0313152A00D1
:101F400056950841780034005000050AEA97DA9760
:101F50008C4397000000E780E0D26DBF197106C284
:101F600012C416C61AC81ECA22CC26CE2AD02ED219
:101F700032D436D63AD83EDA42DC46DECAC0CEC2C9
:101F8000D2C4D6C6DAC8DECAE2CCE6CEEAD0EED2F9
:101F9000F2D4F6D6FAD8FEDA971500009385058EAE
:101FA0008841E700050092402242B2424243D243B8
:101FB0006244F244025592552256B2564257D257C5
:101FC0006258F25806499649264AB64A464BD64BBD
:101FD000664CF64C065D965D265EB65E465FD65F45
:101FE0000961730020300000972100209381810156
:101FF000175100201301018117F5FFFF1305C500DC
:102000009705002093850500171600201306C6FDCE
:1020100063FAC5008322050023A055001105910530
:10202000E3EAC5FE17050200130585349715002065
:102030009385C5FB171600201306C66763FAC50013
:102040008322050023A0550011059105E3EAC5FE92
:102050001715002013050566974500209385852BED
:102060006377B500232005001105E36DB5FEFD4241
:10207000739002BC8D4273904280B722000093821D
:10208000828873900230970200209382A2F793E235
:10209000320073905230975200009382A2A873903E
:1020A00012346FB0F47573002030397101436EC67D
:1020B00019A0397141536AC866CA62CC5ECE19A0B4
:1020C000397101535AD056D252D44ED64AD826DA54
:1020D00022DC06DE33016140828241114AC026C201
:1020E00022C406C68282B24D4101024D924C224C5E
:1020F000B24B4101024B924A224AB2494101024984
:1021000092442244B240410182803D432A87637356
:10211000C3029377F700BDEFADE5937606FF3D8AE6
:10212000BA960CC34CC30CC74CC74107E36BD7FE30
:1021300011E28280B306C3408A0697020000969699
:102140006780A6002307B700A306B7002306B700E1
:10215000A305B7002305B700A304B7002304B70005
:10216000A303B7002303B700A302B7002302B700FD
:10217000A301B7002301B700A300B7002300B700F5
:10218000828093F5F50F93968500D58D9396050182
:10219000D58D61B7939627009702000096968682A8
:1021A000E78086FA9680C1171D8F3E96E374C3F8C8
:1021B000A5B73367B500FD530D8B79E7B7877F7FF0
:1021C0009387F7F710419441B372F6003363F6003A
:1021D000BE92B3E262006397720C6318D606504158
:1021E000D441B372F6003363F600BE92B3E26200EC
:1021F0006398720A631BD60410459445B372F600C7
:102200003363F600BE92B3E262006391720A631E0A
:10221000D6025045D445B372F6003363F600BE9241
:10222000B3E26200639A72086311D60210499449BE
:10223000B372F6003363F600BE92B3E262006393BA
:1022400072085105D105E30FD6F6131706019397CF
:102250000601631CF7001357060193D706013305E7
:10226000F7409375F50F91E982804183C18333056F
:10227000F7409375F50F91E182801377F70F93F78D
:10228000F70F3305F74082800346050083C605003B
:10229000050585056313D60065FA3305D6408280AF
:1022A00011059105E312D6FE014582802105A105A5
:1022B000E31CD6FC014582803105B105E316D6FC4E
:1022C000014582804105C105E310D6FC01458280AD
:1022D000B717004003C777051377E70FA38BE70411
:1022E000130700F8A38DE7043D47238CE704130789
:1022F0005003A38CE70403C7A7051377D70F238DDB
:10230000E7048280B717004003C7E7020D89411137
:102310001377C70F498F93068008F3B6068093F6AC
:10232000860836C601000100930670052380D70495
:10233000930680FA2380D704010001002387E70277
:1023400023800704B247F3A7078001000100410181
:10235000828041112A83014E930E407E130F001993
:10236000930F400663E56E129308001913034006AD
:10237000B3781503854E0D4FA14F337365020D8958
:102380001335150063EFBE121308F6FF79467298F5
:102390004208135808013307C70213D61700BE07B7
:1023A00032976146B3F6C60213068070B386C60242
:1023B0003697A166F58F42075D8FB716004083C739
:1023C000F60293F70708A303F1000346710083C7E1
:1023D000F60293F70708E394C7FE83477100B71628
:1023E000004093F7F70F6388071293078008F3B74D
:1023F000078093F787083EC401000100B71700402B
:10240000930670052380D704930680FA2380D704AF
:102410000100010023AA070383C6170393E60608F9
:10242000A388D70223800704A247F3A707800100EF
:1024300001001166B71700407D16D45BC85F938515
:102440004703A98EF18EF5FA93068008F3B606804D
:1024500093F6860836C601000100930670052380B6
:10246000D704930680FA2380D7040100010098C1A5
:1024700003C7170313670704A388E7022380070431
:10248000B247F3A7078001000100410182807D135C
:102490003368E3039308E016630E08003368F30320
:1024A0009308D016630808009378330093B8180097
:1024B0009388D81633081E01131E0801135E0E01FF
:1024C00055B56393E5030548638608000148630337
:1024D00003002A8871087298FD15131E0801C205B1
:1024E000135E0E01C18179BD13F8150063F4BF00BE
:1024F0007908D5B713381800E5BF83C7F60293F7FC
:102500000708A303F1000346710083C7F60293F79F
:102510000708E394C7FE8347710093F7F70FF1DFD5
:10252000E9B531714AD966CB06DF22DD26DB4ED70D
:1025300052D556D35AD15ECF62CD6AC96EC7AA8C26
:1025400002D897100000E78020B12A8993078008FD
:10255000F3B7078093F787083EDA01000100B71749
:102560000040130770052380E704130780FA2380D7
:10257000E7040100010003C7F7021377770FA38771
:10258000E70203C7F70213678700A387E7022380E8
:102590000704D257F3A70780010001000545970003
:1025A0000000E78060D6130780C13347E902116A53
:1025B00093070AE893065002BD69930BA004814A71
:1025C000014B13048008930470057D1AB347F90288
:1025D0003307D7023EC0FD873ECC938709A69309F7
:1025E000803E3347F7023AC27D873AC43347390306
:1025F0008549B399990193D93940B306D702B30BF2
:102600007703B3C6F602B3CBFB0236C6FD8636C8E7
:1026100093D6FB4136CEB7460F0093860624334946
:10262000D9028566938606FAB3969601B389E902C4
:10263000130760553309D90293060010B389E902E4
:102640003349D902B3C9F9029316390036CA37198A
:102650000040FD8636D0930D090493D7F9413ED250
:10266000F336048093F6860836DC010001009307F8
:1026700070052380FD00930680FA2380DD000100B1
:1026800001008346390593F6860FA309D9048346D2
:10269000390593E61600A309D90423800D00E256FC
:1026A000F3A6068001000100130C80FA116DF336C9
:1026B000048093F6860836DE01000100930770055A
:1026C0002380FD0023808D01010001008346390530
:1026D000216693E60602A309D90483560905B3E6E9
:1026E000A6012318D90483560905D18E2318D904CD
:1026F00023800D00F256F3A60680010001008346F8
:10270000390593F606026381061A03463905218AC4
:102710006DDE081897100000E7800098733604807B
:1027200013768608B2C20100010023809D00238039
:102730008D0101000100B717004003C6370513766D
:10274000F60DA389C70403C6370513660602A389DD
:10275000C704835609052166B3E6A6012318D904E8
:1027600083560905D18E2318D90423800D0096467F
:10277000F3A60680010001008346390593F60602A0
:10278000638B061483463905A18AEDFE970000206D
:10279000E7806090AA8636D497000020E780A08F5B
:1027A000A256E30AD5FE835609054255B3E6A601B3
:1027B0002318D90497100000E780C08F834639059D
:1027C000A18AEDDE03560905834629058247337643
:1027D000CA00B306DA0293D5F641B296B388F64042
:1027E000E24733B8C6002E983308F840A247B3B684
:1027F00016013308D84063C70701631DF8009247EC
:1028000063FA1701C247634FF80E63950701B24799
:1028100063EAF80E894663E9660FF24693151800DD
:1028200013D3F8015E8613951800B365B30042D642
:1028300046D497C00100E780E00D3258050B137BAA
:10284000FB0F63470001631A0838A25863870838F2
:1028500013081500B336A800B69513D6F5013298C3
:10286000B336C800AE9613581800FE06B3E606014C
:102870007336048013768608B2C6010001002380F7
:102880009D0023808D01010001000356C902B2960C
:10289000C206C1822316D90223800D00B646F3A6D4
:1028A00006800100010021B5F336048093F6860806
:1028B000B6C00100010023809D0023808D0101002E
:1028C00001008346390593E60602A309D904238053
:1028D0000D0086460DB5F336048093F68608B6C41F
:1028E0000100010023809D0023808D010100010073
:1028F0008346390593E60602A309D90423800D0017
:10290000A646BDB5E30B0BF0F336048093F68608BC
:10291000B6C801000100930680FA23809D00238041
:10292000DD00010001008346390593F5FC0F93F6A5
:10293000860FA309D90483463905CD8EA309D9048E
:1029400023800D00C646F3A6068001000100130592
:1029500080FA03463905930639051D8A631C9629BA
:102960007336048013768608B2CC0100010013068A
:1029700080FA23809D002380CD000100010003C662
:1029800006001376F60D2380C60003C60600136604
:1029900006022380C600835609051166D18E2318CE
:1029A000D904835609052166D18E2318D9042380C2
:1029B0000D00E646F3A6068001000100130680FA2A
:1029C0008346390593F60602638006268346390559
:1029D000130C3905A18AFDDA081897000000E7807A
:1029E000A06BF336048093F68608B6D00100010090
:1029F000930680FA23809D002380DD000100010002
:102A000083460C00116693F6F60D2300DC00834626
:102A10000C0093E606022300DC0083560905D18EE4
:102A20002318D904835609052166D18E2318D904A9
:102A300023800D008656F3A60680010001001306D0
:102A400080FA8346390593F60602638A0620834698
:102A50003905A18AEDFE97F0FF1FE780C0632A8C3D
:102A600097F0FF1FE7802063E30C85FF835609057D
:102A700011664255D18E2318D90497000000E780D3
:102A800060638346390513063905A18AFDDAF336FA
:102A9000048093F68608B6D401000100930680FAFC
:102AA00023809D002380DD00010001008346060095
:102AB00093F6F60D2300D60023800D00A656F3A64C
:102AC0000680010001008356090503462905D24707
:102AD000B376DA003306CA021305800C9355F6412B
:102AE0003696330DF6408257333CD6002E9C333653
:102AF000A601330CFC40330CCC40330885039256BE
:102B00004E86B335A5033305A503C29597C00100D2
:102B1000E78040E063468001631E0C16630C0D16CF
:102B2000130615003335A6002E959356F5013696FB
:102B3000B335D600AA959396F50105828585D18E89
:102B40006346B000639D051A638B061A0356C902DB
:102B500015823305D6003336C500B2956348B00000
:102B6000639105241306F00F637DA622894663F363
:102B7000561593078008F3B7078093F78708BED6EA
:102B80000100010037170040930770052300F70488
:102B9000930780FA2300F704010001008356C7025F
:102BA00089678117D58FC207C1832316F7022300D7
:102BB0000704B657F3A7078001000100FA506A54D2
:102BC000DA544A59BA592A5A9A5A0A5BFA4B6A4C49
:102BD000DA4C4A4DBA4D296182801308F5FF33352E
:102BE000A800FD152E951356F5013298B336C8008E
:102BF000AA9695B9F336048093F68608B6CA010002
:102C0000010023809D002380AD0001000100834668
:102C10003905CD8EA309D90423800D00D646F3A62D
:102C200006800100010035B3F336048093F6860870
:102C3000B6CE0100010023809D002380CD0001005D
:102C400001008346390593E60602A309D9042380CF
:102C50000D00F646F3A606800100010095B3F33699
:102C6000048093F68608B6D20100010023809D00FF
:102C70002380CD00010001008346390593E606025A
:102C8000A309D90423800D009656F3A606800100FF
:102C9000010045BB9306F5FF33B5A600FD152E9543
:102CA0009355F501AE96B3B5B600AA951396F50106
:102CB000858269B5F336048093F68608B6D801009C
:102CC0000100930680FA23809D002380DD0001002F
:102CD00001008356C9020566011693F6F60FD18EE0
:102CE000C206C1822316D90223800D00C656F3A660
:102CF000068001000100850A93FAFA0F95B233E6C7
:102D0000B60045C20356C9023305D0403338A0008F
:102D1000B305B040B385054115826345B000D1E1EC
:102D20006371A608894663F0560593078008F3B7D8
:102D3000078093F78708BEDA01000100B71700404B
:102D4000130770052380E704130780FA2380E70444
:102D50000100010003D7C7027D8B2396E702238081
:102D60000704D65781BDF336048093F68608B6DC97
:102D700001000100930680FA23809D002380DD007E
:102D8000010001008356C9020566011693F6F60F8D
:102D9000D18EC206C1822316D90223800D00E656C9
:102DA000B9B793078008F3B7078093F78708BEDEAB
:102DB0000100010037170040930770052300F70456
:102DC000930780FA2300F704010001000356C702AD
:102DD00093975600B297C207C1832316F7022300C8
:102DE0000704F657C1BB914763EEB70217D701003E
:102DF0001307874F8A05BA959C41BA978287B71700
:102E0000004003A7470B1345F5FF698F23AAE70A84
:102E100003A7070B698F23A8E70A03A7070A798D81
:102E200023A0A70A8280B717004083A6470B134749
:102E3000F5FFF98E23AAD70A83A6070B558D23A881
:102E4000A70A83A6070A758F23A0E70A8280B7170F
:102E5000004003A7470B498F23AAE70A03A7070BE4
:102E60001345F5FF45BFB717004083A6470B13472F
:102E7000F5FF758F23AAE70A03A7070A598D4DB7F7
:102E8000B717004003A7470B498FEDB7914763EE93
:102E9000B70217D70100130767468A05BA959C4108
:102EA000BA978287B717004003A7470D1345F5FF70
:102EB000698F23AAE70C03A7070D698F23A8E70CE6
:102EC00003A7070C798D23A0A70C8280B7170040B9
:102ED00083A6470D1347F5FFF98E23AAD70C83A6C7
:102EE000070D558D23A8A70C83A6070C758F23A06B
:102EF000E70C8280B717004003A7470D498F23AA2C
:102F0000E70C03A7070D1345F5FF45BFB7170040B2
:102F100083A6470D1347F5FF758F23AAE70C03A778
:102F2000070C598D4DB7B717004003A7470D498FC0
:102F3000EDB7797122D43714004026D24AD0035914
:102F400024028354040206D64209C2044ECE52CC57
:102F500056CA13590901C1802DE11379F9F793F489
:102F6000F49F4209C20413590901C18093078008E4
:102F7000F3B7078093F787083EC401000100930769
:102F800070052300F404930780FA2300F404010081
:102F90000100231124032310940223000404A247F8
:102FA000F3A7078001000100B25022549254025945
:102FB000F249624AD24A45618280B7F507008146EC
:102FC0003000B105194597000020E7808081A247B5
:102FD00013972701E34A07FC1369090893E40440A7
:102FE00093098008F3B7098093F787083EC0010072
:102FF0000100930A700523005405130A80FA230088
:10300000440501000100231124032310940223002E
:1030100004048247F3A7078001000100294597F0C7
:10302000FF1FE7802031F3B9098093F989084EC268
:1030300001000100230054052300440501000100A4
:103040008357040293E707202310F40223000404AB
:103050009247B9B7B7170040884742054181937737
:10306000050491EB9377F5013755E80113050580C9
:103070003345F50282809377050C130700046397AC
:10308000E7009377F50137459C1CCDB72165130503
:1030900005D0828037E700E01C435443A183E20659
:1030A000D58F1CC1FD572320F7182322F7188280E3
:1030B00013178500B7E700E023A0E710618123A282
:1030C000A7108280B7F700E08847CC47828081470D
:1030D00037370040A14663C4C7003285828003456C
:1030E000B740E38EA6FE3385F5000345050085074E
:1030F0002304A740CDB797070020938727EF9C4371
:1031000017370020130707213E95636EE500173738
:1031100000201307274F6368A70017070020232705
:10312000A7EC3E858280FD57EDBF8280411122C40D
:1031300006C62A8497000000E78000F22947B307FB
:10314000E502B2408D83B3D7870222449507B3D7F7
:10315000E70237370040C207C1832316F700410159
:103160008280411137150E0006C697000000E780E7
:1031700020FCB7370040130770F82381E7000D47A4
:10318000A381E70013070004A380E7000547238716
:10319000E700B24041018280B737004003C7170003
:1031A00019C9D98DA380B70003C70700136787002B
:1031B0002380E700828093C5F5FFF98DA380B700D7
:1031C0008280AE872A87B7360040214637380040D4
:1031D00089E717030000670083F583C8B600E30999
:1031E00016FF05078348F7FFFD17C20723041801E0
:1031F000C183F9BF411122C406C62A84970000008A
:10320000E78080E52947B307E502B2408D83B3D755
:10321000870222449507B3D7E70237370040C20739
:10322000C1832316F7404101828071654111130566
:10323000052006C697000000E78000FCB737004075
:10324000130770F82381E7400D47A381E740130778
:103250000004A380E74005472387E740B2404101CF
:103260008280CC41411106C6328503C6150083C554
:10327000050022064D8E42068D654186138875A293
:10328000630C0611634BC804138845A26300060D46
:10329000634AC800938535A26301B60823900600EF
:1032A00029464DA0138855A26305060D938565A296
:1032B000E316B6FE8D451D4663E6E5081146198EF8
:1032C00063F3C7003E86B7E704002390C600FC47BF
:1032D00097D501009385C5049DA0138895A263032B
:1032E0000611634E060D1388A5A26300061393858D
:1032F00005A5E315B6FA99451D4663E5E504198E63
:1033000063F3C7003E86B7E704002390C600FC477E
:10331000970500209385C5D71DA09D451D4663E3F5
:10332000E5022146198E63F3C7003E86B7E7040025
:10333000FC472390C6009705002093852538BA9551
:1033400082970146B240328541018280AD451D46DB
:10335000E3EAE5FE3146198E63F3C7003E86B7E720
:1033600004002390C600FC4797D501009385C5FD56
:10337000F9B7B1451D46E3E7E5FC3546198E63F321
:10338000C7003E86B7E704002390C600FC4797D5E8
:103390000100938565FC65B78D451D46E3E4E5FABC
:1033A0001146198E63F3C7003E86B7E704002390E9
:1033B000C600FC4797D50100938545F749B78D4571
:1033C0001D46E3E1E5F81146198E63F3C7003E861A
:1033D000B7E704002390C600FC4797D5010093850A
:1033E00065F9B1BFA5451D46E3EEE5F42946198E02
:1033F00063F3C7003E86B7E704002390C600FC478E
:1034000097D50100938545F31DBFB5451D46E3EBF8
:10341000E5F23946198E63F3C7003E86B7E704002C
:103420002390C600FC4797D50100938565EE01BF48
:10343000B7E7040003A3071397060020938646C44A
:103440004146A54517050020130585BA02832D4581
:103450005DE703C505000947631FE50803A84500AC
:10346000411106C6034718003285034608002207AB
:103470004168518F930828FE6307170563E9E80048
:1034800005186303070323900600294591A8130636
:1034900048FE630AC7041518E31707FF15463E8761
:1034A000637BF600154701A8130600023E8763748C
:1034B000F60013070002B7E704002390E600FC477C
:1034C0001316070111A83E8691C30546B7E704000D
:1034D000FC472390C6004206CC45418282970145B5
:1034E000B24041018280130600083E87E375F6FC76
:1034F00013070008C9B72390060005458280828023
:10350000416779176304E504411122C406C6854763
:103510002A84639FF500B7E7040022852244B24065
:1035200003A3871397050020938585334101028308
:1035300089476399F500B7E7040083A7070B854522
:10354000829771D9B2402244410182808280797190
:1035500026D252CCAE842A8A97D50100938585E382
:1035600017D50100130585E506D63AC622D44AD000
:10357000368432894ECE97C00100E780E084A28570
:1035800017D50100130585E497C00100E780C083CB
:10359000294597C00100E780008883C7840093F71E
:1035A0000702F9E383C9040089470545324763965A
:1035B000F908D44083C7160083C60600A207D58F3A
:1035C000C166138616FE638CC7028D16638FD706FD
:1035D0008D669386269029456391D706B7E7040048
:1035E000A286225403A34714B250F2494A86A68504
:1035F000025992545285624A8547456102832D459E
:103600000DEF93070002354563E98702B7E7040031
:10361000FC47C84413060002CA8582978149970770
:1036200000209387A7249C43014581CB9C4391C7ED
:103630004E852286CA8582970145B2502254925403
:103640000259F249624A456182802D457DF7930710
:10365000700F3545E3E387FEB7E70400FC47C84435
:103660002286CA85829765BF2145C1BF411122C408
:1036700037E404008327841326C2AA84416506C662
:10368000970500209385C51D7D1582978327C40A61
:1036900017050000130505E78588829795C0032369
:1036A00004132244B2409244970600209386C6AF8A
:1036B0004146C545170500201305059E41010283BB
:1036C000B2402244924401454101828019C59707C6
:1036D000002023ADA718014582804545828011470F
:1036E000636AA70A97D60100938686C90A053695AC
:1036F0001841411106C63697AE87B2850287130777
:1037000000026145639DE700B7E70400FC4713062C
:103710000002170500201305E5FA82970145B24023
:103720004101828005476145E39BE7FEB7E704005E
:10373000FC470546170500201305C5FAF9BF130716
:10374000700F6145E39DE7FCB7E70400FC471306F3
:10375000700F17050020130525F9C1B713070008DE
:103760006145E39EE7FAB7E70400FC47130600084B
:10377000170500201305C5064DB715476145E390B1
:10378000E7FAB7E70400FC471546170500201305C4
:10379000650D61B709458280411126C2B7E4040076
:1037A00083A7C41322C44AC006C62E8497050020EE
:1037B0009385050B2A898297058905C597070020FF
:1037C0009387878D83D7A70BA28503A3440D23106E
:1037D000F4002244B24092444A8502490146410124
:1037E0000283B24022449244024949454101828009
:1037F00097070020238E07069707002023AC0706B3
:10380000B717004003A7070CB706C0FFFD16758F5A
:1038100023A0E70C03A7070DB7064000558F23A888
:10382000E70C03A7070C3D9B23A0E70C03A7070D9C
:103830001367070123A8E70C8280B717004003A590
:10384000470C83A7470C598113451500C18B058987
:1038500099E3136525009707002083C767016380FC
:10386000A702970700202385A70011C9970700200A
:103870009387470003A3070063030300028382804A
:10388000114517F3FFFF670003CA011122CC06CED2
:103890003714004026CA4AC84EC652C48344740531
:1038A000034AB405834984050349940597F0FFFF53
:1038B000E78040A28347A40593F4F40F137AFA0F2C
:1038C00093E71700230DF40493F9F90F1379F90F17
:1038D000B717004003C7A705058B6DFF03D5C705C4
:1038E000A38D4705238C3705A38C2705A38B97044D
:1038F000F2406244D2444249B249224A0561828080
:1039000041119397050122C406C626C2C1872E84A1
:1039100063DC0700B7E40400FC54829719C1BC546F
:1039200082972165218D15A893F7150013C5150001
:103930008DE793F725009DC797000000E78020F0F2
:10394000B7E70400BC4F1306000A8945170500209D
:103950000345C5F2829713452400B24022449244A5
:10396000410182809397250163D80702B7E40400E0
:1039700083A7C41E829797000000E780A0F0BC4C8C
:1039800037560700130606308965170500200345E2
:10399000E5EE8297096579B7939715010145E3DE56
:1039A00007FA17D50100130565AA97B00100E78053
:1039B0008059B7E70400BC4F1306006491651705F2
:1039C00000200345A5EB82971165A9BF1D71A2CC0C
:1039D00037E404005C5C485886CE494697D5010020
:1039E000938545A2829711E917D501001305C5A259
:1039F00097B00100E780205501A0B7F600E07957A5
:103A000098CAFD57DCCA0567B7E700E023A0E710B6
:103A10001306F00290C223A0E71801000100370747
:103A2000002018471306000481459706002023A5AF
:103A3000E6E44157A38AE7403C4408088297971779
:103A40000020938727803EC88567138707409387A8
:103A500057D1231AE1002312F1021307B00F97F791
:103A6000FFFF938767662310E1023ED8154797074B
:103A700000009387C7E1B7F50700A30FE1003EDC24
:103A80000547970700009387E7DF81463000E1058F
:103A900019452301E1023EDE97F0FF1FE78060D465
:103AA00018088147994630003E9603460600850770
:103AB0000507A30BC700E398D7FEC24791C703577A
:103AC000410185676373F70001A0B7E7040083A78E
:103AD000470A08088297AA8511C917D5010013055E
:103AE000E59497B00100E780202E01A0F6406644DF
:103AF00025618280411126C2B7E4040083A704082F
:103B000006C622C4170500001305C5DF82971704F7
:103B100000201304A4D62300A40097000000E7802F
:103B2000800297000000E780E0CC034504002244B7
:103B300003A38405B2409244130600328965410113
:103B40000283797106D622D413078008F3370780E1
:103B500093F787083EC201000100B71700409305A4
:103B600070052380B704130680FA2380C704010080
:103B7000010083C6F70293F6A60FA387D70223801E
:103B800007049246F3A60680010001007337078000
:103B9000137787083AC4010001002380B70423800B
:103BA000C7040100010003C7F70213672700A387BA
:103BB000E70223800704A247F3A707800100010062
:103BC000054597E0FFFFE780207497000000E7803D
:103BD00060CB014781468147054685451305407EF8
:103BE00097E0FFFFE780207737E404003C4468005B
:103BF000514681458297B707C0A83EC8B787E803FA
:103C0000938707D03ECA97E7FF1F9387477B3EC63F
:103C10007C5868008297B2502254456182804111DD
:103C200097D50100938585E617C501001305057931
:103C300006C697B00100E780201917D501001305CB
:103C400025FF97B00100E7802018B24029454101C7
:103C500017B301006700231C411197D5010093851C
:103C600025E417C501001305657506C697B0010068
:103C7000E780801517D50100130545FA97B00100BC
:103C8000E7808014B2402945410117B30100670065
:103C90008318411122C406C6834705002A849DC7A4
:103CA00097D50100938505E717C501001305057138
:103CB00097B00100E78040114C4017D50100130573
:103CC000250C97B00100E78020103DA058410DEF72
:103CD00097D50100938505E417C501001305056E0E
:103CE00097B00100E780400E17D501001305C50A03
:103CF00097B00100E780400D2244B24029454101C0
:103D000017B3010067002311A1679386D7036313DC
:103D1000D70297D501009385E5DF17C5010013058C
:103D2000E56997B00100E780200A17D50100130567
:103D3000A5077DBFED0797D501009385A5DD17C5C4
:103D400001001305A567631BF70097B00100E7802A
:103D5000A00717D501001305650659BF97B00100EC
:103D6000E78080064C4017D501001305250791BF59
:103D7000411197D501009385E5D317C501001305BF
:103D8000E56306C697B00100E7800004B24029450C
:103D9000410117B3010067000308797122D426D2CC
:103DA0004AD02E842A898145B2844800714606D6BD
:103DB00097E0FFFFE780A03597F7FF1F9387C76065
:103DC000DC4783D70700231421012313F100975008
:103DD0000000E78000169547A305F1009307401FF8
:103DE0003EC6FD572305A100230AF10097500000AD
:103DF000E78060282686A285480097500000E7806B
:103E00002016B250225492540259456182804111C9
:103E1000814617F6FF1F13066657854517050020D4
:103E20000355452706C697C00000E780A06B15C95B
:103E300097D50100938585CA17C50100130505585C
:103E400097B00100E78040F817D50100130545EF52
:103E500097B00100E78040F7294597B00100E7805F
:103E600080FB97D50100938565C717C50100130531
:103E7000E55497B00100E78020F517D50100130540
:103E800065ED97B00100E78020F4294597B0010067
:103E9000E78060F897F7FF1F93870753DC470547D4
:103EA00097D50100938585C32390E70017C50100CE
:103EB0001305C55097B00100E78000F117D5010048
:103EC000130585EA97B00100E78000F0B24029456C
:103ED000410117B30100670003F4172500200355C3
:103EE000E5869307E5FFC2072167C1839306D7FFE5
:103EF00063F5F6029707002083C7479997060020CD
:103F000083C6D698A207D58F9306E7FFFD8E1305CB
:103F1000001081C67D1733F5E7008280411126C26B
:103F2000B7E40400FC4406C622C44AC02A844146C1
:103F300097D50100938505ED17F5FF1F130505467D
:103F4000829797000000E78080F917090020130985
:103F5000091E2310A90097D50100938565B917C5DF
:103F600001001305A54597B00100E780E0E5835502
:103F70000900228617D50100130505ED97B0010051
:103F8000E78080E4294597B00100E780C0E82286F9
:103F9000224403A38405B24092440249170500203D
:103FA0000345458E894541010283011122CC06CE8D
:103FB00026CA4AC84EC693F715002E84A5CB970093
:103FC0000000E78000E5930710F817070020230D95
:103FD000F7169707002083D7A70B914517050020F8
:103FE0001305851617070020A300F716A1831707EE
:103FF0000020230CF71497070020A388071497606C
:104000000000E780A0B997200000E78040530545F5
:1040100097600000E78080C193441400F24062443E
:1040200026854249D244B2490561828093F7250032
:10403000E9CF170700200357870F69C7AD64B71989
:1040400000409384A4AA23A0990097060020938699
:10405000660E944297D70100938707E31706002066
:104060000346060D814517F5FF1F1305253397708D
:104070000000E780E06223A0990097F7FF1F2391DB
:10408000A7242A8941C197D50100938525AE17C57C
:1040900001001305A53297B00100E780E0D2CA8580
:1040A00017C501001305454997B00100E780C0D14D
:1040B000294597B00100E78000D697070020239894
:1040C0000706930710F817070020230FF706970736
:1040D000002083D7E7FB17070020A307F706A1837B
:1040E000170700202303F70691458D471705002089
:1040F0001305850517070020A309F7049760000042
:10410000E780C0A99344240011BF93F70510C5C3ED
:10411000AD64371900409384A4AA23209900171591
:1041200000200355A56297200000E780806C2320C3
:10413000990097000000E78080DA2A899700010043
:10414000E780C0EE9344041031C5171400200354D7
:1041500024636311240597D50100938525A117C514
:1041600001001305A52597B00100E780E0C5A285F1
:1041700017C501001305053E97B00100E780C0C4D4
:10418000294597B00100E78000C997200000E7802B
:10419000003B69B5B7E70400BC4F13060014930554
:1041A000004017F5FF1F0345E56D829785BD93F726
:1041B000054091CFAD67371700409387A7AA1CC36E
:1041C00097E0FF1FE780C0089344044081BD8564E9
:1041D00093840480B3F7950099CFAD6737170040FB
:1041E0009387A7AAA18C1CC3C20497200000E78074
:1041F0000040C18025B59397350163DE0704AD67A4
:10420000371700409387A7AA1CC397F7FF1F938710
:10421000A71BDC4703D70700C167FD176316F7002C
:1042200097000000E780E0BE97700000E7806067BD
:104230001305C51497700000E7806067AD673717F6
:1042400000409387A7AA1CC3856497200000E780DD
:10425000002FA18CE1B393F705209DCFAD673717F1
:1042600000409387A7AA1CC397000100E78000DCE9
:1042700009CD854717070020230AF7EA9770000049
:10428000E780E0519344042051BB130500329700AE
:104290000000E780E0C8FDB793F74500D1C397D58C
:1042A00001009385A58C17C501001305251197B052
:1042B0000100E78060B117C501001305652B97B0B9
:1042C0000100E78060B0294597B00100E780A0B405
:1042D000930720F8170700202308F7E69707002028
:1042E00083D747DD17070020A300F7E6A183170750
:1042F0000020230CF7E4854717070020A307F7E405
:1043000097500000E78020D791451705002013053E
:10431000A5E397600000E780608893444400FDB9FE
:1043200093F78500A9C797D501009385258417C504
:1043300001001305A50897B00100E780E0A817C5A4
:1043400001001305252497B00100E780E0A7294567
:1043500097B00100E78020AC9344840097070020C9
:10436000239707DC97700000E780604345B993F717
:104370000501D1C38545170500200355A5D39760D6
:104380000100E78060F997C501009385257E17C578
:1043900001001305A50297B00100E780E0A217C550
:1043A00001001305651F97B00100E780E0A12945D2
:1043B00097B00100E78020A6930730F81707002088
:1043C0002304F7D89707002083D7C7CE170700200C
:1043D000A30CF7D68D45A183170500201305C5D67C
:1043E000170700202303F7D69344040197500000D9
:1043F000E780C07A25B193F70502D1C797C50100C0
:104400009385C57617C50100130545FB97B00100DC
:10441000E780809B17C501001305451A97B001007E
:10442000E780809A294597B00100E780C09E9307F6
:1044300040F8170700202309F7D09707002083D7FB
:10444000A7C517070020A301F7D0A18317070020F5
:10445000230DF7CE854717070020A308F7CE97074F
:104460000020239B07C297500000E780C0C0914501
:1044700017050020130545CD97500000E780007216
:104480009344040261BE93F70504FDC397C5010080
:104490009385C56D17C50100130545F297B001005E
:1044A000E780809217C501001305C51297B001007F
:1044B000E7808091294597B00100E780C095970774
:1044C000002083C767C81307700A6386E7061307CF
:1044D000800A638CE7081307600A6393E704930775
:1044E00060F8170700202301F7C69707002083D73D
:1044F000C7C317070020A309F7C4A183170700202B
:104500002305F7C4854717070020A304F7C4B14566
:1045100017050020130545C397500000E780006889
:1045200097500000E78020B59344040497070020CB
:10453000239D07BEE5B4930770F8170700202305F5
:10454000F7C09707002083D747BE17070020A30DA9
:10455000F7BEA183170700202309F7BE8547170779
:104560000020A305F7BE994565B7930780F8F1B71A
:1045700093F705088144E38307AA97C50100938553
:10458000E55E17C50100130565E397B00100E780FC
:10459000A08317C501001305650597B00100E780EA
:1045A000A082294597B00100E780E0869307A0F834
:1045B00017070020230AF7B89707002083D7C7B74B
:1045C00017070020A302F7B8A18317070020230EC6
:1045D000F7B6854717070020A309F7B6970700200D
:1045E000239C07B497500000E780E0A89145170589
:1045F0000020130565B597500000E780205A9344CA
:10460000040829BC411122C497C501009385C551F6
:104610002A8417C50100130565DA06C697A00100B4
:10462000E780807A4C4017C501001305E56E97A01E
:104630000100E7806079294597A00100E780A07D0F
:10464000034704009307F00F631FF70297C50100AB
:104650009385854D17C50100130545D697A0010028
:10466000E78080764C4017C501001305E56B97A0E5
:104670000100E78060752244B2402945410117A33B
:10468000010067004379B2402244410182809707CC
:1046900000202391A7A097070020239BB79E854762
:1046A000411117170020231DB70C17C50100130572
:1046B000E5D097C501009385654117070020231AAF
:1046C000F79C17170020230FF7F606C697A00100E6
:1046D000E780806F9715002083D5850A17C50100F4
:1046E0001305057997A00100E780006E294597A082
:1046F0000100E780407297F7FF1F9387E7CCDC4704
:1047000003D70700C167FD176311F702B7E704007D
:10471000B24003A38705056617F5FF1F03458516FD
:10472000130606C8854541010283B24041018280DB
:10473000B1C1411122C417C50100130525C82E843B
:1047400097C501009385C53706C697A00100E7808D
:10475000A067A28517C501001305456E97A001004B
:10476000E78080662244B2402945410117A3010039
:104770006700636A828097170020239307009717CA
:104780000020238107ECB7E70400FC47411106C66F
:10479000414697C501009385E56517F5FF1F130591
:1047A000E5BF8297170700200347079A9307F00A8F
:1047B0006315F7029307F0F88945170500201305E4
:1047C000A598170700202301F79897070020A38DCD
:1047D000079697500000E780603C97500000E78004
:1047E000C0678145370504009707002023A407947C
:1047F00097070020239D079297070020238A07929E
:10480000970700202398078A970700202396078898
:1048100097070020239B079097070020239E07906F
:1048200097300000E78060BF014597500000E780A7
:10483000E03F9707002083C7678F1305003299C7B1
:10484000970700202384078E13050064B2404101BE
:1048500017F3FFFF6700C36CB7E7040003A38705E6
:10486000130600149305001017F5FF1F034585017B
:104870000283B7E7040003A38705856513060014C8
:104880009385058017F5FF1F0345C5FF02837971E6
:1048900022D437E404005C5C06D626D24AD03546E2
:1048A00097C501009385053A17D501001305051238
:1048B000829711E917C50100130505B697A00100FD
:1048C000E780606801A097F7FF1F938767FC3ECCE5
:1048D000B7F50700856793870780814617F6FF1FA6
:1048E000130686FAE10519453ECE97E0FF1FE780E3
:1048F00040EF7C44194697F5FF1F9385E5F817F5BF
:10490000FF1F1305657B8297340817F6FF1F1306F8
:10491000A6F797D501009385258917D501001305C2
:10492000258A97700000E780A0ACAA8429C197C5AA
:1049300001009385A52217C50100130525A897A09E
:104940000100E7806048A68517C501001305853082
:1049500097A00100E7804047294597A00100E78024
:10496000804BB2502254925402594561828097E0A4
:104970000000E780601217C501001305A5249760A9
:104980000000E780A0A097A00000E780A0669760E5
:104990000100E78020CB17F5FF1F1305659E976088
:1049A0000100E780C0B317C501001305A522976079
:1049B0000100E780A0CBAA8497600000E780E006B2
:1049C00097100100E78000A397800100E780203C5A
:1049D00097700000E780C06297600000E780E07C8D
:1049E00097300100E780606497C501009385051743
:1049F00017C501001305859C99C897A00100E780A1
:104A0000A03CA68517C501001305052791B797A0FF
:104A10000100E780603B17C501001305252897A01A
:104A20000100E780603AAD64371900409384A4AA7E
:104A3000294597A00100E780003E23209900973088
:104A40000100E780603F2320990097F00000E78095
:104A5000E05D630F051085453705040097300000C1
:104A6000E780A09B97C501009385450F17C50100FE
:104A70001305C59497A00100E780003517C5010014
:104A80001305452397A00100E7800034294597A02E
:104A90000100E780403897F7FF1F9387678183D72E
:104AA000070017170020231DF7CC85471717002094
:104AB000230AF7B897200000E78080BF1715002071
:104AC000035505CC97500000E780A0E205459750BC
:104AD0000000E780A01597F0FFFFE78040409717A0
:104AE000002083D7E7C92AC6638FA70697C50100B0
:104AF0009385C50617C501001305458C97A00100D5
:104B0000E780802C32469715002083D565C717C5EE
:104B100001001305651C97A00100E780E02A2945E4
:104B200097A00100E780202F3C4C130600649305FA
:104B3000002017F5FF1F0345E5D4829797C50100B4
:104B40009385C50117C501001305458797A001008E
:104B5000E780802717C501001305C51A97A001003B
:104B6000E7808026D5BB3C4C130600328565D1B763
:104B700097500000E780800B1305003297F0FFFF8D
:104B8000E780003A65BF411122C437E4040083275F
:104B9000041A06C6829797500000E78040D9832701
:104BA000040817F5FFFF13058540829797F7FF1F4D
:104BB000238AA7CC17F5FF1F130505819740000036
:104BC000E780007E2244B2404101170300006700E5
:104BD00043CCB7E70400FC471171A2DDCAD986DFD8
:104BE000A6DBCED72E8432892E86AA8517F5FF1F25
:104BF00013058555829717F7FF1F1307E75483475F
:104C00000700930680029387E70793F7F70FE3EC1B
:104C1000F610BA898A0717C7010013076783BA9786
:104C20009C43BA9782878D4797C50100938545F5C8
:104C300017B5010013058578630FF40097A00100F4
:104C4000E780801817C501001305C5B097A00100C3
:104C5000E7808017BDA497A00100E780E01617C584
:104C600001001305A5B097A00100E780E0152945D4
:104C700097A00100E780201A930720F8114697F5C6
:104C8000FF1F9385654C4A8517F7FF1F230EF74AD0
:104C900097F7FF1FA38B074A97F0FFFFE7802010CD
:104CA0002A841DC997C50100938585ED17B50100BC
:104CB0001305C57097A00100E7800011A28517C5F4
:104CC0000100130565AE97A00100E780E00F2945BC
:104CD00097A00100E780201497C50100938545EA5D
:104CE00017B501001305856D97A00100E780C00D81
:104CF00017C50100130585AC97A00100E780C00C23
:104D0000294597A00100E78000114165930730FA1B
:104D1000054697F5FF1F938525437D1517F7FF1F60
:104D20002304F74297F0FFFFE78060072A841DC93C
:104D300097C501009385C5E417B501001305056803
:104D400097A00100E7804008A28517C50100130560
:104D5000A5A597A00100E7802007294597A001009D
:104D6000E780600BB7E70400BC4F0566130606C872
:104D7000A14517F5FF1F0345E5B08297FE506E541D
:104D8000DE544E59BE591161828091476303F4028B
:104D900097C501009385C5DE17B5010013050562AF
:104DA00097A00100E780400217C50100130545A444
:104DB00071BDB7E70400FC4F914517F5FF1F034590
:104DC00065AC829797C50100938585DB17B5010017
:104DD0001305C55E97A00100E78000FF17C501001D
:104DE0001305C5A297A00100E78000FE294597A002
:104DF0000100E780400297400000E780C02791450E
:104E000035A485476303F40297C50100938545D710
:104E100017B501001305855A97A00100E780C0FA75
:104E200017C50100130505A015B597F7FF1F2393BC
:104E30002729B7E704000566BC4F130606C8C1451D
:104E40000DBF8D476303F40297C50100938545D3D9
:104E500017B501001305855697A00100E780C0F63D
:104E600017C501001305C59DD5B3930740F811463A
:104E700097F5FF1F9385452D4A8517F7FF1F2305DB
:104E8000F72C97F7FF1FA382072C97F0FFFFE7800F
:104E900000F12A84E30405EE97C50100938545CE11
:104EA00017B501001305855197A00100E780C0F1F7
:104EB000A28517C501001305258F97A00100E78083
:104EC000A0F0294597A00100E780E0F445BD914797
:104ED000E31CF4F6B7E70400FC4F9305000217F556
:104EE000FF1F0345259A829797C50100938545C901
:104EF00017B501001305854C97A00100E780C0ECB1
:104F000017C5010013054595F1BD894763E3870285
:104F100097C501009385C5C617B501001305054A5D
:104F200097A00100E78040EA17C50100130505942A
:104F300031BB97F4FF1F83C4442197F7FF1F83C73A
:104F4000B72097C501009385A5C3A20417B501003A
:104F50001305C546DD8C97A00100E780E0E6A28539
:104F600017C501001305C59197A00100E780C0E5B2
:104F7000C204294597A00100E780E0E9C1849305B8
:104F8000D4FF93960401C1824A8693F5F50F17F575
:104F9000FF1F1305951B97200000E780C04BE35FC0
:104FA00090DC930750F817F7FF1F230FF71883C7FC
:104FB0003900228697F5FF1F9385051985074A85D5
:104FC00017F7FF1FA303F71897F0FFFFE78020DD17
:104FD0002A84E30505DA97C50100938565BA17B5FC
:104FE00001001305A53D97A00100E780E0DDA28543
:104FF00017C50100130585E3C9B5894763E3870237
:1050000097C501009385C5B717B501001305053B8A
:1050100097A00100E78040DB17C501001305058854
:1050200035B197400000E7800005A28517F5FF1F06
:105030001305851197500000E78040B681B38D4776
:105040006303F40297C50100938585B317B501008A
:105050001305C53697A00100E78000D717C50100EA
:1050600013058585E5B6B76602000146B7750200EF
:10507000054597D0FF1FE780C076930760F817F7C4
:10508000FF1F2303F70C97F7FF1FA380070C93075D
:10509000000617F7FF1F230BF70A894717F7FF1FB3
:1050A000A306F70A97F7FF1F2383070A97F7FF1F47
:1050B000A38F0708C14717F7FF1F230BF7089307B4
:1050C00020F917F7FF1FA305F708314697F7FF1FD1
:1050D000A381A70897F5FF1F938505074A8597F7D2
:1050E000FF1F2388070697F0FFFFE78040CB2A8445
:1050F000E30605C897C50100938585A817B501008B
:105100001305C52B97A00100E78000CCA28517B539
:1051100001001305E57B55B3B1476303F40297C55E
:1051200001009385E5A517B501001305252997A072
:105130000100E78060C917B501001305257B39B66A
:10514000B7E70400FC4F9305000417E5FF1F034574
:105150006573829797400000E780E0F1B145F9B5AB
:10516000914763E3870297C50100938565A117B551
:1051700001001305A52497A00100E780E0C417B53E
:10518000010013056578D9B497F4FF1F83C404FCAC
:1051900097F7FF1F83C777FBA204DD8C8E04B777D8
:1051A00002006D14BE942286A68517B50100130572
:1051B000E57697A00100E78020C1B7E70400FC472F
:1051C000228697F5FF1F938575F82800829793161E
:1051D0000401C1823000A685094597D0FF1FE780F2
:1051E00040602A8409C917B501001305E57497A02A
:1051F0000100E78040D5930770F8194697F5FF1F27
:10520000938585F44A8517F7FF1F230FF7F297F769
:10521000FF1FA38D87F297F0FFFFE78040B82A8435
:10522000E30E05B497C501009385859517B5010078
:105230001305C51897A00100E78000B9A28517B52E
:1052400001001305657095B99947630BF41297C572
:1052500001009385E59217B501001305251697A067
:105260000100E78060B617B501001305656FF9BA54
:10527000914763E3870297C501009385659017B551
:1052800001001305A51397A00100E780E0B317B54F
:1052900001001305656E5DBA97F4FF1F83C404EB2C
:1052A00097F7FF1F83C777EAA204DD8C8E04B777D8
:1052B00002006D14BE942286A68517B50100130561
:1052C000E56C97A00100E78020B0B7E70400FC4739
:1052D000228697F5FF1F938575E72800829793161E
:1052E0000401C1823000A6850D4597D0FF1FE780DD
:1052F000404F2A8409C917B501001305E56A97A034
:105300000100E78040C4930780F8194697F5FF1F16
:10531000938585E34A8517F7FF1F2307F7E297F781
:10532000FF1FA38587E297F0FFFFE78040A72A844D
:10533000E30605A497C501009385858417B5010090
:105340001305C50797A00100E78000A8A28517B53F
:1053500001001305A56695B699476303F40297C546
:1053600001009385E58117B501001305250597A078
:105370000100E78060A517B501001305A565F9B028
:10538000B7E70400FC4F9305000417E5FF1F034532
:10539000654F829797400000E780E0CD994579B14D
:1053A0008D476303F40297B501009385657D17B5BA
:1053B00001001305A50097A00100E780E0A017B544
:1053C00001001305A56259B017B501001305056367
:1053D00097A00100E78020B71305C01297D0FF1FE8
:1053E000E78020F6014597E0FFFFE780E0CA0D4522
:1053F00097100000E78080A0294597D0FF1FE78025
:1054000040F497D0FF1FE780A0E48DBA994763036B
:10541000F40297B501009385A57617B50100130531
:10542000E5F997A00100E780209A17B50100130560
:10543000A55D29B817F7FF1F034757D197F7FF1F3F
:1054400083C7C7D022075D8F9166BA96C2061166E0
:10545000C1821306F6EF8D476365D60297E7FF1FFB
:10546000938787F69C4B17F6FF1F034616CE93864D
:10547000C7002DC203D6070069CA8907E39CD7FE7F
:1054800089471307A0F8114697F5FF1F9385C5CBF1
:105490004A8597F6FF1F2389E6CA17F7FF1FA30661
:1054A000F7CA97F0FFFFE780808F2A84E308058C16
:1054B00097B501009385C56C17B50100130505F07C
:1054C00097A00100E7804090A28517B50100130561
:1054D000E554E5B203D60700630EE60A8907E39BAD
:1054E000F6FE8D4779BF91476304F40297B501003A
:1054F0009385056917B50100130545EC97A00100D8
:10550000E780808C17B501001305C5526FF00FF4CA
:10551000B7E70400FC4F9305000817E5FF1F03459C
:1055200065368297C9B897B501009385656517B54B
:1055300001001305A5E897A00100E780E08817B5F2
:1055400001001305A5506FF06FF02390E70017E5F9
:10555000FF1F130565E797300100E78060B397B53B
:1055600001009385E56117B50100130525E597A0B6
:105570000100E780608517B501001305254E97A04F
:105580000100E7806084294597A00100E780A0889A
:105590008147C5BD2390070017E5FF1F1305C5E22E
:1055A00097300100E780C0AE97B501009385455D57
:1055B00017B50100130585E097A00100E780C080C2
:1055C00017B501001305054B5DBF411122C406C686
:1055D000834705002A849DC797B50100938505562A
:1055E00017B50100130585DD97900100E780C07DA8
:1055F0004C4017C501001305258A97900100E780EC
:10560000A07CC9A85841B707CF009387777D631264
:10561000F70897B501009385655217B5010013058A
:10562000E5D997900100E780207A1C448356E40076
:105630008355C40003C6070017C50100130545873D
:1056400097900100E7804078294597900100E78016
:10565000807C0357E4009707002083D76712630E0E
:10566000F7008355C4000844854717070020230E20
:10567000F70C97300000E780A03F0356E400835505
:10568000C40008442244B240410117F3FFFF670001
:105690008354B707CC009387777D6315F70497B5DC
:1056A00001009385A54917B50100130525D19790F1
:1056B0000100E78060711C448356E4008355C400F8
:1056C00003C6070017B501001305857E97900100FA
:1056D000E780806F2244B2402945410117930100C1
:1056E00067006373B707CE009387777D6304F70283
:1056F00097B501009385854417B50100130505CCC6
:1057000097900100E780406C4C4017B501001305ED
:10571000E56CE5B5B240224441018280B7E7040060
:10572000FC4741112E8606C622C426C24AC02E84DA
:105730002A89AA8517F5FF1F130505A1829797B53A
:1057400001009385A54517B50100130525C797905E
:105750000100E780606797F5FF1F83C5E59E17B5D9
:105760000100130525EA97900100E780E0652945CF
:1057700097900100E780206A97F4FF1F9384C49CF0
:1057800083C7040041479387070693F7F70F636EBB
:10579000F75A17B701001307E7D58A07BA979C4352
:1057A000BA9782879D476307F40297B501009385F6
:1057B000E53E17B50100130565C097900100E7802D
:1057C000A06017B50100130565E497900100E7801C
:1057D000A05F8DA497F7FF1F83C71797DDCB17F73F
:1057E000FF1F0347979697F7FF1F83C70796220768
:1057F0005D8F97F7FF1F83C76795C2075D8F97F788
:10580000FF1F83C7B794E207D98F17F7FF1F232322
:10581000F79283C7640097B501009385253817B5C3
:1058200001001305A5B917F7FF1F2303F790979001
:105830000100E780605997F7FF1F9387A78F8C437C
:1058400017F6FF1F0346C68E17B501001305C5DD09
:1058500097900100E7804057294597900100E78025
:10586000805B97F7FF1FA381078E2244B2409244CA
:105870000249930700F817F7FF1F2307F78C9D4590
:1058800017F5FF1F1305458C410117430000670002
:10589000E33097600000E780000097F7FF1F238642
:1058A000A78A9357850017F7FF1FA300F78A93571E
:1058B00005012A8417F7FF1F230AF78893578501EC
:1058C000014517F7FF1FA303F78897600000E780E3
:1058D000E00097F7FF1F238CA78697B501009385FB
:1058E000E52B17B50100130565AD97900100E78022
:1058F000A04D17F6FF1F03468685A28517B5010048
:10590000130505D4B1B7CD476303F40297B5010081
:105910009385C52817B50100130545AA9790010086
:10592000E780804A17B50100130505D379BD37E438
:1059300004007C44414697F5FF1F9385F58017E5E9
:10594000FF1F1305A5A5829797F7FF1F83C7E78061
:1059500017F7FF1F03475780A20703238405D98F3A
:1059600017E7FF1F2315F77C1306000A8945224419
:10597000B2409244024917E5FF1F0345A5F04101DB
:1059800002838D476303F40297B5010093850521D7
:1059900017B50100130585A297900100E780C0426A
:1059A00017B50100130505DB0DB517E4FF1F034410
:1059B000C47997E7FF1F83C7377997B501009385AF
:1059C000E51D220417B501001305459F5D8C9790D6
:1059D0000100E780603FA28517B50100130545C9A6
:1059E00097900100E780403E294597900100E780AD
:1059F00080420D4697E5FF1F93850575228597E048
:105A0000FFFFE780C039AA8421C197B501009385C3
:105A1000E51817B501001305659A97900100E78016
:105A2000A03AA68517B501001305C5C597900100DA
:105A3000E78080392244B24092440249294541011D
:105A4000179301006700233D97E7FF1F23948766A4
:105A5000B7E70400116603A38705130606E891451E
:105A600039B78D476303F40297B501009385051399
:105A700017B501001305859497900100E780C034A5
:105A800017B501001305C5DB89B317E4FF1F0344F5
:105A9000C46B97E7FF1F83C7376B97B501009385EA
:105AA000E50F220417B50100130545915D8C979011
:105AB0000100E7806031A28517B501001305C5BD5F
:105AC00097900100E7804030294597900100E780DA
:105AD00080340D4697E5FF1F93850567228597E083
:105AE000FFFFE780C02BAA841DC197B501009385F5
:105AF000E50A17B501001305658C97900100E78052
:105B0000A02CA68517B50100130545BA05B797E780
:105B1000FF1F23938758B7E70400116603A3870587
:105B2000130606E89305000299B5894763E38702E7
:105B300097B501009385850617B501001305058803
:105B400097900100E780402817B50100130505D2A2
:105B5000ADB997E4FF1F83C4445F97E7FF1F83C776
:105B6000B75E97B5010093856503A20417B50100E0
:105B70001305C584DD8C97900100E780E024A6859D
:105B800017B50100130505B497900100E780C02305
:105B9000294597900100E7800028228697E5FF1F9E
:105BA0009385855A268597E0FFFFE780401F2A846A
:105BB000630E051A97B50100938545FE17A50100F0
:105BC0001305C57F97900100E7800020A28517B5D7
:105BD0000100130565B099BD854763F987188345B2
:105BE00019002244B24092440249B335B00097E70D
:105BF000FF1F238BB74C17B50100130525AF4101DB
:105C0000179301006700431CA2852244B2409244CE
:105C10004A85024941011703000067006324994740
:105C20006303F40297B50100938545F717A50100BA
:105C30001305C57897900100E780001917B501009A
:105C4000130585DC59B617E4FF1F0344045097E79A
:105C5000FF1F83C7774F97B50100938525F4220472
:105C600017A50100130585755D8C97900100E780ED
:105C7000A015A28517B501001305C5A897900100CE
:105C8000E7808014294597900100E780C0181946E5
:105C900097E5FF1F9385454B228597E0FFFFE7803F
:105CA0000010AA841DC197B50100938525EF17A5A3
:105CB00001001305A57097900100E780E010A6850C
:105CC00017B50100130505A595B397E7FF1F2395A9
:105CD0008746B7E70400116603A38705130606E8A5
:105CE0009305000869B1854797B50100938505EBD9
:105CF00017A501001305856C630BF4009790010054
:105D0000E780800C17B50100130505A27DBC9790B4
:105D10000100E780600B17B50100130565A297909D
:105D20000100E780600A294597900100E780A00EF6
:105D30002244B2409244024997E7FF1F2399073E4D
:105D4000410117630000670083A597B501009385A3
:105D5000E5E417A501001305656697900100E7804B
:105D6000A00617B50100130565CE85B4B2402244E4
:105D70009244024941018280411106C622C497E043
:105D8000FFFFE780C00121CD97E7FF1F83D7E733EF
:105D900085072A8417E7FF1F2319F73297B50100FB
:105DA000938545E197E7FF1F2392A73217A50100CE
:105DB0001305C56097900100E7800001A28517B523
:105DC00001001305A50697900100E780E0FF22443B
:105DD000B24029454101179301006700C30397E7CB
:105DE000FF1F83D7C72EB2402244850717E7FF1F46
:105DF000231FF72C41018280411122C491462A843D
:105E000017E6FF1F130686429D652D4506C697D0EF
:105E1000FF1FE780009DB7F7070003C70701A547ED
:105E20006313F70001A09306001001469D65254508
:105E300097D0FF1FE780E09A97E7FF1F2388873EF0
:105E40002244B240914617E6FF1F1306263E9D6589
:105E50002945410117D3FF1F6700A3981171CED7C1
:105E6000B7E9040083A7C904CAD917E9FF1F1309BA
:105E7000A92DA2DD2E8686DFA6DB2E84AA854A8583
:105E8000829797E7FF1F83C7272C1307700A638544
:105E9000E710636DF7001307600A6385E704FE509F
:105EA0006E54DE544E59BE59116182801307800A28
:105EB0006385E7161307900AE393E7FE8D476306B1
:105EC000F41C97B501009385250A17A50100130559
:105ED000E54E97900100E78020EF17B5010013050C
:105EE000E50525A08D47630CF40297B50100938565
:105EF000A50717A501001305654C97900100E780E1
:105F0000A0EC17B501001305A5FC97900100E780F0
:105F1000A0EB294597900100E780E0EF49B785475E
:105F200017B50100130585FC17E7FF1F230EF718AF
:105F300097900100E7802001B7750200B766020064
:105F40000146054597D0FF1FE780A089930760F8B9
:105F500017E7FF1F230AF71E97E7FF1FA387071EF8
:105F60009307002617E7FF1F2322F71EE577938785
:105F7000072117E7FF1F231DF71CB14597E7FF1FF8
:105F80002389071C97E7FF1FA385A71C4A85970055
:105F90000000E780E01621B7914763E3870297B5D9
:105FA0000100938565FC17A5010013052541979015
:105FB0000100E78060E117B50100130525F5B1B7D1
:105FC00097E4FF1F83C4841897E7FF1F83C7F71761
:105FD000A204DD8C83A7C9046D14228697E5FF1FF8
:105FE0009385D516280082978E0493160401B77501
:105FF0000200C1823000A695094597C0FF1FE780C7
:10600000407E930770F817E7FF1F230FF71299459B
:1060100097E7FF1FA38CA71295BF914763E3870201
:1060200097B50100938545F417A5010013050539BF
:1060300097900100E78040D917B50100130585EE60
:10604000E9B597E4FF1F83C4641097E7FF1F83C778
:10605000D70FA204DD8C83A7C9046D14228697E5AF
:10606000FF1F9385B50E280082978E0493160401B6
:10607000B7750200C1823000A6950D4597C0FF1F7D
:10608000E7802076930780F8BDBF17B501001305A0
:1060900025EC97900100E78000EB930790F823042C
:1060A000F100834719008D452800A304F1008347C0
:1060B00029002305F10097000000E7806004130524
:1060C000C01297C0FF1FE780C027014597D0FFFF90
:1060D000E78080FC0D4597000000E78020D229452D
:1060E00097C0FF1FE780E02597C0FF1FE78040169D
:1060F0007DB397E7FF1F23A3A714828097E7FF1FB5
:106100009387C71303A307006303030002831743A6
:1061100000006700A3A841114AC097F6FF1F83D66D
:106120002666328917F6FF1F0356466222C426C22E
:1061300006C62A84AE8497000000E780A06235C1BD
:106140002DC0994763FF9704834714000347040059
:10615000A207D98F13978700A183D98FC207316710
:10616000C1831307C755639EE70297F7FF1F83D7C5
:10617000E75DA301F400A1832302F40097F7FF1F5A
:1061800083D7076091C7A302F400A1832303F4001F
:10619000A68517B50100130525E197900100E7805A
:1061A000A0C297F7FF1F83C7E749B9CF97F5FF1F35
:1061B00083D5C55917B501001305C5E097900100B7
:1061C000E78080C02686A28517F5FF1F0355055876
:1061D00097000000E78080BA6301090497E7FF1F7A
:1061E00083C707069DCB95C897E7FF1F83C7C7EDF9
:1061F0008DE722852244B2400249A685924441019E
:10620000174300006700839917B50100130585DC6B
:1062100097900100E78020D3C1B7B2402244924456
:10622000024941018280834755008345450017B5E7
:106230000100130525D6A207DD8D17930100670025
:10624000A3B817B501001305E5D317930100670044
:1062500083CF8D4763FBB70A011126CA06CE22CC35
:106260000344350097E4FF1F83C494FD97B50100F4
:10627000938505D7B337800017E7FF1FA302F7FC0C
:1062800009C497B50100938565D617B501001305BC
:1062900065D697900100E78020B397E7FF1F83C77B
:1062A00037FA6386970097E0FFFFE780C05C97E7C7
:1062B000FF1F83C7F7F88DC785472306F100B7E7AF
:1062C000040083A747177000854513055030829757
:1062D00017B50100130505D397900100E780A0C60C
:1062E0009967938757EE2316F1006800854791451B
:1062F000A30781002307F10097000000E78040E03A
:10630000F2406244D244056182808280894763F80A
:10631000B70A011122CC06CE8347250005472A84FF
:106320006393E706914763FCB7048347450003473F
:106330003500A207D98F17F7FF1F03572741630ABC
:10634000F70017F7FF1F2313F74097E0FFFFE780E1
:10635000E0509967938767EE2314F1008547230582
:10636000F10083473400A305F100834744009545BD
:1063700028002306F10097000000E78060D8F24073
:10638000624405618280E5FF97F7FF1F83D7073CD2
:106390009386E7FFC2062167C18275176376D7002F
:1063A00097F7FF1F83D7C73D1967130767EEA3054C
:1063B000F1002314E10023050100A1834DBF828079
:1063C0000111996722CCD51717F4FF1F13048427F6
:1063D0002314F1008347040026CA97F4FF1F938417
:1063E000243A2305F10083D7040028009545A3052E
:1063F000F100A18306CE2306F10097000000E7809C
:1064000020D003D604008345040017B5010013050E
:10641000E5C097900100E780209BF2406244D2449F
:10642000056182809D677971D9172316F10097F76E
:10643000FF1F83C7272106D62307F100A9C3B7E7AB
:106440000400FC47414697D5FF1F938525F51305AA
:10645000F10082976800CD4597000000E78040CAB0
:1064600097F5FF1F83C5051E17B50100130505BE6F
:1064700097900100E7804095B25045618280B7E770
:106480000400BC47414681451305F1008297D9B706
:1064900045C5411106C622C4930750FA2300F500F2
:1064A0009307A005A300F50089472301F500914754
:1064B000A301F50093073003A302F50097F7FF1F30
:1064C0009387471883C70700230205002A84230304
:1064D000F50097E7FF1F9387B7D683C707004146AC
:1064E00097D5FF1F938585EBA303F50097F7FF1F53
:1064F00083D707292304F500A183A304F50097F7A8
:10650000FF1F83D7A7242305F500A183A305F5006A
:10651000B7E70400FC47310582972285F1459700D3
:106520000000E7802020230EA4002181A30EA400F8
:10653000B24022444101828082805D710A8586C614
:10654000A2C497000000E780E0F437E404007C4434
:106550008A850810794682973C441305E103094671
:1065600081458297101093050002014597D0FFFFE7
:10657000E7802017B640264461618280011122CC59
:106580002D6426CA4AC84EC652C456C25AC006CE48
:10659000B71400401304A4AA80C037E900E0B7098B
:1065A00040002A8AAE8A328B23203919010001006B
:1065B0008566AA850146254597C0FF1FE7806022B2
:1065C000DA865686D285294597C0FF1FE78060216D
:1065D0002320391180C0F2406244D2444249B2497A
:1065E000224A924A024B056182800111B7C7A55A1F
:1065F00022CC9387C73317E4FF1F130474C43EC42F
:10660000834704002C002146196506CE3EC697003C
:106610000000E780E0F68345040017B5010013058C
:1066200065B197800100E780207AF24062440561FD
:1066300082800111A146300099652D4522CC06CEFD
:1066400097C0FF1FE780E019A24737C4A55A13047B
:10665000C43363958702B24517B50100130545A100
:10666000B335B00097E7FF1FA38CB7BC978001003C
:10667000E7808075F2406244056182809165A146A1
:106680003000938505F02D4597C0FF1FE78060150A
:10669000A247E38287FC854717E7FF1FA302F7BAEB
:1066A000854517B501001305E59EC9B77971D14637
:1066B000700091652D4522D406D697C0FF1FE78054
:1066C0004012B24737C4A55A1304F43563988702C1
:1066D000B7E70400FC4717D5FF1F130525CC41463B
:1066E0000C08829717B50100130545A0979001008B
:1066F000E7806085B2502254456182809165D14621
:106700007000938505E82D4597C0FF1FE780600D59
:10671000B247E38F87FA17B501001305259FF9B734
:10672000C16769768146FD17050613970601418307
:106730006364B7003E8582803307D50003470700B6
:10674000B98F214713F81700858363050800B18FBF
:10675000C207C1837D171377F70F6DF78506F1B771
:1067600041C5A547054763F2B708834715000347AE
:1067700005003168A207D98F13978700A183D98FAD
:10678000C207C1831308C855054763900707411125
:1067900006C622C426C203442500914763F087043D
:1067A0009307540063ECF502A301C5002182230284
:1067B000C5009304340091C6A302D500A18223032F
:1067C000D5002A84A68597000000E780A0F52694CE
:1067D0002300A4002181A300A4000147B240224469
:1067E00092443A854101828005473A8582800111B1
:1067F000B7C7A55A22CC9387E7342A842AC62C002F
:106800002146156506CE3EC497000000E78040D7BC
:10681000A28517B501001305E59397800100E78075
:10682000A05AF2406244056182800111A146300005
:1068300095652D4522CC06CE97C0FF1FE78060FAF4
:10684000A24737C4A55A1304E43463958702B245BE
:1068500017B501001305058697F7FF1F2398B7EEBC
:10686000C205C18197800100E7800056F240624472
:10687000056182809165A1463000938505EE2D4526
:1068800097C0FF1FE780E0F5A247E38287FC17B5BA
:1068900001001305258497F7FF1F239907EA9780C6
:1068A0000100E780406AD9B797B701009387878EC8
:1068B00013D7C5003E97034707001105230EE5FED9
:1068C00013D785003D8B3E9703470700A30EE5FED7
:1068D00013D745003D8BBD893E97AE970347070010
:1068E00083C70700230FE5FEA30FF5FE8280011189
:1068F00022CC06CE26CA4AC84EC693F715002E846F
:10690000638E0716AD679387A7AA371700401CC38D
:1069100097F7FF1F83C767E399EF97F7FF1F83C7B9
:1069200047E6850793F7F70F1D47636AF70217F7E6
:10693000FF1F2308F7E4B7E70400BC4F1306001954
:10694000854517D5FF1F034525AA829713451400D7
:10695000F2406244D2444249B2490561828097F7CD
:10696000FF1F238007E2B75720419304D00393878A
:10697000777497F5FF1F83D5A5E017F5FF1F130563
:1069800075DD1309000217F7FF1F2323F7DC97F7C4
:10699000FF1F238197DC97000000E78020F1230090
:1069A000250197F7FF1F83C7E7C9B337F000938727
:1069B0000703A301F5009309000593072004A30032
:1069C00035012301950023022501A302F5002303CD
:1069D000950097D5FF1F83D5E59E1D059700000004
:1069E000E780C0EC23002501A30035019307500484
:1069F0002301F500A301950097D5FF1F83D5458C92
:106A0000110597000000E78060EA9307B0042300B7
:106A1000250123019500A300F50097D7FF1F83C729
:106A2000E797A20797D5FF1F83C55597DD8D0D0505
:106A300097000000E78080E797D7FF1F83C727965E
:106A4000A20797D5FF1F83C59595DD8D97000000A0
:106A5000E780C0E5B5472300F500A947A300F5008E
:106A60009305250017F5FF1F130585CE898DC205F7
:106A7000C18197200000E780C00875BD93F725000D
:106A800081CB97F7FF1F239107CC13C52500C9B50C
:106A900093F745000145E38D07EA17A501001305AB
:106AA000256D97800100E780004A97300000E7805D
:106AB000803C1345440069BD411122C437E4040001
:106AC0005C5C06C6354697A501009385A51717B5EA
:106AD00001001305A5EF829711E917A50100130521
:106AE000E56997800100E780004601A08327041C28
:106AF00082972A84054597C00000E78040F9976097
:106B00000100E780607E97600100E780605397B0E6
:106B10000000E780C00A2285B24022444101828001
:106B20004111054506C622C426C297C0FFFFE78073
:106B300080401305A00497B0FF1FE780405775758C
:106B400085457D1597C0FFFFE780202A7D75854527
:106B50001305F53697C0FFFFE780803337140040F8
:106B60008327840A8D451305002093E707202324FB
:106B7000F40A97C0FFFFE7804027B7E4040097C0FE
:106B8000FFFFE780C06AC85897800100E780A03BFC
:106B900017B50100130585E397800100E780A03A4F
:106BA0008327840C8545414593E707082324F40C8B
:106BB00097C0FFFFE780C02D8D451305000897C0E3
:106BC000FFFFE780E02C97C0FFFFE780C05937A5A3
:106BD00007001305051297C0FFFFE78060559D452C
:106BE000014597C0FFFFE780605BB7E700E037072C
:106BF000000423A0E7180100010097D0FFFFE78001
:106C000020DD97D0FFFFE78020EF97000000E780AE
:106C1000E0EA97000000E78000A297000000E7800C
:106C200000C197E0FFFFE78040F697000000E78093
:106C3000A02597000000E780801083A704081705AF
:106C40000000130505CB829797C7FF1F238EA778F7
:106C5000BC4C130600648545829797B0FF1FE78000
:106C6000207901458280AD67371700409387A7AA36
:106C70001CC3B7E700E03707400023A0E718010076
:106C80000100B7F7070003C70701A5476316F70020
:106C90009397450191C301A04111AE860146AA8593
:106CA000254506C697C0FF1FE780A0B3B240B7E7EF
:106CB00000E03707400023A0E71041018280411126
:106CC000B2862E86AA852D4506C697C0FF1FE7808F
:106CD00040B1B2400145410182809307000463EC5A
:106CE000C7041D71A2CC2A840808A6CACAC886CEC9
:106CF00032C697800100E780C001AD6737170040BA
:106D00009387A7AA1CC3B7E400E03709400023A07B
:106D1000241901000100B2461008A285294597C038
:106D2000FF1FE78000ACF640664423A02411D64440
:106D30004649256182803955828041110D658D4516
:106D400006C697C0FFFFE780400AB71700408D6670
:106D500023A6D70A17F5FF1F1305C5A21387C70A75
:106D60009387870A1CC15CC5856689675CC958C161
:106D700014C518C9B7E70400B24003A3871E410138
:106D800002838145B307B5008387070089E717238E
:106D900000006700E3CD8505C205C181E5B797A76F
:106DA00001009387A75D1357C5003E97034707006F
:106DB000011106CE2304E100135785003D8B3E9759
:106DC0000347070023060100A304E1001357450011
:106DD0003D8B3D893E97AA970347070083C707006D
:106DE00028002305E100A305F10097000000E780DB
:106DF00080F9F24005618280411126C2E97797F45B
:106E0000FF1F9384A4A822C49387A7552E842381AF
:106E1000B4002E86AA8517F5FF1F130565A706C6C1
:106E20002390F400A381040097800100E78060EEC6
:106E300093052400C205C18117F5FF1F130525A581
:106E400097000000E780008EB38784002382A700AC
:106E50002181A382A700930564002244B2402685C5
:106E60009244C205C181410117230000670043C05D
:106E700009C99307800263E6B700170300006700A3
:106E8000E3F7828097F7FF1F83C727A399EF41118C
:106E900006C697200000E78080B5B240854717F707
:106EA000FF1F230CF7A041018280828063040556F6
:106EB000638205565D71A2C4A6C286C6CAC04EDEF4
:106EC00052DC56DA5AD85ED662D466D26AD0B94756
:106ED0002A84AE8463F9B706394697A501009385E5
:106EE000E53297800100E78060E031ED8347E40000
:106EF000130710036394E702854717F7FF1F230565
:106F0000F79817A501001305653197F7FF1F239C1C
:106F1000079697000000E78000E771A013070003C1
:106F200017A5010013058532E395E7FE97F7FF1FCC
:106F3000238C079497F7FF1F2397079417A5010049
:106F40001305452FF9B797F7FF1F83C7E7936389A9
:106F50000722BD6AB96B938CFA55014A17FBFF1FD4
:106F6000130B0B84138CEB65938AFA6605A8B307A1
:106F7000440183C6070097F7FF1F83D7C790B1E38B
:106F80009307A005639BF600854717F7FF1F231C97
:106F9000F78E97F7FF1F2385D780050A93170A01FD
:106FA000C183E3E697FCB640264496440649F2596D
:106FB000625AD25A425BB25B225C925C025D6161B2
:106FC0008280054D639BA7039307500A639EF600DA
:106FD000894717F7FF1F2318F78A930750FA17E717
:106FE000FF1FA30FF77A55BF9307A005E387F6FAB3
:106FF00097F7FF1F239907884DB71387170042079C
:10700000DA9741832380D70017F6FF1F231DE686FA
:107010008D47E3F4E7F817E9FF1F0349997897E7ED
:10702000FF1F83C7077822093369F9009307F9FF27
:10703000C207C1839306F00DE3ECF6FA93076900EB
:10704000C207C183E31BF7F493052900C205C18180
:1070500017E5FF1F1305E57497F0FFFFE780806CCD
:1070600033072B018347570003474700A207D98FF7
:1070700017F7FF1F231907806319F50E8149630D68
:10708000A90197E9FF1F83C9E971A20997E7FF1FCB
:1070900083C75771B3E9F90017050000130585DDB3
:1070A00097F0FFFFE780200563878907636D3C0346
:1070B0009387EB556382F90497E7FF1F83C7876EB9
:1070C00005476389E70681CB1387A7051377F70F79
:1070D0008D4663F2E6081307F0072300E100A300E2
:1070E000F10089459DA063829905E39759FD97F0CA
:1070F000FFFFE780603311A8CA8517E5FF1F13055E
:10710000656A97F0FFFFE7800015014597F0FFFFE4
:10711000E78060FE59B5CA8517E5FF1F130585682E
:1071200097F0FFFFE780C01ECDB797F0FFFFE78025
:107130006029E1BF930710F8130511002300F10047
:1071400097F0FFFFE7800035FD450A8597000000B6
:10715000E780C0CA5DBFCA8517E5FF1F13058564B8
:1071600097F0FFFFE780C0CF4DB79307F007894541
:107170000A852310F10097000000E78020C831BD88
:10718000BD4763F99722414697A501009385450EB7
:10719000228597800100E78060B5631C051417A560
:1071A00001001305250E97000000E780C0BD17E51C
:1071B000FF1F0355E55C97000000E78080BE97E75E
:1071C000FF1F83C7274817A501001305250389E77B
:1071D00017A501001305050397000000E780A0BA7A
:1071E00017A501001305850B97000000E780A0B9E3
:1071F00017C5FF1F0355051D97000000E78060BA03
:1072000017A501001305C50997000000E780A0B786
:1072100017E5FF1F0355855397000000E78060B80E
:1072200017A501001305450897000000E780A0B5E9
:1072300017D5FF1F0355A5E997000000E78060B64A
:1072400017A501001305C50697000000E780A0B34D
:1072500017D5FF1F035565E797000000E78060B46E
:1072600017A501001305450597000000E780A0B1B0
:1072700017D5FF1F035585E597000000E78060B232
:1072800017A501001305850397000000E780A0AF54
:1072900017C5FF1F0355C50297000000E78060B0C7
:1072A00017A501001305050297000000E780A0ADB7
:1072B00097C7FF1F83C7870EA20717C5FF1F034588
:1072C000F50D5D8D97000000E780A0AD97C7FF1F0B
:1072D00083C7E70CA20717C5FF1F0345550C5D8D3B
:1072E00097000000E780E0AB179501001305856B60
:1072F0000DB1414697A50100938505FD2285978034
:107300000100E780A09E5DE5C114C204930604015C
:10731000C180510401498D452545154663FC950002
:10732000639F86001307E9FF4207A1674183F517B2
:1073300063FAE70417A50100130545FAD9BE83C710
:107340000600138707FD1377F70F637CE5001387AB
:10735000F7FB1377F70F636EE600938797FC13F73D
:10736000F70F12093369E90042091359090185062B
:1073700075B71387F7F91377F70FE36DE6FA93877D
:1073800097FAF1BF97E7FF1F83D7473C638A27012E
:1073900097E7FF1F239C273B97D0FFFFE780004C18
:1073A00017A501001305C5F597000000E780A09D13
:1073B0004A853DB7C147E3F897BE414697A501000E
:1073C000938545F5228597800100E7802092E31C94
:1073D00005BC8347040113071003639CE70085473E
:1073E00017E7FF1F230CF73A17A501001305C5F394
:1073F0000DB61307000317A501001305E5F5E39A81
:10740000E7B097E7FF1F238B073817A50100130587
:1074100025F301B68280411126C2AE848D4522C477
:1074200006C62A8497C0FFFFE78080A6B7170040F2
:1074300099C803A5C70C418D23A6A70CB2402244CE
:1074400092444101828003A5870C418D23A4A70C9F
:10745000F5B78347050003471500A207D98FC20778
:107460006177C18713072720639AE70083452500CA
:107470003705040017030000670023FA828017E62F
:10748000FF1F1306E6438147B2861303F00FA94896
:107490003308F6000348080013F7F70F6307A80C3A
:1074A000630668008507E39517FF2947B387E60061
:1074B0002380A70097E7FF1F938747415DA84111ED
:1074C00013D765001347170006C693F63500058BE2
:1074D000954791CA054699476387C60009469D4767
:1074E0006383C600A14713F645003336C00093F608
:1074F0008503050685C2A145638BB604E145638A11
:10750000B604930580026388B604930580036393F1
:10751000B600914697E5FF1F238FF56097E5FF1FA3
:10752000238AC56097E5FF1FA386D560BE8517A592
:1075300001001305A5E897800100E780E088B240CC
:10754000854717E7FF1FA308F75E41018280854644
:10755000D1B78946C1B78D4675BF17A50100130580
:1075600065E8178301006700238617E7FF1F1307ED
:10757000E735BA972380B700E147E302F5F49307B4
:107580007002E30CF5FC82802A8723800500814786
:1075900017E5FF1F1305C5321308F00F2946B30680
:1075A000F50083C606006396E60297E6FF1F938602
:1075B000E631B69783C7070005452380F500994754
:1075C000636EF7029D4763FDE700E147630DF70037
:1075D0008280638506018507E393C7FC0145C5B733
:1075E000238005008280B737004003C7370083C778
:1075F000050093F70704D98F2380F50082805D7121
:1076000052DC56DA5ED6716A97EBFF1F938BCB6321
:107610008D6AA6C24EDE62D486C6A2C4CAC05AD83B
:1076200066D26AD06ECEC1495E8C97E4FF1F938408
:10763000A42A130A0A20938A7ADC17E9FF1F034958
:10764000A963B3872B0183C7070093F7F70FC9EF2F
:10765000B787004003C76700058BE310077C03C7AB
:107660006700118BE30D077E83C75700918B99E369
:107670006F10200317E7FF1F034727608547630448
:10768000F7006F10400197E7FF1FA386E74A97E7CF
:10769000FF1F2383073097E7FF1F2381073C97E7EE
:1076A000FF1F238F074697E7FF1F238C074697E7A7
:1076B000FF1FA383072E97E7FF1FA381073A97E7D2
:1076C000FF1FA38F074497E7FF1FA38C074497E78B
:1076D000FF1FA383074697E7FF1FA380075AB787BB
:1076E000004011476F0070779307190093F7F70F69
:1076F0003D476364F70617E7FF1F230FF75697E729
:10770000FF1F93876756CA9783C7070013071002A6
:1077100093F7F703638EE71E6366F70405446385FA
:10772000871CE38C07620947638EE710130700028A
:10773000E384E74EB7E700E03707400023A0E718EF
:1077400001000100629923000900FD1923A0E71040
:1077500093F9F90FE39309EEE5BD97E7FF1F238D3A
:10776000075071BF130730026388E70C63E8E71620
:1077700013074002638CE70A13070003E39CE7FA50
:1077800097E7FF1F9387474DCA9703C70700A14795
:107790001377F70FE31BF71483C7640097E6FF1F07
:1077A0002382F63897E7FF1F83C7771391C7FD57EA
:1077B00097E6FF1F2388F63697E5FF1F83C5D5118F
:1077C00097E7FF1FA380B73697E7FF1F83C7C71050
:1077D00013FB07089306000493F70706639FD74C33
:1077E0009307A009638DF51663EAB7129307F005B6
:1077F0006386F54A930750096384F52A014497E7A5
:10780000FF1F83C737321547E392E736B7E700E03B
:107810003707400023A0E71801000100B7860040A9
:1078200023808602130680FC6F00500EFD5717E779
:10783000FF1F2308F72EFDBDFD5717E7FF1F23018C
:10784000F72ECDBD17A50100130545CB977001009C
:10785000E780606F97E7FF1F93870740CA9703C4CD
:107860000700014B97ECFF1F938C8C1F1374F40FD0
:1078700017AD0100130D0DC963478B04294597709F
:107880000100E7804059854717E7FF1FA308F71C51
:1078900017E7FF1F2305871C17E7FF1F230EF72895
:1078A00037E700E0B70640002320D71801000100A9
:1078B000378600408347A60293F7370F2305F60269
:1078C0002320D71085BDB3876C0183C507006A8567
:1078D000050B97700100E780204F79BF854717E7B8
:1078E000FF1F230DF716B9B517E7FF1F1307C7369C
:1078F0004A970347070097E6FF1FA38FF60897E60E
:10790000FF1F238CE60817E7FF1F2307F7221DB58B
:10791000854717E7FF1F2301F70829BD9307400A92
:107920006389F5349307200B6384F5369307100AB7
:10793000E396F5EC838724000144E3D207EC97E754
:10794000FF1F83C797F993F63700638A061A054627
:10795000638AC62209466395C61A1D4755A217E5D4
:10796000FF1F034585F7C94797ECFF1F83CCFCF643
:1079700097E5FF1F83C585F617E4FF1F034414F640
:107980006315F510CD476392FC1093077008639C54
:10799000F5021307300FB7170E006308E400130752
:1079A000900DB7B704006314E40817E7FF1F232105
:1079B000F718BE8517A50100130545B5977001009E
:1079C000E780804025BD93078008639DF500B307DD
:1079D000804013F4F70FB7774600938787CDB3D76E
:1079E0008702E1B793079008639AF500B3078040D8
:1079F00013F4F70F91679387C766D5B79307A0086D
:107A0000639BF500B307804013F4F70FB7173D00F1
:107A100093870790E9B79307B008639AF500B30717
:107A2000804013F4F70F9167938797D04DBF93F57C
:107A3000F5078D47639BF500B307804013F4F70FFC
:107A4000B7975B00938707D859BF8947639BF500B9
:107A5000B307804013F4F70FB7770B009387071B2A
:107A6000BDBF8547639AF500B307804013F4F70F55
:107A7000DD67938767E3A5B7D28785F9B3078040B1
:107A800093F7F70FB3D7FA020DB797000000E7801E
:107A9000409FA285668597000000E780809EB9BB65
:107AA0009305610017E5FF1F034525E317E4FF1F5A
:107AB0000344B4E297000000E78040AD93057100F5
:107AC000228597000000E78060AC3C0017E7FF1FAD
:107AD000232AF716834761002304F10083477100CE
:107AE000A304F100894717E7FF1F230DF70283570F
:107AF000810017E7FF1F2311F7DE094409B315477B
:107B000093F64700B336D00093F78703850685C305
:107B10002146638BC7066146638AC7061306800247
:107B20006388C706130680036393C700914717E66F
:107B3000FF1F2301D60097E6FF1FA38DF6FE97E7F0
:107B4000FF1F238AE7FE17E7FF1F034727D9937616
:107B5000070497E7FF1F83C777D88DEE1377770C5D
:107B600093067008630CD7021377F7078D466312EC
:107B7000D70CB307F040B7955B0093F7F70F9385E9
:107B800005D849A81947ADBF854755B7894745B7B7
:107B90008D4771BF930670086311D7021307300F2A
:107BA000B7150E006389E7021307900DB7B50400FF
:107BB0006383E7021307700845BF9306800C6311C7
:107BC000D702B307F040B775460013F7F70F938756
:107BD00085CDB3D5E70297E7FF1F23ABB7F4D9BB39
:107BE0009306900C631CD700B307F04093F5F70F92
:107BF00091679387C766B3D5B702F1BF9306A00C10
:107C0000631DD700B307F040B7153D0093F7F70F9A
:107C100093850590B3D5F5027DBF9306B00CE315AF
:107C2000D7F4B307F04093F5F70F9167938797D098
:107C3000D9B78946631BD700B307F040B7750B006F
:107C400093F7F70F9385051BF1B78546631AD700A5
:107C5000B307F040DD6593F7F70F938565E35DBFEC
:107C6000D28535FBB305F04093F5F50FB3D5BA02D5
:107C70009DB783C72400C18B99C7854717E7FF1FAE
:107C80002305F7EAA5BE97E7FF1F238007EABDB6E5
:107C9000854717E7FF1FA300F7EA8DB63C0017E7FB
:107CA000FF1F2321F7FA0947930700032314F1006C
:107CB00097E6FF1F2388E6E62DBD63940756A94784
:107CC00063E5B742179701001307876C8A05BA95D9
:107CD0009C41BA97828717E4FF1F034414C0894C64
:107CE0006306940D63E68C0685476303F4089307E7
:107CF000F00F17E7FF1F0347E7E263F6E70017E718
:107D0000FF1F2301F7E297ECFF1F83CCACE1930741
:107D1000000413F4FC0F63F497011304000497E7C5
:107D2000FF1F938727F203AD070022862685EA8589
:107D3000B38C8C40229D97700100E78080FD97E70F
:107D4000FF1F238197DF97E7FF1F23ADA7EF45BCF8
:107D50008D47630CF40A9947E31BF4F897970100E9
:107D60009387876917E7FF1F232EF7ECA94751B7C1
:107D700017E7FF1F034767F097E7FF1F938787DC2D
:107D8000494697950100938525706306870097956E
:107D900001009385656B3E8597700100E78060F771
:107DA00017E7FF1F2320A7EAC947A1B797E6FF1FE0
:107DB00083C6A6EC054797E7FF1F9387A7D8639470
:107DC000E6023E851306700297950100938545698A
:107DD00097700100E780E0F317E7FF1F2324A7E671
:107DE0009307700239B73E8513063004979501005A
:107DF0009385456197700100E780A0F117E7FF1FA9
:107E00002322A7E493073004EDB597E5FF1F83C550
:107E1000C5AC179501001305A57097700100E780A8
:107E2000A0FA054D97EDFF1F83CD2DE597E5FF1FC8
:107E300083C5A5AA179501001305856E6398AD0B40
:107E400097700100E78040F897E7FF1F83C7E7A816
:107E5000B5CBE36EF4E81794010013042467638C38
:107E6000B701179401001304E46663869701179421
:107E700001001304A467228597700100E780E00DDC
:107E80001375F50F93071500860717E7FF1F230BE0
:107E9000F7CA8D4717E7FF1FA306F7CA97E7FF1F2B
:107EA000938747CA0147BE861376F70F8907636534
:107EB000A60297E7FF1F23A7D7D897E7FF1F83C71F
:107EC00067C805BD979701009387475917E7FF1FBC
:107ED000232AF7D6914731BD3306E4000346060056
:107EE000A380070005072380C7007DBF97700100AE
:107EF000E78080ED97E7FF1F83C7279EE1D7E36800
:107F0000F4DE1794010013046459638CA7011794DD
:107F10000100130424596386970117940100130488
:107F2000E459228597700100E78020031375F50F4F
:107F300093071500860717E7FF1F2305F7C08D4736
:107F400017E7FF1FA300F7C097E7FF1F938787BFBF
:107F50000147BE861376F70F8907E37CA6F4330644
:107F6000E40003460600A380070005072380C7003E
:107F7000D5B797E5FF1F83C54596179501001305F3
:107F8000E55A97700100E78020E497E7FF1F83C759
:107F900037BB93E7470017E7FF1FA303F7BA83C771
:107FA000240017E7FF1FA30BF7B889B81795010046
:107FB0001305055997700100E780E0F897E7FF1F68
:107FC0009387C7B783C7070017E7FF1F2306F790FC
:107FD00017E4FF1F034404B5333480000DB0179538
:107FE00001001305255797700100E780C0F597E75A
:107FF000FF1F83C7F7B493E7070117E7FF1FA3012C
:10800000F7B483C7240017E7FF1F2309F7B26FF007
:10801000EFFE179501001305255597700100E780C5
:1080200080F203C704007D8B51EFB787004003C780
:1080300067021377C70B136727002383E70203C781
:10804000A7021377C70B136727002385E70203C72F
:10805000E7021377C70B136727002387E70203C7DD
:1080600027031377C70B136727002389E702854788
:1080700017E7FF1F2302F79217E7FF1F2300F79E62
:1080800017E7FF1F230EF7A817E7FF1F230BF7A81B
:1080900097E7FF1FA382079097E7FF1FA380079C26
:1080A00097E7FF1FA38E07A697E7FF1FA38B07A6DF
:1080B00097E7FF1FA38207A897E7FF1FA38F07BAC1
:1080C0006FF0CFF389476312F70297E7FF1F83C76B
:1080D000E7809146638CD70863E0F604638EE70C73
:1080E0006369F70A05476380E70EFD5717E7FF1F2F
:1080F000A30AF7A237074000B7E700E023A0E7187C
:1081000001000100B78600401306F0FC2381C6027F
:1081100023A0E7106FF00FE2130720086382E7083F
:108120006362F70213071008E391E7FC378700400A
:108130008347670293F7C70B93E727002303F702F0
:108140006FF0CFEB130730086389E702130740088D
:10815000E39DE7F8378700408347270393F7C70B72
:1081600093E727002309F7026FF04FE937870040B4
:108170008347270393F73707F5B7378700408347CF
:10818000E70293F7C70B93E727002307F7026FF087
:10819000EFE6378700408347E70293F73707F5B7E5
:1081A000378700408347A70293F7C70B93E7270061
:1081B0002305F7026FF08FE4378700408347A7025B
:1081C00093F73707F5B7378700408347670293F780
:1081D0003707ADB7179501001305053A97700100F1
:1081E000E78060D697D7FF1F2388076ED5B3179512
:1081F00001001305653997700100E780C0D497D757
:10820000FF1F239B076C97E7FF1F9387A79103C46A
:108210000700894763F3870009441374F40F6FF074
:108220000FDE13070002E392E7EC631B0B0A638F78
:10823000F500930720026383F508179501001305E5
:10824000253897700100E78020B845B517950100E3
:108250001305453497700100E780E0CE0144179D77
:108260000100130D6D34A14CB387840083C5070052
:108270006A85050497700100E78000B5E31694FF56
:10828000178501001305057897700100E780A0CBE2
:1082900017D4FF1F0344846401E897D7FF1F238F7F
:1082A0000760014B6FF0AFD58947E310F4E48547D1
:1082B00017D7FF1F2304F7606FF04FD417D6FF1FA7
:1082C0000346B66197D5FF1F83C525611795010049
:1082D0001305052E97700100E78000AF6FF00FD2F5
:1082E0006380F50693071002E399F5F497D5FF1F15
:1082F00083C5C55E179501001305852D9770010094
:10830000E78080AC97E7FF1F23AE979297E7FF1FA8
:1083100093870782944383D7470017E7FF1F0347DC
:10832000878117D6FF1F2329D65A1D4497D6FF1FD2
:108330002396F65A97D7FF1F2383E75A6FF02FCC67
:1083400097D5FF1F83C58559179501001305C529CA
:1083500097700100E78040A797D7FF1F238007563B
:1083600097D7FF1F239A07566FF02FF92547638F82
:10837000E7C89946378700406394D70223008702F5
:10838000B7E700E0B706400023A0D71801000100BE
:10839000130600FC2301C70223A0D7106FF08FB98A
:1083A0009306100A639FD70023008702B7E700E017
:1083B000B706400023A0D71801000100130680FC77
:1083C000D1BF9306A009E381D7FE9306400AE38D4F
:1083D000D7FC93062002639DD700B7E700E0B706FD
:1083E000400023A0D7180100010023008702F9B73D
:1083F0008546E384D7FE93070008E300FBFEB7E75A
:1084000000E0B706400023A0D718010001001306C2
:1084100020FC23008702BDBF17D7FF1F03479770BB
:108420006302F71E63E7E70295476300F710994779
:10843000630AF704B786004023800602B7E700E02E
:108440003707400023A0E718010001001306A0FC35
:1084500075B99307F005630AF7009307500963069F
:10846000F70093071002E317F7FCB7E700E03707C0
:10847000400023A0E71801000100B7860040130662
:1084800020FC69B117DBFF1F034BCB699307000486
:108490005A8D63F46701130D000497D7FF1F93876C
:1084A000677A83AC07001374FD0F2286E685268564
:1084B00097700100E780E085B3078B40669417D77B
:1084C000FF1F2301F76697D7FF1F23AD8776B78776
:1084D0000040630C0B022380A703B7E600E03706D9
:1084E000400023A0C6180100010003C7270213475C
:1084F00007042381E70203C727021377C70F2381ED
:10850000E70223A0C6106FF0EFA22380070237E72F
:1085100000E0B70640002320D71801000100130631
:1085200020FC2381C7026FF0AFB937870040834733
:10853000370097D6FF1F83C6766093F70708D58F5D
:10854000A301F700B7064000B7E700E023A0D71863
:10855000010001001306A0FC35BD97D7FF1F9387CC
:10856000A76FCA9783C7070093F7F70FC1CF97D7B5
:10857000FF1F83C78770D9E717D7FF1F0347975A95
:10858000930700026310F70883AD040017DDFF1F97
:10859000034DCD3497DCFF1F83CC5C3417DBFF1F0A
:1085A000034BEB33E6876A87DA866E8697D5FF1F23
:1085B00083C5C53017950100130585049770010028
:1085C000E780808097D7FF1F23A4B75797D7FF1F57
:1085D0002382A75797D7FF1FA38E975597D7FF1FC3
:1085E000238B675597D7FF1FA389872CB7E700E038
:1085F0003707400023A0E71801000100B7860040BC
:108600006FF04FA2B7E700E03707400023A0E7185C
:1086100001000100B786004015BD97D6FF1F83C635
:10862000C6650547639CE60429472381E70209479D
:108630002383E7022385E70297D7FF1FA38E074E08
:1086400097D7FF1FA38B0762B7870040A38107005E
:1086500017D7FF1FA304074E05472383E700B64043
:10866000264496440649F259625AD25A425BB25B9A
:10867000225C925C025DF24D616182802947238118
:10868000E70209472383E7022385E7022387E702FE
:108690002389E70255B717D7FF1FA300F7226FE022
:1086A0001FFF854717D7FF1F2308F72E17D7FF1F78
:1086B0002306F73A17D7FF1F2304F74617D7FF1FE4
:1086C0002301F7466FE0BFFE854717D7FF1F23053D
:1086D000F72C17D7FF1F2303F73817D7FF1F2301E6
:1086E000F74417D7FF1F230EF74217D7FF1FA30525
:1086F000072A17D7FF1FA303073617D7FF1FA301AA
:10870000074297D7FF1FA38E07408280411106C6FC
:1087100097000000E78080FBB787004023800700B8
:10872000130740FC2386E7001307C004A386E70075
:1087300017D7FF1F1307471A2398E70017D7FF1F04
:108740001307871D239AE70017D7FF1F1307072971
:10875000239CE70017D7FF1F13078734239EE700EA
:1087600029472381E70209472383E7022385E7029C
:108770002387E7022389E702A3810700930600F815
:10878000A380D700930690022380D700FD56238351
:10879000D7002381E7009306000537E700E0230BAD
:1087A000D740B70640002320D71003C71700136730
:1087B0001700A380E700B24097D7FF1F2390073828
:1087C00041018280411106C697000000E78000F059
:1087D000B787004023800700130700FC2386E700CB
:1087E0003147A386E70017D7FF1F1307E70E23982B
:1087F000E70017D7FF1F13072712239AE70017D7A1
:10880000FF1F1307A71D239CE70029472381E702C9
:1088100009472383E7022385E702A3810700930624
:1088200000F8A380D700930690022380D700FD565E
:108830002383D7002381E7009306000537E700E094
:10884000230BD740B70640002320D71003C71700DB
:1088500013671700A380E700B24097D7FF1F239F3D
:10886000072C41018280F1679387072017D7FF1FEC
:108870002320F72C854717D7FF1F231DF72AA14771
:1088800017D7FF1F2309F72A97D7FF1FA385072AAA
:1088900097D7FF1F2382072A97D7FF1F238007023E
:1088A00097D7FF1FA38B0700814717D5FF1F13051D
:1088B0002501FD5517D6FF1F130646012947B306AC
:1088C000F5002380B600B306F60023800600850776
:1088D000E397E7FE97D7FF1FA387072497D7FF1FCC
:1088E000A385072497D7FF1F2380072497D7FF1F4F
:1088F000238B072297D7FF1F238A072297D7FF1FB3
:10890000A384072297D7FF1F23810722814717D609
:10891000FF1F130666334147B306F60023800600A7
:108920008507E39BE7FE828017D7FF1F0347E734E5
:1089300085476316F700170300006700E3E8170395
:1089400000006700E3DC411122C406C617D7FF1FF1
:108950000347A73285472E8613F4F50FAA856317C0
:10896000F70417D5FF1F1305650B97600100E7801B
:10897000403A97D7FF1F2383070EB7870040238411
:108980008702B7E600E03706400023A0C6180100C2
:10899000010003C7A7021377C70F2385E702B24080
:1089A000224423A0C61001454101828017D5FF1F34
:1089B000130585FA97600100E780A03597D7FF1F60
:1089C000238C07FCB787004023828702B7E600E0CC
:1089D0003706400023A0C6180100010003C7670244
:1089E0001377C70F2383E7025DBF411106C69700C7
:1089F0000000E78080E7B2404101170300006700F4
:108A0000E3F2411106C697F0FFFFE78080BF97D7DA
:108A1000FF1F83C777F8A1CB97D5FF1F83C5E5F765
:108A200089C917D5FF1F130565F797E0FFFFE7809A
:108A3000204897D7FF1FA38107F697D7FF1F238DE5
:108A4000070E37E700E0B70640002320D7180100E3
:108A50000100378600408347660293F7370F2303F0
:108A6000F6022320D710B2404101828041C9D9C506
:108A700097D7FF1F83C7870CD1C3011122CC4AC8E7
:108A80004EC656C25AC006CE26CA52C42E89AA89DC
:108A90000144930A0004371B030063772403B307E0
:108AA0008940C207C183BE8463F4FA0093040004C2
:108AB000C204C180130A1BD497D7FF1F83C7C7ED19
:108AC0009DE37D1A631C0A00F2406244D24442498D
:108AD000B249224A924A024B0561828097F0FFFF19
:108AE000E78020B2D1BF338589002694A685420451
:108AF00097000000E78060E5418045B78280411122
:108B000006C622C429C12E8495C997D7FF1F83C7E3
:108B1000E70295CB97D7FF1F83C707E88DC71307D9
:108B20000004AE876374B700930700041394070131
:108B30004180A28597000000E78020E12285B240B5
:108B40002244410182800144D5BF97D7FF1F9387FC
:108B5000671618429C4383D645000345070083C52A
:108B6000C700035646006396A50083D5E700638DD2
:108B7000D502011106CE2386A7002397D700B7059B
:108B8000CF00DC4B9385757D05077D162EC2230033
:108B900001003AC42316C1002317D10099C30A85E6
:108BA0008297F240056182808280DC4DDC4B81CF70
:108BB000B7E70400904503A38705914517D5FF1F2C
:108BC0000345850F028382806D713C083EC6B7075E
:108BD000E500232291103EC8AA843C083285232652
:108BE00011103ECA23248110232021112E89973091
:108BF0000000E780C0672A84979501009385C5A38C
:108C0000177501001305857B97600100E780C01B85
:108C1000A285179501001305A5B297600100E780B2
:108C2000A01A294597600100E780E01EB705CB0038
:108C30009385757D680097100000E780406DA285E0
:108C4000680097300000E780E054014781467000DB
:108C5000CA85268597200000E780C09005CD2A842C
:108C6000979501009385459D1775010013050575BE
:108C700097600100E7804015A28517950100130554
:108C8000E5AC97600100E78020142945976001005A
:108C9000E78060188320C1100324811083244110D1
:108CA000032901105161828097D7FF1F93878700A6
:108CB00018429C43797122D406D60348070083C822
:108CC00007012A8483D645000355460063960801B0
:108CD00083D82701638DD8022388070105072399CC
:108CE000D7003708CC00DC4B1308787D3ACC13074B
:108CF000F5FF42CA23080100231EE100231FD10013
:108D000099C7080832C62EC482973246A2452285EA
:108D100097000000E78080EBB250225445618280CA
:108D20006D713C083EC0B707E5003EC23C083EC43A
:108D300023261110232481102322911023170100D0
:108D40002318010023190100231A0100231B01002D
:108D500097A7FF1F83D7C76B99E3C167FD1723163A
:108D6000F10097A7FF1F83D7C76A91EB97D7FF1F23
:108D7000938747F49C439C43DC4783D7070017A4A1
:108D8000FF1F1304E468584C2317F1008357440075
:108D9000484B2318F10031E1979501009385C59068
:108DA000177501001305856197600100E780C00118
:108DB000179501001305859097600100E780C000BA
:108DC000294597600100E78000058320C110032436
:108DD0008110832441105161828097A7FF1F83C7B0
:108DE000976389EBB7E70400BC5782975C4C23AAD2
:108DF0000700E1BFFD1797A6FF1FA38EF66003567D
:108E00000701834704014C470A85230BF100973083
:108E10000000E780403597D7FF1F9387A7E99C4361
:108E20000147814688430A866C0097100000E7805E
:108E30006073AA8429C1979501009385E58617750B
:108E400001001305A55797600100E780E0F7A685AC
:108E5000179501001305458797600100E780C0F66C
:108E6000294597600100E78000FB584CB7E70400F4
:108E7000BC57484B9DBF97A7FF1F83C7D759F5D74E
:108E8000B7E70400BC4F1044854517D5FF1F0345C5
:108E9000A5E282971DBF5C4EDC4BB9CFB1CD41112D
:108EA00022C417750100130565512E8497850100B2
:108EB0009385C57D06C697600100E780E0F0A28536
:108EC000179501001305058397600100E780C0EF47
:108ED000294597600100E78000F4B7E704002244C9
:108EE000B24003A3870517D5FF1F0345E5DC130632
:108EF00040069145410102838280411122C417A49A
:108F0000FF1F1304A44E1C4C06C689C7DC4399C33B
:108F10004C488297584CB7E70400BC57484B82979F
:108F20005C4CB240224423AA07004101828017A76B
:108F3000FF1F1307A74D834707009306F00B850714
:108F400093F7F70F63E9F60097A6FF1F2380F64C0F
:108F5000034507008280930700F8FDB7835745005B
:108F60006386071001114AC817A9FF1F1309494A50
:108F700052C4032AC90106CE22CC03274A0126CABD
:108F80004EC656C2F15735E31307D00DFD57636E39
:108F9000C704B7E9040083A709072A8413058600DC
:108FA00042054181B284AE8A8297232AAA00032512
:108FB000C9015C49A9E7978501009385256B177561
:108FC00001001305A53F97600100E780E0DF1785EA
:108FD00001001305657A97600100E780E0DE29450E
:108FE00097600100E78020E3DD57F2406244D244FD
:108FF0004249B249224A924A3E850561828093875E
:109000004400B705CF002319F5009385757D310520
:1090100097100000E780A02F0325C9018345640055
:10902000310597300000E780E0160325C901268648
:10903000D685310597300000E780E0127146A285A1
:109040004A8597600100E780C0CC504419CA83A7C5
:109050008905854517D5FF1F034505C682978147BA
:1090600069B797000000E780E0CBD5BFFD573E858C
:109070008280411126C297A4FF1F93846439D84C83
:1090800022C437E404003C54484B06C68297DC4CAB
:109090000323C4052244B240924423AA070017D5F3
:1090A000FF1F034565C1854541010283411126C269
:1090B00097D4FF1F938404C09C4006C622C44AC0B4
:1090C000D5C3DC43C5C35CC12300B5002A849785A2
:1090D00001009385E554177501001305252E97604F
:1090E0000100E78060CE294597600100E780A0D2AB
:1090F0009C4023A4070023A2070097A7FF1F938784
:10910000E72EDC4FDC4B91C7295597000000E78024
:1091100000DF97A7FF1F9387A72FDC4FDC4B89C782
:1091200097000000E78020F537E904008327C90590
:10913000894517D5FF1F034525B882978327C905A1
:10914000914517D5FF1F034525B782979C4003A380
:1091500047016309030022852244B2409244024938
:1091600041010283B240224492440249410182807B
:109170000111328506CE22CC26CA2E8497300000FB
:10918000E780E00EAA84978501009385A54C1775AA
:1091900001001305A52297600100E780E0C20307E4
:1091A00084000356640083554400A6861785010099
:1091B0001305455697600100E78000C12945976077
:1091C0000100E78040C597A7FF1F83C78722639DE3
:1091D0009700014597000000E78060D281450A852D
:1091E00097000000E780C0ECF2406244D244056181
:1091F00082806D7123248110232611102322911067
:1092000093F745002E84638707143C083EC0B707D8
:10921000E5003EC23C083EC42317010023180100AC
:1092200023190100231A0100231B010097A7FF1F28
:1092300083D7C71B99E3C167FD172316F10097A7D2
:10924000FF1F83D7C71A91EB97D7FF1F938787A676
:109250009C439C43DC4783D7070017A7FF1F1307D6
:10926000E7182317F100544F835747002318F100E4
:10927000DC4AA1E797850100938505421775010037
:109280001305C51397600100E78000B4178501003E
:109290001305C54297600100E78000B32945976038
:1092A0000100E78040B7134544008320C110032428
:1092B0008110832441105161828097A7FF1F83C7CB
:1092C00057132555D9C3FD1717A6FF1FA303F61281
:1092D00003D6060183470701CC460A85230BF1001C
:1092E00097300000E78020E897D7FF1F9387879C7F
:1092F0009C4317A7FF1F1307670F978601009386EC
:10930000E63E88430A866C0097100000E7808025BF
:10931000AA8451D9978501009385053817750100F6
:109320001305C50997600100E78000AAA685178587
:1093300001001305653997600100E780E0A8294521
:1093400097600100E78020AD268597000000E78048
:1093500000BB91BF93F725009DC7B7E70400BC474A
:109360004146814528088297255597000000E780EF
:1093700000B928089305F00F97000000E78040D35C
:10938000134524001DB793F71500014599DF970099
:109390000000E78020991345140001BF5C4D411186
:1093A00006C688C317D7FF1F2326F790B7E7040028
:1093B00083A70708170500001305E5E38297B2406D
:1093C00097D7FF1F238AA78E014541018280011193
:1093D0003335A000A307A100B7E7040083A7471710
:1093E00006CE1306F1008545130550308297F240F2
:1093F000056182808280411122C406C697D7FF1F73
:1094000083C7078D014489EF97B7FF1F83C757E3D1
:10941000054499E717B4FF1F034484E21344140082
:10942000228597000000E780C0FA17850100130528
:10943000A53F09E417850100130505402244B24009
:1094400041011763010067002398797122D4A30FAB
:10945000010037E404008327841726D24AD006D6B9
:10946000AA842E89130550309305F10132C68297E4
:1094700032468347F10193150601C18185CB014531
:109480002EC697000000E780C0F483274417B2453A
:109490004A8626858297054597000000E78060F39D
:1094A000B250225492540259456182808327441756
:1094B0004A8626858297EDB741119397050122C40C
:1094C00006C626C2C1872E8463D40702B7E404000F
:1094D000FC5417A5FF1F0345A5F6829719C1BC547C
:1094E00082972165218DB2402244924441018280BD
:1094F00093F715008DC7B7E7040083A7471A17A68F
:10950000FF1F1306E6F297C5FF1F9385A57B17A5DE
:10951000FF1F0345E5F2829713451400E9B793F75F
:10952000250099CFB7E70400BC4F130600648945B6
:1095300017A5FF1F0345C5F082971345240065B7A3
:1095400093F7850085CF97C7FF1F83C7277985E7E6
:10955000B7E7040003A8871A1307401F97A7FF1F48
:1095600083C707EE814613064006994517C5FF1FBE
:1095700003554576029813458400B5B793F7450027
:109580000145B5D3B7E4040083A7041817C5FF1F2E
:10959000035545748297BC4C13060064914517A58A
:1095A000FF1F0345E5E98297134544002DBF97C788
:1095B000FF1F83D727726398A70217C7FF1F231CBB
:1095C000B77017C7FF1F2319C77017C7FF1F2316D0
:1095D000D7702E86178501001305852CBE8517537D
:1095E00001006700637E178501001305E52C1763F2
:1095F0000100670043950357450097C7FF1F83D7B6
:10960000676D631EF704C1674111F91722C417C7BC
:10961000FF1F2321F76C37E4040097C7FF1F23AD1A
:10962000076A97C7FF1FA385076A97C7FF1F23878E
:10963000076A7C4C06C6894517A5FF1F034545E010
:1096400082977C4C914517A5FF1F034565DF8297E4
:109650002244B240410117030000670003DA178576
:10966000010013056525176301006700C38D7D1593
:10967000954763E2A71C17870100130767190A05BE
:109680003A951C41011122CC06CEBA972E848287CE
:10969000178501001305C52297600100E780A08AA5
:1096A000A1A203C7250099476311F7022E859700F1
:1096B0000000E78080F483456400178501001305EE
:1096C000252197500100E780207097B7FF1F23895D
:1096D00007B617850100130565217DBF03C7250067
:1096E00095476319F702C16717C7FF1F0357875EC6
:1096F000F91703D5A5006309F702B7E7040083A7AC
:10970000C7178297178501001305451F9760010051
:10971000E7806083854717B7FF1F2303F7B21785DC
:109720000100130525208DBF97C7FF1F2394A75A5B
:1097300083D7E50097C6FF1F239FF65883D70501FF
:1097400097C6FF1F239AF65883D7250197C6FF1F98
:109750002395F65897C7FF1FA38C0756631BE50296
:10976000B7E70400BC4F096613060690A14517A58C
:10977000FF1F0345E5CC82970356E4008355A40000
:10978000178501001305C51897500100E780C063D5
:1097900051B79307700F2316F100B7E7040083A7B2
:1097A000870D17A6FF1F0346A6C96C0082974DF9C7
:1097B000854717C7FF1FA30DF7505DB71785010039
:1097C00013050517D1BD83C5250091476392F502A6
:1097D000178501001305451797500100E780A07613
:1097E00097000000E78060C1F2406244056182801A
:1097F00099476392F502228597000000E780E0DF39
:1098000083456400178501001305850C97500100FE
:10981000E780805BD1BF9547639AF50083471400CA
:10982000E1F31785010013056514BDB51785010027
:1098300013054514E1BF82800111B7F50700300020
:109840008146E105194506CE9790FF1FE78060F934
:109850008347C1000347D100B7562D47A207D98FD0
:10986000938676D517A7FF1F1307C7BE14C3B73655
:10987000302D9386360354C39566938676742314ED
:10988000D7009306D0022305D70013D6C7009786CA
:1098900001009386A6FD36960345060013D6870081
:1098A0003D8A36968345060013D647003D8ABD8B18
:1098B0003696B69783C607000346060097A7FF1F94
:1098C0009387C7BAA305A7002306B700A306C7005E
:1098D0002307D700A3070700A386A7002387B700A5
:1098E000A387C7002388D700F24005618280411119
:1098F00006C697000000E78060F4B7E7040083A77E
:10990000871417A6FF1F1306E6B4D54501458297B5
:10991000B240694697A5FF1F938545B51305703082
:10992000410117030000670083B261712324811A8B
:1099300037E40400832704082326111A2322911AEE
:109940002320211B232E311917050000130505B70D
:10995000829717A9FF1F1309A9AE994785442300D1
:10996000A900231CF10097850100938525EF93073B
:10997000400617750100130565A4231CF108230890
:10998000910097C9FF1F9389A9DF97500100E780D5
:10999000A04383D5090017850100130525EB9750D7
:1099A0000100E7806042294597500100E780A0460A
:1099B00003D50900896997000000E78020E8832724
:1099C00044171008854513055030829783274417A4
:1099D00017A6FF1F130686A9E94513057030829765
:1099E0008327441717A6FF1F1306C6A5B545130501
:1099F000603082978327441730088945130510315A
:109A000082978327441730098945130520318297AF
:109A100083274415938509900D4582978327441524
:109A20009385099011458297A30591002306910023
:109A300002CD23080100230C01008327841630097E
:109A40009145130570408297832784161306B10051
:109A5000854513050040829783278416700085454D
:109A60001305104082978327841630088545130517
:109A7000204082978327841610088545130550409F
:109A80008297832704157D558297832744137D553C
:109A900082977D5597A0FFFFE78080BD8327440C08
:109AA000829797A0FFFFE780E0988327841417A68A
:109AB000FF1F1306269AD54501458297894713064D
:109AC000700F814528092306F1009780FFFFE7808A
:109AD00000648D471306000881452808230CF1080F
:109AE0009780FFFFE780A0629147230CF100976702
:109AF00001009387277E984383C747003AC8230A0B
:109B0000F10097D0FFFFE78080A3700085450545F1
:109B100097A0FFFFE780E0BC30099305700F09456F
:109B200097A0FFFFE780E0BB3008930500080D45D4
:109B300097A0FFFFE780E0BA10089545114597A070
:109B4000FFFFE78000BAC16717C7FF1F1307871819
:109B5000F9171CC32322070017A5FF1F1305058E45
:109B600097A0FFFFE780C0B68327C41D17C5FF1F5E
:109B70001305C51482973C48034509008545829723
:109B80008320C11A0324811A8324411A0329011A4C
:109B90008329C1195D618280C16717C8FF1F0358FF
:109BA0006813F9176301F8083DCDB5CD011126CA38
:109BB000B7E4040083A7841222CC2E862315B100BB
:109BC00006CE2A8401478146ED45428582972AC602
:109BD00011ED178501001305A5CA97500100E78014
:109BE0008036F2406244D24405618280FC440356D0
:109BF000A100A28582972C0017C5FF1F0355850D74
:109C000097A0FFFFE78080B969DD17850100130584
:109C100065C897500100E780003383A7C412ED4563
:109C2000280082977DBF82800DC5854717A7FF1F3B
:109C3000A30FF78097A7FF1F238C0780354697A5B2
:109C4000FF1F938525801305603017030000670010
:109C500003809797FF1FA38C077EE9BF97C7FF1F5D
:109C600083C7C707A9EFC16717C7FF1F0357870639
:109C7000F9176306F7044111854722C417C7FF1F70
:109C8000230EF70437E404007C4C06C6A145179563
:109C9000FF1F0345E57A82970323841A2244B240CA
:109CA0009797FF1F83C7C77917C5FF1F0355850205
:109CB0001307401F81463146994541010283828046
:109CC0006D712324811023261110232291103284D8
:109CD00001CD8947630AF5028320C1100324811056
:109CE000832441105161828017850100130545C905
:109CF000AE8497500100E7800025A285268597C095
:109D0000FFFFE780E0A1C9BFB7E70400FC472800D8
:109D1000829717850100130565C797500100E780FA
:109D200080228347810039C41307000B6380E70258
:109D30001387A7051377F70F8D4663EDE602A2851B
:109D4000280097C0FFFFE780A01179B78547E3F5AA
:109D500087F8834591001775010013052599B335E0
:109D6000B00097A7FF1F2381B73697500100E78007
:109D7000A0059DB703479100A207D98F3567130748
:109D8000D7556385E7086368F7022D671307B75552
:109D90006387E70631671307C755638AE7042967B6
:109DA0001307A7556394E702A285280097C0FFFF19
:109DB000E780604915B739679306E7656381D7087F
:109DC00063E9F6001307E7556384E706A2852800D8
:109DD0003DB73D679306F755638AD7061307F766C5
:109DE000E396E7FE97C0FFFFE7800064F5B5014604
:109DF000A285280097C0FFFFE7802032F1BDA28531
:109E0000280097C0FFFFE7804042F9B58947E3F596
:109E100087EC97000000E780A0E49305E4FFC2050B
:109E2000C1811305A1009790FFFFE780C0396DB590
:109E3000A285280097C0FFFFE780E04171BDA285A1
:109E4000280097C0FFFFE780A04C79B597C0FFFFBF
:109E5000E780405751B5C16717C5FF1F035585E718
:109E6000F9176307F500B7E7040003A3C7170283D8
:109E70008280854717C7FF1F230CF7E4014517F3BE
:109E8000FFFF670003551783FFFFE702A3232A8420
:109E900008452E89B28919C900C19715000093851C
:109EA000A586610597300100E780200581447D5A31
:109EB00097100000E780E03963C7A404814497103D
:109EC0000000E780003A63C8A40497C7FF1F938788
:109ED00027E19C43DC47B307F94091872302F40054
:109EE000638309048327C900B307F4409587A3025D
:109EF000F4001C4C89C79C4799C32285829717831D
:109F0000FFFF6700631F5C44139714008504BA9732
:109F10002390470171BF1C48139714008504BA971A
:109F20002390070069BF832789000547B307F440E2
:109F30009587A302F40083570400638EE7028DC364
:109F400009476384E7040D47E395E7FA9787010023
:109F5000938787F61CCC978701009387E7F611A8B3
:109F6000978701009387C7BC1CCC97870100938714
:109F700027BD5CC8BDBF97870100938767A81CCC2D
:109F8000978701009387C7A8EDB79787010093874C
:109F900067F71CCC978701009387C7F7D9BF95E572
:109FA0001783FFFFE702A31300461844834794007A
:109FB00075839D8B6317F70097100000E78060B4EE
:109FC00048C41783FFFF6700C31382801783FFFF16
:109FD000E702430F13893500C16442094111AA8980
:109FE0000144F11413590901054A2EC697100000C7
:109FF000E7802026B2456348A4000145410117834C
:10A00000FFFF6700630F83A7090013171400BA97B7
:10A0100083D707006388B7006394970063742A01AD
:10A020000504E1B70545D9BF1783FFFFE702A30881
:10A03000AA892E89328BB6843A8ABE8A97A00000FC
:10A04000E780C0FE71C9268597200000E780C00C1C
:10A050008D4763E7A7007D551783FFFF670023093E
:10A0600083DB440097100000E780A0242A84971027
:10A070000000E780402593077400314433058502D2
:10A0800063CDA70297100000E780A0229710000080
:10A09000E78020222A8497100000E780C0229307DF
:10A0A000740031443305850263C3A7049710000090
:10A0B000E78020209307450029A897100000E7803B
:10A0C0008020330585021307F0179307C017E35F5D
:10A0D000A7FA2D55E3C277F963040B02D6865286A0
:10A0E000A6854A8597200100E780C0BDB5B79710C7
:10A0F0000000E780401D330585029307C5FFD1BFEF
:10A10000832749001385C90083D5270097000000E5
:10A11000E78000EC61F581B769553DBF97C7FF1F28
:10A120002392A7BC97C7FF1F938787BB90438147A4
:10A130000C463307F500420741836393B7008280E2
:10A140005446139847008507C2962390E600D5B77A
:10A1500097C7FF1F9387C7B89C4303C587008280BA
:10A1600017C5FF1F035505B882801783FFFFE7025D
:10A1700003F7C1671387D7FF630BE502636AA70084
:10A18000F1176300F50201451783FFFF670063F7CE
:10A190001387E7FF6302E502FD171D8D13351500D8
:10A1A000E5B797500000E780602A7D15C5BF97503E
:10A1B0000000E780E0FED5BF97500000E78000FD7B
:10A1C000EDB71783FFFFE70283F14111AA84014431
:10A1D0002EC697100000E780C008B2456348A4006F
:10A1E000014541011783FFFF6700A3F19C48131548
:10A1F00014003E9583570500E385B7FE0504C9BFEB
:10A2000003485500814693F7F60F63E50701814740
:10A210003E858280584593975600BA9703D727000A
:10A220006316B70003D70700E304C7FE8506E1BF46
:10A230008346450001479377F70F63E4D7008147D2
:10A2400011A81C45131657000507B29703D607003F
:10A25000E313B6FE3E8582801783FFFFE70283E6A5
:10A2600093170501C18797CAFF1F938A6AA7635B8B
:10A27000F00883A70A00C0479C4703570400198DC4
:10A28000420541816368F500014422851783FFFF81
:10A29000670083E612052A94CDBFDC47139449007A
:10A2A000014A3E94834744006341FA02014A8347CE
:10A2B00054006349FA028509C20993D9090183A7A9
:10A2C0000A009847E3EBE9FCC1B71C4413195A0094
:10A2D000A6853E994A8597000000E780C0EE05E11B
:10A2E000050AC9B75C4413195A00A6853E994A85E8
:10A2F00097000000E78020ED19E1050A4DBFE30C4F
:10A3000009FA61B7AA8481495DBF1783FFFFE7029D
:10A3100003DD1C452A8481E79307C5001CC51C4446
:10A32000231204001CC09307F00F63EDB70093F5F0
:10A33000F50F228597200000E780C0E51783FFFF17
:10A34000670023DC93940501C167C18063F9F500C0
:10A35000A685228597200000E780E0E8C5B7C18187
:10A3600093F5F50F228597200000E780A0E2A685EF
:10A37000228597200000E780E0E3C9B797C7FF1F59
:10A3800093870796884382801C4599C797C7FF1F0C
:10A3900023A8A794014582807D55828097C7FF1F1F
:10A3A00093870794984383474500484792073E9513
:10A3B00082801783FFFFE70283D2617100451C187A
:10A3C0003EC6B70780013EC81C183ECA83574400EA
:10A3D00002CE02D002CC231EF100834784002A89DA
:10A3E00002D22301F1023C083ED402D697000000BD
:10A3F000E78000FB835705002316F1029750000009
:10A40000E78000C82307A1025C4003556400F18384
:10A4100013F717008347F10252055181F99BD98F39
:10A42000A307F10297100100E780207939CDAA84B3
:10A430000355050097A00000E78020C083D70400E3
:10A440002AD26800231CF10083D72400231DF100C9
:10A450001C4803D647008C4397200000E780A0D01B
:10A460008347B400CA86177601001306E6528117A7
:10A47000A305F4006C00481097200100E780808459
:10A480005D611783FFFF6700C3C72155D5BF1C451A
:10A49000B1CF03C5A700894613576500630BD702E8
:10A4A0008D46630ED70285466300D7021307400628
:10A4B0003305E50203C7B700418B15CB83C7B7004F
:10A4C000BD8B3355F54082801375F5031307803E2D
:10A4D000C5B709671375F50313070771D1BF372790
:10A4E00009001375F5031307077CD9B7014582806E
:10A4F0001783FFFFE702A3BE03A98500630C0904CD
:10A500008347B900AE8493F7070E85C303459900CE
:10A51000930520030D810505B305B5028844610547
:10A5200097300100E78080AD35A02E8597000000B0
:10A53000E78020F62A8419CD97000000E780605C50
:10A540008325C900B307B54063FA87002E94B3058D
:10A55000A440E9F51783FFFF6700A3BA85457DBFD7
:10A560001783FFFFE702A3B72A8403D50500011173
:10A5700032C636C43AC22EC002CA02CC02CE97A05E
:10A580000000E78080AB82452ACA22852ECC970046
:10A590000000E780E0E003570500231EE10097502C
:10A5A0000000E780E0ADA24632469247230FA100AB
:10A5B00036874C08B2862285014697000000E78066
:10A5C000E0A605611783FFFF6700A3B31783FFFFB2
:10A5D000E702E3B061711C183EC6B70780013EC8B0
:10A5E0001C183ECA3C0800453ED4AA8402CC02CEC8
:10A5F00002D002D202D697000000E78060DA8357CB
:10A60000050035592316F10297500000E78040A756
:10A610002307A10209C48357440081EB21594A85CD
:10A620005D611783FFFF6700C3AD035564005205EA
:10A63000518197100100E78040582A8965D18347EE
:10A64000B40093F7070E99C71305840197300100F2
:10A65000E780009D83574400231EF1008347840058
:10A660002301F1025C4003550900D98313F7070861
:10A6700083471102231CA10093F7F707D98FA3008A
:10A68000F10283572900231DF1005C40F18313F789
:10A6900017008347F102F99BD98FA307F10297A016
:10A6A0000000E78080992AD235D98347940068005A
:10A6B000139757008347B400FD8BD98FA305F4008F
:10A6C0001C4803D647008C4397200000E780A0A9D0
:10A6D000A687177701001307272C740005464C1036
:10A6E000268597000000E78060942A890DD983476A
:10A6F000B400A685FD8BA305F40097000000E78059
:10A7000060DF31BF1783FFFFE702639D832485FE6F
:10A710002A844111268597000000E78080D783476F
:10A7200034FF93F7070E8DCB2AC6268597000000CD
:10A73000E78060C809CD834734FFB245FD8BA3098C
:10A74000F4FE91C5228597300100E780208B4101FE
:10A750001783FFFF6700E39A7DD98327C4FF26850F
:10A76000829775F5834734FF93F7070E91C72285CB
:10A7700097300100E780C08A032584FE970000001F
:10A78000E78000E5E9B71783FFFFE70243929C41AA
:10A7900041112A8903C7070089472E849356670011
:10A7A0006380F6040D466388C6049307F0076304CC
:10A7B000F7022E8597200000E78060ABAA848149CC
:10A7C000C16B130C490097B7FF1F938767519C43D8
:10A7D000984763E4E90441011783FFFF6700E390B2
:10A7E00003D745008547E3F8E7FE2E859720000054
:10A7F000E78040ADE1B703D74500E3FEE7FC2E85D7
:10A8000097200000E780A0A6AA8422859720000058
:10A81000E78000A8C204C98C5DB7DC470355A900D6
:10A82000139A49003E9A93170501C187635DF000B2
:10A8300083570A006397A70263E774038327CA005C
:10A84000034D5A002DA0A1672167A98F1307F7EFC9
:10A85000E374F7FE6397090097000000E7802091FA
:10A8600061FD85098DB783278A00034D4A00835D0A
:10A87000A90003576900216A138BC7003AC6814AB1
:10A8800033CA4D01631E5D0197B7FF1F9387C7450C
:10A890009C43E1DBA2866286814526858297D1B7FB
:10A8A000A1679387F7EF930C4BFF63F24703B24521
:10A8B0005A8597F0FFFFE780A0710DC103278B0039
:10A8C000104709CE10436382C4023107D5BFEE851D
:10A8D000668597000000E780008F71F993861A0063
:10A8E00093FAF60F130B0B0271BF835644005C43BF
:10A8F000E3E9F6F622853AC697200000E78020813A
:10A90000A1679387D7042A8A035D4400324763E82E
:10A9100097008347D90093E707F8A306F9001C477F
:10A9200066852286E2858297C1670844FD17337ADF
:10A93000FA00529508C02312A40125B797B7FF1F4C
:10A940009387073A9843814715C31447814763FFAC
:10A95000D500939745004C47BE9519C903C75500CC
:10A9600081476375E600DC451606B2973E85828016
:10A9700003C745008147E37BE6FE16069C45F5B715
:10A980001773FFFFE7020374AA892E8A814497BADE
:10A99000FF1F938AEA3483A70A00984763E6E4001E
:10A9A0001773FFFF67004375DC47139444000149A8
:10A9B0003E9413BB140083474400634BF9000149E4
:10A9C00013BB140083475400634FF9008504E1B7BB
:10A9D0000844931759005287DA860146A2853E95AE
:10A9E00082990509C9BF4844931759005287DA86EE
:10A9F0000546A2853E9582990509E9B71773FFFFC1
:10AA0000E702E36D814517F5FFFF1305054897B78A
:10AA1000FF1F2399072C97000000E780A0F617730B
:10AA2000FFFF6700036E97B7FF1F9387672B9C4359
:10AA300095C31773FFFFE702836A814517F5FFFF90
:10AA40001305A54497000000E780C0F31773FFFFCC
:10AA50006700236B82801773FFFFE702A36637E46A
:10AA600004008327841241112315E100AE89328945
:10AA7000368A3A8681460147ED45AA8482972AC6DE
:10AA800021C90356A100D28597400100E7806028C4
:10AA90008327C413CE8526858297058905C9832718
:10AAA000440D2314210101462C00268582972A8417
:10AAB00001C9B7E7040083A7C712ED4528008297B4
:10AAC000228541011773FFFF670003634944D5B72F
:10AAD0006554FDB75C41FD175CC182801773FFFFB1
:10AAE000E702E35FB7E70400FC5F82979547330511
:10AAF000F50281450D811773FFFF670083601773AF
:10AB0000FFFFE702C35DB7E70400FC5F829795474C
:10AB10003305F5020D811773FFFF6700835E17731E
:10AB2000FFFFE702C35BB7E7040083A7870B03556A
:10AB3000050082971773FFFF6700A35C1773FFFF81
:10AB4000E702E359035505003287AE861796FF1FCB
:10AB50000356669897B5FF1F938545199700000027
:10AB6000E780A0EF1773FFFF6700A3591773FFFF7C
:10AB7000E702E356B7E7040083A7C7178297177366
:10AB8000FFFF670003581773FFFFE7024355B7E75E
:10AB9000040083A7871397B5FF1F93852515829718
:10ABA00001451773FFFF6700C3551773FFFFE702E7
:10ABB0000353B7E7040083A7C71F81451795FF1FFD
:10ABC0000355658D82971773FFFF670083531773D3
:10ABD000FFFFE702C350B7E7040083A7871397B5C9
:10ABE000FF1F9385A511829701451773FFFF67002B
:10ABF00043511773FFFFE702834EB7E7040083A7B3
:10AC0000C71F81451795FF1F0355E58E8297177360
:10AC1000FFFF6700034F1773FFFFE702434C2E85CA
:10AC200097800000E78080B397800000E78080F085
:10AC30001773FFFF6700E34C1773FFFFE702234A18
:10AC400097800000E78080FA1773FFFF6700634B6F
:10AC50005C49E1175CC95CC583572501A10723192D
:10AC6000F50083570501A1072318F5008280F147FD
:10AC70003305F50297B7FF1F9387470A9C433E951C
:10AC800082808D476315F60803D74600854763F039
:10AC9000E7081773FFFFE7028344368536842E8961
:10ACA00097100000E780A05C29C9835744009314E3
:10ACB0000501C18063E39704228597100000E780B7
:10ACC000005BFD14231294009307A0026300F502B9
:10ACD0009307B0026307F50293079002631FF50024
:10ACE000228597000100E780608901A80146CA8596
:10ACF000228597A00000E78000B41773FFFF67006C
:10AD00004340228597100000E7806007FDB78280EE
:10AD100097B6FF1F9386C6009C42014599CF984382
:10AD2000D44217B6FF1F232DE6FE6396D70097B6D1
:10AD3000FF1F23A9E6FE1385C7FE82801773FFFF5E
:10AD4000E702E33997000000E780A04B7144330528
:10AD50008502914597900000E780C0EC11E56555AC
:10AD60001773FFFF6700E33997B7FF1F23A6A7FA02
:10AD700097000000E780E0483305850291459790F1
:10AD80000000E78020EA61DD97B7FF1F23A8A7F83E
:10AD900097000000E780E04697B7FF1F2398A7F6CB
:10ADA00097000000E780E04597B7FF1F2391A7F6C3
:10ADB00097770100938787C317B7FF1F232CF7F4FA
:10ADC00097070000938707E917B7FF1F2322F7F4BF
:10ADD000014579B71773FFFFE7026330AA8517B5FE
:10ADE000FF1F1305A5F297100000E780605F17733F
:10ADF000FFFF670003311773FFFFE702432E970041
:10AE00000000E78060FD97100000E780E05E97B7E4
:10AE1000FF1F9387E7F09C4391CF1387C7FE19CBA1
:10AE200083D5C7FF17B5FF1F130505F09720010055
:10AE3000E780C01C1773FFFF6700A32C1773FFFF89
:10AE4000E702E32997000000E780C0EC09CD8347C3
:10AE500085002A8493F7070499EB0355E5009700D2
:10AE60000000E78080F91773FFFF6700832983479D
:10AE7000C5009304450117B9FF1F130969EA85E36B
:10AE8000832709005CC997B7FF1F23AB97E8832787
:10AE90004900F1FB97B7FF1F23A697E8E9B7FD1715
:10AEA0002306F500610597800000E78060DA8307DC
:10AEB000840063CB07048347840093E707F82304E7
:10AEC000F400B7E704009C5F82974205A9474181DF
:10AED0003375F5028347840093F707FCC98F230479
:10AEE000F4008347D4003E951C402318A40089CF6A
:10AEF000984319CB8347C4005040814585073305EB
:10AF0000F502420541810297832709005CC897B783
:10AF1000FF1F23A797E08327490089E797B7FF1F03
:10AF200023A297E08347C4009DDF8355040117B532
:10AF3000FF1F130565DF97200100E780200C25B770
:10AF40001773FFFFE702A31997B7FF1F9387070344
:10AF50009C4701448583858B85E3AE84B2853A8620
:10AF600097100000E780204F2A8419C59710000031
:10AF7000E7806045829408CC22851773FFFF670045
:10AF800043181773FFFFE702E31341112E8932C6FE
:10AF9000AA8997000000E780C031324713060502F6
:10AFA000CA86970500009385C5CC17B5FF1F13050A
:10AFB000E5D597000000E780E0F82A8425C99304CE
:10AFC000C50097000000E780E0411946AA85268564
:10AFD00097100000E780201985452685971000000E
:10AFE000E7800015177501001305059E4E958345F2
:10AFF0000500268597100000E780C0195C4831469F
:10B000008145A1075CC85CC483572401E11723195B
:10B01000F40083570401E1172318F4001C4C3E850B
:10B020009770FFFFE780A00EA30425012285410150
:10B030001773FFFF6700430C1773FFFFE702230A34
:10B040004111AA842EC632C497100000E780003A4E
:10B05000004DB2452246834784000CC050C093F790
:10B06000F70393E707042304F4002318040026855C
:10B0700097100000E780203583479400A9462317E6
:10B08000A40013D7370005073307D7029D8B850728
:10B090002306F400A306E40083C70401D84885070B
:10B0A000230FF7FE17B7FF1F130787C75843232A3D
:10B0B00004009307440129E317B7FF1F2324F7C6B1
:10B0C00017B7FF1F232EF7C417B4FF1F1304C4C5FF
:10B0D000228597200100E780A0E41C44858B5D8DCC
:10B0E00019E58145228597200100E78020F1410183
:10B0F0001773FFFF6700E3001CC317B7FF1F23236D
:10B10000F7C2D9B71773FFFFE70263FD9705000089
:10B11000938565B7014597000000E78000B00145C1
:10B120001773FFFF6700E3FD1773FFFFE70223FBC1
:10B1300097000000E78080B01773FFFF670063FC93
:10B140008347C500A5E31773FFFFE70243F92A848D
:10B150000355E50097000000E78000C821C1834740
:10B16000840093F7F7FB2304F4001C4091C7DC43F1
:10B1700081C74C400145829797000000E78080B965
:10B1800017B5FF1F130545BA97200100E78040E976
:10B190000355E40097000000E78020C61773FFFF07
:10B1A000670023F682801773FFFFE70243F397B728
:10B1B000FF1F9387E7B697050000938565C817B50D
:10B1C000FF1F130565B623A0070023A207009720E1
:10B1D0000100E78080D21773FFFF670083F21C4DE8
:10B1E00091CFDC4381CF1773FFFFE70243EF834525
:10B1F000070082971773FFFF6700A3F0828097B75D
:10B20000FF1F9387A7B49C4303C50700828097B7AD
:10B21000FF1F9387A7B39C4303C51700828097B78E
:10B22000FF1F9387A7B29C4303C52700828097B76F
:10B23000FF1F9387A7B19C4303C54700828097B740
:10B24000FF1F9387A7B09C4303C53700828097B741
:10B25000FF1F9387A7AF9C4303C55700828097B712
:10B26000FF1F9387A7AE9C4303C56700828097B7F3
:10B27000FF1F9387A7AD9C4303C57700828097B7D4
:10B28000FF1F9387A7AC9C4303C58700828097B7B5
:10B29000FF1F9387A7AB9C4303C59700828097B796
:10B2A000FF1F9387A7AA9C4303C5A700828097B777
:10B2B000FF1F9387A7A99C4303C5B70011E11D4554
:10B2C000828097B7FF1F938767A89C4303C5C70079
:10B2D000828097B7FF1F938767A79C4303C5D7005A
:10B2E000828097B7FF1F938767A69C4303C5E7003B
:10B2F000828097B7FF1F938767A59C4303D50701FB
:10B30000828097B7FF1F938767A49C4303C52701DB
:10B31000828097B7FF1F938767A39C4303D547019C
:10B32000828097B7FF1F938767A29C4303D567016D
:10B33000828097B7FF1F938767A19C4303D587013E
:10B34000828097B7FF1F938767A09C4303C5A7011F
:10B35000828097B7FF1F9387679F9C4303C5B70100
:10B36000828097B7FF1F9387679E9C4303C5C701E1
:10B37000828097B7FF1F9387679D9C4303C5D701C2
:10B38000828097B7FF1F9387679C9C438857828072
:10B3900097B7FF1F9387879B9C4303D5C702828083
:10B3A00097B7FF1F9387879A9C4303D5E70219E15C
:10B3B0001305800C828097B7FF1F938727999C43C2
:10B3C00003C50703828097B7FF1F938727989C4385
:10B3D000C85B828097B7FF1F9387C7968843828098
:10B3E00097B7FF1F938747968843828019E17D5561
:10B3F0008280F5DE984265DFFDD917B7FF1F13077E
:10B40000E7B71847AA877155058B631D072403C545
:10B4100007001547E37DA7FC03C737001305F005B8
:10B420007D171377F70FE364E5FC03C35700E300D0
:10B4300003FC83C86700E38C08FA03C7770049451B
:10B4400079171377F70FE364E5FA03C7A7001148EC
:10B450001305F7FF1375F50FE36BA8F803CE9700FC
:10B460000D481305FEFF1375F50FE362A8F803C836
:10B47000B7006309080065181378F80F1305600D0D
:10B48000E36705F703C5C700794879151375F50F0C
:10B49000E36FA8F403C8D7000D457D181378F80FA3
:10B4A000E36705F503D80701930E401751184208CA
:10B4B00013580801E3ED0EF303C8E7007D18137875
:10B4C000F80FE36605F303C827017D181378F80F1A
:10B4D000E36F05F103C88700C54E75181378F80FA0
:10B4E000E3E70EF103D86701856E938EBEE06D1819
:10B4F000420813580801E3EC0EEF03D847016D181A
:10B50000420813580801E3E40EEF03D887017918C5
:10B51000420813580801E36C05ED03C8A7017D1824
:10B520001378F80FE36505ED03C5B7011D487D15D8
:10B530001375F50FE36DA8EA03C5D70171487915B6
:10B540001375F50FE365A8EA03D5E7011308E00FCB
:10B550007D1542054181E36CA8E803C5070249480F
:10B5600079151375F50FE364A8E8C85301C937C806
:10B5700034005915130858BFE36BA8E603A88702E7
:10B5800037C53400130555BF5918E36205E717A501
:10B59000FF1F232BC57A03C6050117A5FF1F23270D
:10B5A000F57A0545E375C5E403D82501D04933761E
:10B5B0000603E31E06E203C61501E30A06E217A628
:10B5C000FF1F2321B67883C5270001466387A500A6
:10B5D00003C61700F1453306B60283C70703930578
:10B5E000C00272971A071307C70516031A97960821
:10B5F0004697B387B70241553E973297420741833A
:10B600006362E8061773FFFFE70263AD3685978034
:10B610000000E780406C97000100E780C04B2A845F
:10B6200097A00000E780205E2A9497F00000E78052
:10B63000002A2A9497900000E78040852A9497F08A
:10B64000FFFFE780E06F2A9497400000E7800097B3
:10B650002A9497700000E78040A022951773FFFF9F
:10B66000670023AA82801773FFFFE70243A74111F7
:10B67000A307A10097A00000E78040C99305F1004F
:10B68000170500001305E5B597F0FFFFE780802F51
:10B69000014541011773FFFF6700A3A61773FFFF62
:10B6A000E70263A117B4FF1F1304448D032884002D
:10B6B00079599368180097B4FF1F23A5148D137848
:10B6C000180063100802BA84BE89368B328A2E892C
:10B6D000AA8A97F0FFFFE780E0A77D15269519E578
:10B6E00031594A851773FFFF670063A097F0FFFF8A
:10B6F000E78040A67D152695A167E353F5FE97B731
:10B70000FF1F9387A7BE98433E8C814B01CB014519
:10B7100097F00000E780C047933B15004A85DA8622
:10B720005686D28597900000E78060512A8911CD16
:10B730001C44F99B17B7FF1F2326F78483270C00AF
:10B74000CDD3E3800BFA829769BF268597B7FF1F99
:10B7500023A8078297F0FFFFE780809C4146CE85B3
:10B7600017B5FF1F1305058B97300100E780605A5E
:10B7700097D00000E780E09C0325040B97D00000E1
:10B78000E780A0A0054597D00000E780A0A7054569
:10B7900097000000E78060EDA9B797A7FF1F938788
:10B7A000E77D9C47858BEDC71773FFFFE702239367
:10B7B00017B5FF1F1305458497A7FF1F23A0077C1C
:10B7C00097A7FF1F23AE077A97A7FF1F23AC077A1F
:10B7D00097200100E780C08497500000E78080F93F
:10B7E00097100100E780405097100100E780405615
:10B7F00097A7FF1F938707779C4391C705459780BD
:10B800000000E780E02397A7FF1F9387675F9C43B3
:10B8100099C741657D1597700000E780E0A597F016
:10B820000000E780804197D00000E780209397B721
:10B83000FF1F9387A7899C4313971701635607003F
:10B8400097F00000E780A0B097A7FF1F23A4077C14
:10B8500097A7FF1F23A2077C97A7FF1F23A0077CA2
:10B8600097A7FF1F23AE077A97000000E780008CA0
:10B8700097000000E780A07597F0FFFFE780401871
:10B8800097F00000E780E0D91773FFFF6700638738
:10B89000828097A7FF1F9387676E8843828097A750
:10B8A000FF1F9387A76DC8438280B7E7B0009387D7
:10B8B000075063E1A70297A7FF1F9387276CD84320
:10B8C000FD576367E50097A7FF1F23ABA76A814772
:10B8D0003E858280B957EDBF1773FFFFE7022380D3
:10B8E00097800000E780607597800000E780C07750
:10B8F0001773FFFF6700E3801763FFFFE702837C96
:10B900002A849304140201112E85B289A68521464A
:10B9100036C63A8997300100E780403D0DE9B246CE
:10B9200038082686CE851305940497500000E780DA
:10B93000604121462C084A8597300100E780003B92
:10B940001335150005611763FFFF6700E37A0145B2
:10B95000D5BF1763FFFFE70283789305450617A558
:10B96000FF1F1305E53E97100100E780206917636C
:10B97000FFFF670003791763FFFFE702437641117A
:10B980002EC697F0FFFFE780C017B24588C141017E
:10B990001763FFFF6700E3761763FFFFE702837219
:10B9A000AA842E8497800000E780006CAA898545D0
:10B9B000228597000000E780E07D83C7E4011389BA
:10B9C000940899E313890403CE852285970000002B
:10B9D000E780407C214693051902228597000000EC
:10B9E000E780607897A7FF1F938747598C4322858C
:10B9F00097100000E780C08221469385840222854B
:10BA000097000000E78020761763FFFF6700C36E92
:10BA10001763FFFFE702236A397197F00000E780A0
:10BA2000E0B49305400661E997800000E78000607C
:10BA30006302051497A7FF1F83C7473313B7170087
:10BA400097A6FF1F2384E632014499CFC16417A94A
:10BA5000FF1F1309A9529309400EFD14970000001F
:10BA6000E78020836342A40A97F0FFFFE780600924
:10BA70004169B7290900096AFD7A2A8B81447D1939
:10BA80009389F97B130A0A71938A8AC79700000089
:10BA9000E780208063D7A4041304400EB387840298
:10BAA00017A7FF1F1307874D0324070B3E948357E7
:10BAB000C4016382270B18403307EB4063EAE900B7
:10BAC000834744008507B3874703D6976365F70824
:10BAD00001468145094597F0FFFFE780C04AAA8BE0
:10BAE00029E597400000E780808385476317F506C6
:10BAF00089659385057117A5FF1F130565259710A7
:10BB00000100E780A04F95A0B30734030327090B7A
:10BB1000BA9703D7C7016308970003C75700A382EA
:10BB200007002382E700050415BF9305C5002285A1
:10BB300097000000E78080E65E8522869765010019
:10BB40009385C5E997F0FFFFE780404F5E8597102A
:10BB50000000E780608A850415BF97A7FF1F9387C1
:10BB6000E7419C478D83858BC1F721611763FFFFF8
:10BB70006700E35701468545094502D002D202D449
:10BB800002D697F0FFFFE7800040AA8479DD97F0A6
:10BB90000000E780E09C1389C4002A8481454A851F
:10BBA00097000000E780005F0C4041464A859700FF
:10BBB0000000E780405B832944006385090C4E85C3
:10BBC00002D802DA02DC02DE97300100E780E038BA
:10BBD0002ACE141005462C0808184ECC97500000A9
:10BBE000E780E00A1375F50F51ED8355840093E566
:10BBF00025004A8597000000E780E05E11460C10A2
:10BC00004A8597000000E7800056014697650100CD
:10BC1000938545DD268597F0FFFFE7802042268546
:10BC200097000000E780407D5C40A1D30146854538
:10BC30000D4597F0FFFFE7800035AA841DD54840E9
:10BC40001389C40097300100E78020312AC64A8555
:10BC500097000000E780404C3246636FC5004C40BF
:10BC60004A8597000000E7800050014681452685FF
:10BC700097F0FFFFE780803C268597000000E78073
:10BC8000A077E5B583558400ADB71763FFFFE702E2
:10BC9000034597A7FF1F9387672E9C471DC193E716
:10BCA000870017A5FF1F1305A50A17A7FF1F232B42
:10BCB000F72C97100100E78040321763FFFF670001
:10BCC0004344DD9B17A7FF1F232EF72A9730000060
:10BCD000E780E0647DF117A5FF1F13056507971046
:10BCE0000100E780E033D1BF1763FFFFE702A33C09
:10BCF0004169AA892E8AB28A368BBA8B814417ACE5
:10BD0000FF1F130CAC27930C400E7D1997F0FFFF1B
:10BD1000E780205863C4A40001443DA03384940309
:10BD200083270C0B3E948357C401638627055A87EB
:10BD3000D6865286CE851305040397000000E7805F
:10BD4000E0BB01C923800B0022851763FFFF67005A
:10BD5000033A8347F40185C35A87D6865286CE8537
:10BD60001305940897000000E78040B909C585478E
:10BD70002380FB00D1BF850451BF835745006380FA
:10BD8000071E1763FFFFE702E33301112A849700C0
:10BD90000000E780C04D09C985476309F5060561C4
:10BDA0001763FFFF6700433597E00000E780007CE2
:10BDB0007DF5835744004947ED9BE392E7FEC1457B
:10BDC000228597000000E7804033AA8422859700EF
:10BDD0000000E780204F0357440002CE91472A8994
:10BDE000631AF700228597000000E780A0513C0805
:10BDF0002ACC3ECE97E00000E78080765C55C5D324
:10BE000074084A86A6850545829751BF03574400AA
:10BE1000D147E3F6E7F8032A0400C169014997AA6C
:10BE2000FF1F938AAA15130B400EFD1997F0FFFF11
:10BE3000E7802046634FA90E2285032A040097005D
:10BE40000000E780C042A1452A89228597000000B2
:10BE5000E780A02AAA84228597000000E780804A14
:10BE600014402A86AA8978082685CA85970000008A
:10BE7000E780C0E7AA8405D503C7F40189476315A5
:10BE8000F7008347C10181DF5546D28513856400E1
:10BE900097300100E780E0E7014597800000E780E8
:10BEA000C01901C583D7C401A5E797A7FF1F9387D2
:10BEB000E70C9C4793551900858913D73700058BEC
:10BEC00001CF8983858B6399B70001452EC6970002
:10BED0000000E780C0DBB2454E8597800000E78018
:10BEE000601F0346C1012A84937519002685979027
:10BEF0000000E780E03935C1268597800000E780A3
:10BF0000E018268511C0014597800000E780004CAD
:10BF100097300000E780A0408547E312F5E883C72B
:10BF200054001307F00FE38CE7E68507A382F400C3
:10BF3000BDB5B304690383A70A0BBE9483D7C401BC
:10BF4000638B37015546D285138564009730010015
:10BF5000E780C0D955DD0509D1BD5DD86DB78280B8
:10BF60001763FFFFE702031697800000E780000CCD
:10BF700005C1C164014417A9FF1F130929009309D2
:10BF8000400EFD1497F0FFFFE780A030634EA40041
:10BF900017A5FF1F1305C5DB97100100E780E0031D
:10BFA0001763FFFF67004315330534038327090B2D
:10BFB0003E958357C501638897002312050097803B
:10BFC0000000E780A00C050475BF97A7FF1F9387AB
:10BFD000E7FA9C478D83858B8DE31763FFFFE702AC
:10BFE000031017A5FF1F1305A5D697100100E780C2
:10BFF00020031763FFFF6700C31082801763FFFFF2
:10C00000E702E30D970500009385C5A017A5FF1F64
:10C01000130505D497100100E78020EE1763FFFF9A
:10C020006700230E1763FFFFE702630B8841B7E742
:10C030000400BC5B050542054181829709C585471F
:10C040002300F50005051763FFFF6700830B83C717
:10C05000F5FF2E858507A38FF5FE828083C7F5FF48
:10C06000FD1793F7F70FA38FF5FE99EF1763FFFF07
:10C07000E702E306B7E70400BC571385F5FF829794
:10C080001763FFFF6700E30782801C4103574500E9
:10C090008D8FBA951CC12312B5003E85828093D73F
:10C0A0008500A2051441DD8D835745001387E6FF07
:10C0B00018C189072312F50013D685004111238F7B
:10C0C000B6FEA38FC6FE4101828018419307F7FF99
:10C0D0001CC18357450085072312F500A30FB7FE47
:10C0E0008280835745008D8F2312F5001C41BE9539
:10C0F0000CC12E858280AA8703D7470008410D8F87
:10C10000AA952392E7008CC3828018410845330525
:10C11000A740828083574500035765001D8F1C414F
:10C1200008453385A7403305A74082801763FFFF8A
:10C13000E702E3FA41112EC62A8497000000E78047
:10C14000A0FDB2456373B50001A0835744000840C9
:10C15000BE952312B4003E9541011763FFFF6700AF
:10C1600043FA1763FFFFE70283F741112E84B2857C
:10C1700032C697000000E780A0FB3246A2859730C8
:10C180000100E78000B941011763FFFF670063F713
:10C190001763FFFFE702A3F42E8485459700000094
:10C1A000E78000F9230085001763FFFF670063F550
:10C1B0001763FFFFE702A3F241112317B10089457E
:10C1C00097000000E780C0F68347E1002300F500F8
:10C1D0008347F100A300F50041011763FFFF6700EB
:10C1E00043F21763FFFFE70283EF93D78500A205B1
:10C1F0004111DD8D2317B100894597000000E780CC
:10C2000020F38347E1002300F5008347F100A300FA
:10C21000F50041011763FFFF6700A3EE1763FFFFFF
:10C22000E702E3EB1397850193D78501C1669386F7
:10C2300006F0D98F13D78500758FD98FA2053707E0
:10C24000FF00F98D4111DD8D2EC69145970000004C
:10C25000E78000EE6C00114697300100E78060AB8C
:10C2600041011763FFFF6700C3E91763FFFFE702A0
:10C2700003E71C41854503C4070097000000E780E1
:10C2800080E622851763FFFF6700A3E71763FFFFC0
:10C29000E702E3E41C414111894503C7070083C756
:10C2A00017002307E100A307F10097000000E780D3
:10C2B00080E30355E10041011763FFFF670063E47A
:10C2C0001763FFFFE702A3E11C414111894503C742
:10C2D000070083C717002307E100A307F1009700B9
:10C2E0000000E78040E08357E100410113D587005B
:10C2F000A2075D8D420541811763FFFF670063E080
:10C300001763FFFFE702A3DD0C4141112A841146A8
:10C31000680097300100E780C09F91452285970013
:10C320000000E78040DCB247C166938606F01397B1
:10C33000870113D58701598D13D78700758F598DC4
:10C34000A2073707FF00F98F5D8D41011763FFFFDB
:10C35000670023DB1C45BE950CC18280AE879443E9
:10C3600091E6584101EF0CC15CC1828003C75700C0
:10C3700013671700A382E700B687D5B70CC3EDB7E4
:10C38000AA87084119CD1841D44398C36313D50037
:10C39000D8C32A87034657009376160081E62320E8
:10C3A00007008280944381CA8C4203A847008CC353
:10C3B00063930601CCC3799A14C3A302C7003687DE
:10C3C000D1BF1C45DC471D8DB777DBB6938777DB84
:10C3D00009853305F502420541818280F147B38525
:10C3E000F50248452E958280834745008507230244
:10C3F000F50082801763FFFFE70263CE2A8409E419
:10C400001763FFFF6700E3CF83474400F5DBFD17A9
:10C4100093F7F70F2302F400E5F71C4403D7270036
:10C4200005072391E700DC4399C3228582974C4896
:10C4300089CD83475400898B99E71C4422859C470A
:10C440009C439C478297232A040000402320040039
:10C450007DB71763FFFFE70283C8835725004111AB
:10C460002EC681EB0144228541011763FFFF67005F
:10C4700043C9035705008147F146E305F7FEB3853D
:10C48000D702404585072E948345440008C4F5F53E
:10C49000B247AA8481E7232A040009A81C456C003E
:10C4A00022859C439C43829748C84DDD85472312D3
:10C4B000F400B24723200400231804002319F400D9
:10C4C0005C485CC483D72400FD172391F40061BF4E
:10C4D0001763FFFFE702A3C097A7FF1F9387478952
:10C4E00088432326050023240500410597100100F9
:10C4F000E78000B31763FFFF6700A3C01763FFFF68
:10C50000E702E3BD17A4FF1F130484861C404111FA
:10C5100099CF9C472300B5002AC65CC19700000054
:10C52000E78040FB1C40DC4399C3324582974101C0
:10C530001763FFFF6700E3BC0347450029E3584D3D
:10C54000AA877D551DCF1763FFFFE70243B91CC3C0
:10C55000DC4797A6FF1F23ADE680F15613050701C0
:10C560002390D700970500009385050297100100DE
:10C57000E780A09801451763FFFF670083B87D55EA
:10C58000828082801763FFFFE70263B50111614675
:10C59000814528009760FFFFE78060B79797FF1FEE
:10C5A0009387077D9C4328009305F00FDC473EC628
:10C5B00097000000E780C0F405611763FFFF670084
:10C5C00043B49797FF1F9387A77A9C43D847A167E7
:10C5D0009387C702631EF70A397106DE22DC26DA6A
:10C5E00080004AD84ED652D456D23285B2849700B3
:10C5F0000000E780C0C7AA89268597000000E78071
:10C6000020C92318A4FC268597000000E78040C8B5
:10C610002319A4FC268597000000E78060C783D714
:10C6200044000A8A231AA4FC858393F7F70F230E8C
:10C63000F4FC8607BD0793F7073F3301F1408A8A70
:10C6400001498347C4FD6367F902CE85130584FC65
:10C65000232C54FD97000000E78080EA52811301EB
:10C6600004FCF2506254D2544259B259225A925A9E
:10C6700021618280268597000000E78060C19317C2
:10C680001900D69705092390A7001379F90F55BF14
:10C6900082809797FF1F9387A76D9C43D847A16718
:10C6A0009387A702631AF70A397106DE22DC26DABD
:10C6B00080004AD84ED652D456D23285B2849700E2
:10C6C0000000E780C0BAAA89268597000000E780AD
:10C6D00020BCFD572318A4FC26852319F4FC9700E1
:10C6E0000000E780E0BA83D744000A8A231AA4FC3A
:10C6F000858393F7F70F230EF4FC8607BD0793F7A6
:10C70000073F3301F1408A8A01498347C4FD6367CB
:10C71000F902CE85130584FC232C54FD97000000FC
:10C72000E78000DE5281130104FCF2506254D254BF
:10C730004259B259225A925A216182802685970025
:10C740000000E780E0B493171900D69705092390FD
:10C75000A7001379F90F55BF82809797FF1F938722
:10C7600027619C43D847A16789076310F70A39718D
:10C7700006DE22DC26DA80004AD84ED652D456D2C3
:10C780003285328997000000E78060AEAA894A8529
:10C7900097000000E780C0AF835749000A8A23183A
:10C7A000A4FC858393F7F70F230CF4FC8607BD07E1
:10C7B00093F7073F3301F1408A8A8144834784FD20
:10C7C00063E7F402CE85130584FC232A54FD970009
:10C7D0000000E780E0D25281130104FCF250625461
:10C7E000D2544259B259225A925A216182804A85C2
:10C7F00097000000E780C0A993971400D69785049E
:10C800002390A70093F4F40F55BF82809797FF1FE2
:10C81000938707569C43D847A1679387E704631E15
:10C82000F70A397106DE22DC26DA80004AD84ED6B5
:10C8300052D456D23285B28497000000E78020A3FC
:10C84000AA89268597000000E78080A42318A4FC0D
:10C85000268597000000E780A0A3231AA4FC268564
:10C8600097000000E780C0A283D744000A8A2319FA
:10C87000A4FC858393F7F70F230EF4FC8607BD070E
:10C8800093F7073F3301F1408A8A01498347C4FD8A
:10C890006367F902CE85130584FC232C54FD9700B1
:10C8A0000000E780E0C55281130104FCF25062549D
:10C8B000D2544259B259225A925A21618280268515
:10C8C00097000000E780C09C93171900D6970509D0
:10C8D0002390A7001379F90F55BF82809797FF1F08
:10C8E000938707499C43D847A1679387C704631A76
:10C8F000F70A397106DE22DC26DA80004AD84ED6E5
:10C9000052D456D23285B28497000000E780209638
:10C91000AA89268597000000E7808097FD57231895
:10C92000A4FC2685231AF4FC97000000E7804096BB
:10C9300083D744000A8A2319A4FC858393F7F70F51
:10C94000230EF4FC8607BD0793F7073F3301F14040
:10C950008A8A01498347C4FD6367F902CE851305BE
:10C9600084FC232C54FD97000000E78060B95281BD
:10C97000130104FCF2506254D2544259B259225A63
:10C98000925A21618280268597000000E7804090BE
:10C9900093171900D69705092390A7001379F90F6B
:10C9A00055BF82809797FF1F9387873C9C43D8474A
:10C9B000A167DD076317F7041753FFFFE702237230
:10C9C00079713285328497000000E780408A2AC658
:10C9D000228597000000E780A08B2311A102228509
:10C9E00097000000E780A088B2452300A102280834
:10C9F00097000000E780C0B045611753FFFF670054
:10CA0000437082809797FF1F938787369C43D84750
:10CA1000A167938787046317F7041753FFFFE702A3
:10CA2000036C79713285328497000000E78020849E
:10CA30002AC6228597000000E78080852311A10285
:10CA4000228597000000E7808082B2452300A10282
:10CA5000280897000000E780A0AA45611753FFFF50
:10CA60006700236A82809797FF1F938767309C43F4
:10CA7000D847A1679387A7046312F7021753FFFFF4
:10CA8000E702E36501112800814597000000E78077
:10CA900020A705611753FFFF6700A3668280979761
:10CAA000FF1F9387E72C9C43D847A16793875702C2
:10CAB0006319F7021753FFFFE70263620111328522
:10CAC00097F0FFFFE780A07A2308A10081452800A6
:10CAD00097000000E780C0A205611753FFFF6700C1
:10CAE000436282809797FF1F938787289C43D8478C
:10CAF000A1679387E702631BF7041753FFFFE70261
:10CB0000035E01113285328497F0FFFFE7804078A1
:10CB1000AA84228597F0FFFFE7808077854709E99F
:10CB2000228597F0FFFFE78080744205B337A000AD
:10CB300028008145231891003ECA97000000E78035
:10CB4000209C05611753FFFF6700A35B82809797C6
:10CB5000FF1F9387E7219C43D84799476313F70842
:10CB60001753FFFFE702A35779713285328497F09C
:10CB7000FFFFE780C06F2AC6228597F0FFFFE7809E
:10CB800020712310A102228597F0FFFFE780206E1D
:10CB90002301A102228597F0FFFFE780406DA301EA
:10CBA000A102228597F0FFFFE780606C2302A102BB
:10CBB000228597F0FFFFE780806B2313A102228577
:10CBC00097F0FFFFE780A06AB2452314A10228086E
:10CBD00097000000E780C09245611753FFFF670090
:10CBE000435282809797FF1F938787189C43D847AB
:10CBF000A1679387C7036313F7081753FFFFE70283
:10CC0000034E79713285328497F0FFFFE78020660A
:10CC10002AC6228597F0FFFFE78080672310A102D4
:10CC2000228597F0FFFFE780A0662311A1022285ED
:10CC300097F0FFFFE780A0632302A102228597F00F
:10CC4000FFFFE780C062A302A102228597F0FFFFE9
:10CC5000E780E0612303A102228597F0FFFFE780D0
:10CC60000061B245A303A102280897000000E780F5
:10CC7000208945611753FFFF6700A348828017533F
:10CC8000FFFFE702C34501112A8497F0FFFFE78009
:10CC9000005EAA84228597F0FFFFE780605F22850F
:10CCA00097F0FFFFE780C05E035744008D4763F7AE
:10CCB000E700228597F0FFFFE780805D228597F0EF
:10CCC000FFFFE780E05C2800A68597000000E78072
:10CCD000208305611753FFFF6700A3429797FF1F4B
:10CCE000938707099C43D847A167FD07631FF70097
:10CCF0001753FFFFE702A33E328597000000E7804D
:10CD000040F81753FFFF6700C33F82809797FF1FCC
:10CD1000938707069C43D847A167E5076315F70883
:10CD20001753FFFFE702A33B79713285328497F0F6
:10CD3000FFFFE780C0532AC6228597F0FFFFE780F8
:10CD40002055228597F0FFFFE78080542310A10231
:10CD5000228597F0FFFFE780A053520551812311F0
:10CD6000A10222852302010297F0FFFFE7802050F5
:10CD7000A302A102228597F0FFFFE780404F230323
:10CD8000A102228597F0FFFFE780604EB245A30322
:10CD9000A102280897F0FFFFE780807645611753CE
:10CDA000FFFF6700033682809797FF1F938747FC3A
:10CDB0009C43D847A1679387E703631FF700175386
:10CDC000FFFFE702C331328597000000E78060EB88
:10CDD0001753FFFF6700E33282809797FF1F938707
:10CDE00027F99C43D847A16793874704631EF7023E
:10CDF0001753FFFFE702A32E79713285328497F033
:10CE0000FFFFE780C0462AC6228597F0FFFFE78034
:10CE10002048B245280897F0FFFFE780606E456123
:10CE20001753FFFF6700E32D82809797FF1F9387BB
:10CE300027F49C43D847A167938787026310F704C0
:10CE40001753FFFFE702A32979713285328497F0E7
:10CE5000FFFFE780C0412AC6228597F0FFFFE780E9
:10CE60000041B2452300A102280897F0FFFFE780A8
:10CE7000206945611753FFFF6700A328828017537D
:10CE8000FFFFE702C325011197F0FFFFE780203E77
:10CE9000AA85280097F0FFFFE78080660561175399
:10CEA000FFFF670003269797FF1F938767EC9C435C
:10CEB000D847A167D107631FF7001753FFFFE702A9
:10CEC0000322328597000000E780A0FB1753FFFF85
:10CED0006700232382809797FF1F938767E99C430E
:10CEE000D847A167C507631FF7001753FFFFE70285
:10CEF000031F328597000000E780A0F81753FFFF5B
:10CF00006700232082809797FF1F938767E69C43E3
:10CF1000D847A167B907631FF7001753FFFFE70260
:10CF2000031C328597000000E780A0F51753FFFF30
:10CF30006700231D82809797FF1F938767E39C43B9
:10CF4000D847A167AD07631FF7001753FFFFE7023C
:10CF50000319328597000000E780A0F21753FFFF06
:10CF60006700231A82809797FF1F938767E09C438F
:10CF7000D84789476318F7021753FFFFE7022316C4
:10CF80000111328532C897F0FFFFE780402EAA8555
:10CF9000280097F0FFFFE780A05605611753FFFFB9
:10CFA0006700231682809797FF1F938767DC9C4357
:10CFB000D847A1678D076311F7041753FFFFE702F6
:10CFC000031201113285328497F0FFFFE780202A97
:10CFD00013066100AA844C00228597300000E78088
:10CFE000C0232800A68597F0FFFFE7806051056108
:10CFF0001753FFFF6700E31082809797FF1F938707
:10D0000067D79C4381CFDC4391CB1753FFFFE702E7
:10D01000030D82971753FFFF6700A30E82801753FB
:10D02000FFFFE702C30B79713C08AE843ED2A165D5
:10D03000B7070A002A843ED448103C08DD053ED6D6
:10D0400036C432C63AC297D0FFFFE780402C124761
:10D050004810BA8597F0FFFFE780C01332464810AA
:10D06000B28597F0FFFFE780E014A2464810B6852E
:10D0700097F0FFFFE7800012501001478146A68518
:10D08000228597D0FFFFE780E04D45611753FFFFF2
:10D09000670023071753FFFFE702630401117C00B9
:10D0A0000329C501AE843ECAA165B70707002A84DB
:10D0B0003ECC48087C00C5053ECE97D0FFFFE780F8
:10D0C00000258345D900480897F0FFFFE780800CD2
:10D0D000500801478146A685228597D0FFFFE7804B
:10D0E000604805611753FFFF6700A3011753FFFF57
:10D0F000E702E3FE83C7950093F7F707A384F500E3
:10D1000097000000E78040F91753FFFF670063FFB7
:10D110001753FFFFE702A3FC79713C08AE843ED2AF
:10D12000A165B70709002A843ED448103C089385BE
:10D1300045043ED632C636C497D0FFFFE780201D97
:10D14000A2464810B68597F0FFFFE780A00432465C
:10D150004810B28597F0FFFFE780C00550100147E7
:10D160008146A685228597D0FFFFE780A03F4561D5
:10D170001753FFFF6700E3F81753FFFFE70223F69B
:10D1800083C7950041112A8493F7F707A384F5001C
:10D1900032852EC697F0FFFFE780800F85672AC48F
:10D1A0006370F50297700000E78020E92246B245DF
:10D1B00009ED11478146228597000000E78060E66F
:10D1C00041011753FFFF6700C3F301478346F50191
:10D1D000DDB71753FFFFE702E3EE01113C003ECA43
:10D1E000B7070A003ECC3C003ECE83C79500AA8913
:10D1F000328593F7F707A384F5002E8497F0FFFF9D
:10D20000E78000098567637DF504A165AA8493859D
:10D210008504480897D0FFFFE780600F2685977048
:10D220000000E78080E12A8929E19145480897F0CC
:10D23000FFFFE78020F6A685480897F0FFFFE7800C
:10D2400060F7CA85480897F0FFFFE780A0F4014720
:10D2500081465008A2854E8597D0FFFFE780803039
:10D2600005611753FFFF670023E98145480897F0E0
:10D27000FFFFE78020F20349090275BF1753FFFF44
:10D28000E70243E479711C103ECAB7070F003ECC99
:10D29000404D1C10AA84AE894808994532C636898B
:10D2A0003ECE97D0FFFFE780800632464808B28521
:10D2B00097F0FFFFE78000EE630C0902A5454808E0
:10D2C00097F0FFFFE780C0E62546CA85972001005A
:10D2D000E78020A4500801478146CE85268597D057
:10D2E000FFFFE780202845611753FFFF6700C3E079
:10D2F0008355C402480897F0FFFFE780A0EB035571
:10D30000E402814505C5854785456301F502C1678E
:10D31000FD179305F00F630BF5007D159770000066
:10D32000E780208E9305150093F5F50F480897F0D8
:10D33000FFFFE78020E683450403480897F0FFFFDE
:10D34000E78040E583451403480897F0FFFFE78036
:10D3500060E483552403480897F0FFFFE78080E5E9
:10D3600083554403480897F0FFFFE780A0E49DB78A
:10D370001753FFFFE702A3D683C7950081460146F6
:10D3800093F7F707A384F50097000000E78040EFCC
:10D390001753FFFF6700E3D61753FFFFE70223D4BD
:10D3A00079713E841C103ECA2E89B7070F00A16513
:10D3B0003ECCFD051C10AA84480842C03AC23ECEAD
:10D3C00036C432C697D0FFFFE78060F43246480883
:10D3D000B28597F0FFFFE780E0DBA2464808B685FC
:10D3E00097F0FFFFE78000DD12474808BA8597F005
:10D3F000FFFFE78020DC0248630C080291454808E3
:10D4000097F0FFFFE780C0D21146A2859720010068
:10D41000E7802090500801478146CA85268597D02D
:10D42000FFFFE780201445611753FFFF670063CDBE
:10D430008945480897F0FFFFE78080CF83470400C5
:10D440002300F50083471400A300F500E1B717534C
:10D45000FFFFE70223C783C7950001112A8A93F7CC
:10D46000F707A384F5003285AE8432C697F0FFFF3C
:10D47000E78000E232462A89328597F0FFFFE78095
:10D4800000DF85676373F902AA894A8597700000F7
:10D49000E780A0BA2A8419ED114781464A86A685FD
:10D4A000528597000000E780C0B705611753FFFF62
:10D4B000670083C49387E9FF93F7F70F0547E36697
:10D4C000F7FE8347F50195EB8947E380F9FE834634
:10D4D000F401528501474A86A68597000000E7803F
:10D4E00040B4A167D90748083ECC230A010002CE08
:10D4F00097000000E780A0B04DBF639EE70089471A
:10D50000639EF90093071020231FF5009770000019
:10D51000E780C0B76DBF0947E39BE7FA8D47E39803
:10D52000F9FA228597700000E78080DF9797FF1F48
:10D53000938747A39C4399E79797FF1F9387478C4F
:10D540009C4399C703D5040097800000E780A0CED4
:10D55000231F040022855DBF1753FFFFE70223B896
:10D5600001113C003ECAB7070B003ECC3C003ECE4A
:10D5700083C795002A89328593F7F707A384F500BE
:10D58000AE8497F0FFFFE780A0D093170501C18715
:10D59000635AF006A1652A849385E502480897D06E
:10D5A000FFFFE780C0D6A285480897F0FFFFE7801D
:10D5B00060C09797FF1F9387A7849C43A9EB014402
:10D5C0009375F40F480897F0FFFFE780A0BC9355D0
:10D5D000844093F5F50F480897F0FFFFE78080BB84
:10D5E0009355044193F5F50F480897F0FFFFE78046
:10D5F00060BA014781465008A6854A8597D0FFFF4B
:10D60000E78040F605611753FFFF670083AF416570
:10D6100085460546A2857D1597500000E78060BDD0
:10D6200059DD510597000100E780808F1304400603
:10D630003344850271B71753FFFFE70243AA011174
:10D64000B70706003EC683C7950021642A8993F771
:10D65000F707A384F500AE8428009305A4040AC448
:10D660000AC897D0FFFFE78080CA30000147814693
:10D67000A6854A8597D0FFFFE780C0EE97E0FFFFC1
:10D68000E780E01113049404480822CC230A010027
:10D6900002CE97000000E780809605611753FFFFD8
:10D6A000670023A61753FFFFE702C3A1C1642A89BD
:10D6B00001449799FF1F9389698C130A8002FD1416
:10D6C00097E0FFFFE780E0BD6347A40001451753E3
:10D6D000FFFF670063A2B307440303A7C90ABA9711
:10D6E00003D707006306970083D7270063842701C9
:10D6F0000504F9B70545E1BF1753FFFFE702839C17
:10D700002A8A2E8999C123A0050081498144978ADC
:10D71000FF1F938A6A66614B97E0FFFFE780A0BE18
:10D7200063C7A4004E851753FFFF6700E39C338453
:10D73000640383A70A003E948357040099E76304B7
:10D740000900232089008504C1BF4146D285130505
:10D75000440097100100E780605975F5A289E5B78C
:10D760001753FFFFE702039639717C083ED4B707D1
:10D770000A003ED67C083ED883C795002A8A3285A7
:10D7800093F7F707A384F5002E8932C697F0FFFFC1
:10D79000E78000B085676373F5083246AA84328556
:10D7A00097F0FFFFE780A0AC8547AA8963E8A7064A
:10D7B000A16593858504281097D0FFFFE78020B5E9
:10D7C000268597700000E78040872A8429ED9145DF
:10D7D000281097F0FFFFE780E09BA685281097F0C0
:10D7E000FFFFE780209DCE85281097F0FFFFE780A0
:10D7F000609A014781463010CA85528597D0FFFF55
:10D80000E78040D6A1679387770448183EDC230A57
:10D81000010202DE97F0FFFFE780607E216117536F
:10D82000FFFF6700638D8145281097F0FFFFE780B9
:10D830006096A685281097F0FFFFE780A09797973E
:10D84000FF1F938767AA9C4381CB228563890900C8
:10D8500097D00000E78040248345040271B797D039
:10D860000000E780C022CDBF1753FFFFE70283858A
:10D8700083C795004111AA8993F7F707A384F500A0
:10D880003285AE84328A97F0FFFFE78060A085671B
:10D89000637FF5022A8997600000E780007A2A8476
:10D8A000914631C58347F50105476387E70291C774
:10D8B0000D476366F704AD461DA8930505030325D0
:10D8C0000A00414697100100E78040420DE94101FE
:10D8D0001753FFFF670043829305950803250A004D
:10D8E000414697100100E7806040814669F54A860D
:10D8F000A6854E8597000000E780C081C9BF8325BB
:10D900000A001305940897700000E780A02919C148
:10D91000C146F1BF9787FF1F9387C7649C4399E770
:10D920009787FF1F9387C74D9C4399C72285978090
:10D930000000E780208A69FD8547A30FF400228557
:10D9400097B00000E7806084228597600000E78040
:10D95000E0734E8581464A86A68597F0FFFFE780F3
:10D96000607BA1679387570448003EC423020100EF
:10D9700002C697F0FFFFE780806891BF1743FFFF63
:10D98000E702637383C795004111AA8993F7F707EC
:10D99000A384F50032852E89B28A97F0FFFFE780D5
:10D9A000208F85676374F50EAA8497600000E78076
:10D9B000C0682A840DED416B014A978BFF1F938B42
:10D9C000EB5B130C400E7D1B19A833048A0383A75D
:10D9D0000B0B3E948357C40163836705050A97E0E8
:10D9E000FFFFE780008BE342AAFE95460DA0835718
:10D9F000C501639697029305050303A50A004146F6
:10DA000097100100E780802E994611E18146268615
:10DA1000CA854E8597F0FFFFE780C06F85A883A574
:10DA20000A001305040397700000E780A017C146A1
:10DA300079FD2285231E940097A00000E780E07402
:10DA4000228597600000E78060649797FF1F9387A7
:10DA5000A7899C43A9C323000402228597D0000014
:10DA6000E78040F04E8581462686CA8597F0FFFF05
:10DA7000E780406AA1679387070448003EC42302F9
:10DA8000010002C697F0FFFFE7806057410117438E
:10DA9000FFFF6700C36589472300F402E1B73971CE
:10DAA00006DE22DC4AD8800052D456D25AD026DA7A
:10DAB0004ED65ECE2E8A32892A8B97D0FFFFE78022
:10DAC000407A0605710541998A8A3301A1402322D3
:10DAD00024FC231404FC97D0FFFFE7808078834761
:10DAE0009A000605350593F7F7072315A4FCA30450
:10DAF000FA004A85232624FC97E0FFFFE78040795F
:10DB000093170501C1876340F0025681130104FC9D
:10DB1000F2506254D2544259B259225A925A025B7C
:10DB2000F24B21618280AA844A8597E0FFFFE7805B
:10DB30002076AA894A8597E0FFFFE7806075A16596
:10DB40009385C5022A89130544FC97C0FFFFE7802F
:10DB5000007C268597C0FFFFE7804070854511C98E
:10DB60004A86CE8597C0FFFFE780C069AA8B21E96E
:10DB70008945130544FC97E0FFFFE780A061A68577
:10DB8000130544FC97E0FFFFE780C062CE851305D4
:10DB900044FC97E0FFFFE780E061CA85130544FC81
:10DBA00097E0FFFFE780006101478146130644FCD0
:10DBB000D2855A8597D0FFFFE780C09AB9B78145D3
:10DBC000130544FC97E0FFFFE780C05CA6851305C2
:10DBD00044FC97E0FFFFE780E05DCE85130544FC41
:10DBE00097E0FFFFE780005DCA85130544FC97E0DE
:10DBF000FFFFE780205C814497D0FFFFE7806066ED
:10DC0000E3D4A4FA83A70B0113971400BA9783D522
:10DC1000070099C5130544FC97E0FFFFE780805992
:10DC20008504D9BF797106D622D44AD000184ECEC9
:10DC300052CC56CA26D25AC8AE893289AA8A97D0FF
:10DC4000FFFFE78000620605690541990A8A3301F2
:10DC5000A140232A24FC231C04FC97D0FFFFE7806B
:10DC6000406083C7990006052D0593F7F707231D2C
:10DC7000A4FCA384F9004A85232E24FC97E0FFFF2F
:10DC8000E780006193170501C187634FF00052815F
:10DC9000130104FDB250225492540259F249624ACF
:10DCA000D24A424B45618280AA844A8597E0FFFFB1
:10DCB000E780005EA1659385A5022A89130544FDCE
:10DCC00097C0FFFFE780A064268597C0FFFFE7802D
:10DCD000E058854509C9CA8597C0FFFFE780805590
:10DCE0002A8B29E18945130544FD97E0FFFFE78072
:10DCF000604AA685130544FD97E0FFFFE780804B4F
:10DD0000CA85130544FD97E0FFFFE780A04A01475D
:10DD10008146130644FDCE85568597D0FFFFE780E8
:10DD20006084B5B78145130544FD97E0FFFFE780A8
:10DD30006046A685130544FD97E0FFFFE780804716
:10DD4000CA85130544FD97E0FFFFE780A0468144A4
:10DD500097D0FFFFE780E050E3DBA4FA83270B01B5
:10DD600013971400BA9783D5070099C5130544FD8E
:10DD700097E0FFFFE78000448504D9BF1743FFFF0A
:10DD8000E702E33583474500404DD5EFFD575DC4BD
:10DD90008346940009476363D70A0346B400854667
:10DDA00063EEC6088306E40063CA06085C45F956BC
:10DDB0002390D7009787FF1F83C747FC99E3A304ED
:10DDC000E4009787FF1F9387A7039C4381E7894758
:10DDD000A306F4009787FF1F938707519C4381E7B1
:10DDE00089472306F4009705000093854506AA8419
:10DDF0001305040197F00000E7802010FD57231A57
:10DE0000F40281471CDC01489787FF1F23A487F693
:10DE10009787FF1F938747F6232E040304C0804390
:10DE200097D0FFFFE780204E61463306C50281454B
:10DE300022859740FFFFE780802D81473E8517436D
:10DE4000FFFF6700032CFD57D5BF1743FFFFE70215
:10DE500003292A840355450297600000E780E01DEE
:10DE600019E5231E04001743FFFF6700832983572A
:10DE7000E401F5DB930504FF17450100130545F0A8
:10DE800097E00000E780E014F9BF1743FFFFE702C7
:10DE900003252E89A16541119385E5032A8436C4A3
:10DEA00032C6BE843AC297C0FFFFE78040461247A1
:10DEB0002285BA8597E0FFFFE780C02D3246228594
:10DEC000B28597E0FFFFE780E02EA2462285B68567
:10DED00097E0FFFFE780002E63030902914522854A
:10DEE00097E0FFFFE780C0241146A6859710010048
:10DEF000E78020E241011743FFFF67008320894547
:10DF0000228597E0FFFFE780A02283C7040023005B
:10DF1000F50083C71400A300F500E9BF1743FFFF16
:10DF2000E702E31B83C79500444D054793F7F707C6
:10DF3000A384F5001C42411183C707006367F706FD
:10DF40002E842A89B1C003C7D400630FF702178754
:10DF5000FF1F1307E7EA184305C3A386F40097A041
:10DF60000000E780404A83C7D40099E741657D15EA
:10DF700097400000E780403083D72403918B89C706
:10DF800097E00000E780C0134A85A28597F0FFFF65
:10DF9000E7808010A167C10748003EC4230201004A
:10DFA00002C697F0FFFFE780800541011743FFFF9E
:10DFB000670023151743FFFFE702631203D74500ED
:10DFC0008D47AA8441112E8432892E8563E3E702AE
:10DFD00097E0FFFFE780C02BAA8523000900268574
:10DFE00097C0FFFFE780002541011743FFFF67004F
:10DFF000431197E0FFFFE780A0292AC6228597E01A
:10E00000FFFFE780E028B24585472A862300F90014
:10E01000268597C0FFFFE780E01EF9B7397106DE5D
:10E0200022DC26DA80004ED652D456D24AD85AD0B4
:10E030005ECEAE89B284AA8A97D0FFFFE7806021C6
:10E0400006051305250241990A8A3301A1402322BE
:10E0500024FC231404FC97D0FFFFE780801F83C7B4
:10E06000990006054D0593F7F7072315A4FCA38433
:10E07000F9002685232624FC97E0FFFFE780402156
:10E0800093170501C1876340F0025281130104FC1C
:10E09000F2506254D2544259B259225A925A025BF7
:10E0A000F24B21618280AA8B03AB040097C0FFFF73
:10E0B000E780C01A51E583D7440001498544F11730
:10E0C00093B71700A301F4FC834734FCA165C9C7CB
:10E0D0009385E504130544FC97C0FFFFE7802023E8
:10E0E000A685130544FC97E0FFFFE780A00ADE85C4
:10E0F000130544FC97E0FFFFE780C00B834734FC27
:10E10000114691E30946DA85130544FC97E0FFFFC9
:10E11000E78060058144630A0900416B7D1B97D04D
:10E12000FFFFE780001363CCA4020147814613067A
:10E1300044FCCE85568597C0FFFFE780A042B1B76B
:10E14000A685130634FC97000000E780E0E69334D0
:10E1500015002A8986048DBF9385C504A5BF832732
:10E16000C90013971400BA9783D507006388650127
:10E17000130544FC97E0FFFFE780C003850445B723
:10E180001743FFFFE70223F379711C103EC4B70762
:10E190000F003EC61C103EC883C79500AA8A328570
:10E1A00093F7F707A384F500AE89328497E0FFFF69
:10E1B000E780000E93170501C187635AF0062A8A8B
:10E1C000228597E0FFFFE780A00C2A895285032B68
:10E1D000040097C0FFFFE780600839ED83574400D3
:10E1E00081440544F11793B71700A303F100834559
:10E1F0007100DA872287CA865286280097000000BD
:10E20000E780E0C8014781463000CE85568597C03B
:10E21000FFFFE7802035A1679387D70348083ECCEE
:10E22000230A810026CE97F0FFFFE78040DD45619D
:10E230001743FFFF6700A3EBA28513067100970049
:10E240000000E78060D7AA84094455D13544E30033
:10E2500055FB4A8597F0FFFFE78000450D4441D903
:10E26000014497D0FFFFE780C0FE634DA400C16B5F
:10E270000144FD1B97D0FFFFE780A0FD634EA40083
:10E280001544B5B7DC4413171400BA9783D70700B9
:10E29000638327030504F1B7D84493171400BA9792
:10E2A00003D70700631B770123902701268597A0DA
:10E2B0000000E78080DB01441DBF050465BF1743F4
:10E2C000FFFFE70223E083C7950041112A8A93F7F5
:10E2D000F707A384F50032852E89328497E0FFFF8B
:10E2E000E78000FB93170501C1876353F006AA89F5
:10E2F000228597E0FFFFE780A0F92311A1004E855A
:10E30000832A040097C0FFFFE78040F539E5835773
:10E31000440085440144F11793B71700A300F100AE
:10E320000348110003572100D6875285CE862686E2
:10E33000CA8597F0FFFFE7806006A167F1074800F4
:10E340003EC42302910022C697F0FFFFE78020CB56
:10E3500041011743FFFF670023DAA285130611006E
:10E3600097000000E78040C52A84894455D9835727
:10E37000210011678544BA97C2071167C18313074B
:10E38000F7EFE36FF7F89787FF1F9387A7BD9C43CD
:10E3900081CB85451305210097500000E78020754B
:10E3A000835521002285814497C0FFFFE780A0E1CB
:10E3B00025D923100500228597A00000E78040CDD5
:10E3C00085B71743FFFFE70203CF83C795004111CD
:10E3D0002A8B93F7F707A384F50032852E8A3284BF
:10E3E00097E0FFFFE780C0EA93170501C1876351FB
:10E3F000F006AA8A228597E0FFFFE78060E92A8974
:10E400005685832B040097C0FFFFE78020E531E5A8
:10E410008357440081440544F11793B71700A301C3
:10E42000F10003483100DE875A854A87D686228666
:10E43000D28597F0FFFFE78060F6A167ED074800FF
:10E440003EC42302810026C697F0FFFFE78020BB71
:10E4500041011743FFFF670083C9A28513063100FE
:10E4600097000000E78040B5AA8409445DD9916710
:10E47000CA97C2071167C1831307F7EF0544E36228
:10E48000F7FACA8597C0FFFFE780E0D3014451F94E
:10E49000814997D0FFFFE780C0DC63DBA900984883
:10E4A00093971900BA9703D7070005EF2390270128
:10E4B00097D0FFFFE780E0DA1544E384A9F62685CC
:10E4C00097A00000E780C0BC9787FF1F938787A9AC
:10E4D0009C430144B9D74A8597500000E780C05853
:10E4E00089B785097DB71743FFFFE702A3BD79719F
:10E4F0003E847C083EC82E8AB7071400A1653ECA38
:10E50000E5057C08AA89080836C4428932C6BA8A59
:10E51000C6843ECC97C0FFFFE78060DFCA8508084D
:10E5200097E0FFFFE78000C732460808B28597E012
:10E53000FFFFE78020C8A246630A09049D4508083A
:10E5400097E0FFFFE780C0BE1D4681459740FFFF73
:10E55000E780E0BB63890A089145080897E0FFFF60
:10E56000E78000BD1146A68597000100E780607A2C
:10E57000100801478146D2854E8597C0FFFFE7808E
:10E5800060FE45611743FFFF670003B7B6850808C3
:10E5900097E0FFFFE78000C21C400808D84393556E
:10E5A000C701858912075183B205D98D97E0FFFF16
:10E5B000E78040C01C40080883C5870097E0FFFF44
:10E5C000E78040BD1C40080883C5A70097E0FFFF17
:10E5D000E78040BC1C40080883C5970097E0FFFF18
:10E5E000E78040BB85BF8945080897E0FFFFE780CB
:10E5F00020B483C704002300F50083C71400A300E0
:10E60000F500BDB71743FFFFE702C3AB83C7950013
:10E610004111AA8993F7F707A384F5003285AE84E8
:10E62000328497E0FFFFE780A0C693170501C187FA
:10E63000635DF0042A89032A040097C0FFFFE78086
:10E64000E0C119E9835744000548F11793B7170053
:10E65000A307F100814631A81306F100A2859700B7
:10E660000000E78060951DC51C459DC783D6470007
:10E6700001480347F10093078500D2884A86A685A2
:10E680004E8597000000E78040E641011743FFFFF9
:10E69000670083A609487DBF1D486DBF1743FFFF74
:10E6A000E70243A265715C083EC4B7077B013EC622
:10E6B0005C083EC883C795002A8A328593F7F7071E
:10E6C000A384F500AE8997E0FFFFE78040BA835747
:10E6D000E100E1C78945280097C0FFFFE78020C31C
:10E6E0008145280097E0FFFFE780C0AA97C0FFFFA1
:10E6F000E78000C99787FF1F938707BF9C43177464
:10E70000FF1F0344A467AA843334800099C31364B1
:10E7100024009777FF1F9387A76E9C4399C31364C8
:10E7200044009787FF1F9387E7839C4399C3136433
:10E73000840083D504002800014997E0FFFFE780AB
:10E7400060A783D52400280097E0FFFFE78080A61C
:10E7500083D54400280097E0FFFFE780A0A597D06D
:10E76000FFFFE78000AB93150501C181280097E00A
:10E77000FFFFE78020A4A285280097E0FFFFE78045
:10E7800060A39C446360F902014781463000CE8556
:10E79000528597C0FFFFE780E0DC59611743FFFF18
:10E7A00067008395DC441314490028003E9497E0E9
:10E7B000FFFFE780609683474400034754008907C2
:10E7C0000607BA978607E36AF5FC835524002800FC
:10E7D000814A97E0FFFFE780E09D834544002800E1
:10E7E00097E0FFFFE780009B83455400280097E0F7
:10E7F000FFFFE780209A8347440063C9FA00814AFB
:10E800008347540063C1FA020509A5BF1C4413974E
:10E810005A002800BA9783D50700850A97E0FFFFC2
:10E82000E7804099C9BF032BC40093975A00280082
:10E830003E9B83552B00850A97E0FFFFE78080977A
:10E8400083550B00280097E0FFFFE780A0964DBF9F
:10E850001743FFFFE702A3885C4993E717005CC9F1
:10E8600097A00000E78020B61743FFFF6700638989
:10E870001743FFFFE702A3862E84814597F0FFFF31
:10E88000E780C0E705C583570500FD172310F50095
:10E8900009C4835725002310F40097000000E78087
:10E8A00060FB01451743FFFF6700A38531457DD815
:10E8B00023100400C5BF1743FFFFE702A38083C7EF
:10E8C000950041112A8A93F7F707A384F500328552
:10E8D0002E89328497E0FFFFE780809B9317050124
:10E8E000C1876356F006AA89C145228597E0FFFFDC
:10E8F000E780A0802A8B4E85832A040097C0FFFF03
:10E90000E780C09531E98357440023110100054495
:10E91000F11793B71700A300F100814403481100D9
:10E9200003572100D6875285CE862286CA8597F066
:10E93000FFFFE780A0A6A1679387170248003EC4A7
:10E940002302810026C697E0FFFFE780406B41016C
:10E950001733FFFF6700437A13061100A28597F073
:10E96000FFFFE7806065AA8409E5231101000944DF
:10E9700075B7930521005A8597000000E78080EF66
:10E98000835721002A84D9DB9777FF1F9387875D00
:10E990009C4381CB85451305210097500000E780FB
:10E9A0000015835521002685314497C0FFFFE7807D
:10E9B00080812DD523100500268597900000E780E3
:10E9C000206D0144A1BF1733FFFFE70243714111DE
:10E9D0002E896C00AA8402C697F0FFFFE78000D260
:10E9E0000DC10357050005072310E500970000003F
:10E9F000E78040E681473E8541011733FFFF67000E
:10EA000043703247954765DBCA85268597300000FD
:10EA1000E780400DC147E34005FE3244854741464B
:10EA20002310F40083570900A68513054400231121
:10EA3000F40097000100E780C02D228545BF173301
:10EA4000FFFFE702236883C795004111AA8A93F765
:10EA5000F707A384F5003285AE89328497E0FFFF83
:10EA6000E780008393170501C1876356F0062A8A61
:10EA7000C145228597D0FFFFE7802068AA84528590
:10EA8000032B040097B0FFFFE780407D31E98357F7
:10EA90004400231101008544F11793B71700A30028
:10EAA000F10001440348110003572100DA8756851D
:10EAB000D2862686CE8597F0FFFFE780208EA1675D
:10EAC0009387070248003EC42302910022C697E0C4
:10EAD000FFFFE780C05241011733FFFF6700C361AA
:10EAE000A2851306110097F0FFFFE780E04C2A840F
:10EAF00009E523110100894475B726859305210096
:10EB000097000000E78060ECAA8449FD835521004E
:10EB1000228597B0FFFFE780006B49F5014997C058
:10EB2000FFFFE7800074635DA90018489317190080
:10EB3000BA9703D707000DEF035721002390E70092
:10EB400097C0FFFFE780E071630625039777FF1FFB
:10EB5000938747419C4399C7035521009750000074
:10EB6000E78080F0228597900000E78060521DBF0B
:10EB7000050975B795443DB705C19307F00F630FBD
:10EB8000F500C547630CF5009307F5FF0545331500
:10EB9000F5004205418182800145828041657D15F5
:10EBA0008280B9E91733FFFFE70263530345060389
:10EBB000328497000000E78060FC9305803EB30537
:10EBC000B502C205C18181CD0357E402854763F8D0
:10EBD000E7001305040197E00000E7802042835717
:10EBE000E40241677D176385E700FD172317F402F0
:10EBF0001733FFFF6700E35082801733FFFFE70200
:10EC0000834B004283C79500444D0349140093F79A
:10EC1000F707A384F50083470400220911673369CD
:10EC2000F900A167B347F90041112A8BAE8A63EC62
:10EC3000E70E834724001307C00EB91793F7F70FA9
:10EC40006373F71003473400C14763EEE70E834751
:10EC500044001307E00793C707086371F70C834963
:10EC6000840083477400A209B3E9F900856763F75C
:10EC7000F90A034A6400834754004E85220A336A26
:10EC8000FA0097500000E780403B61C123962403BF
:10EC9000834B3400137AFA00239A340323887403D5
:10ECA0002399440393890401631C090023A60402E9
:10ECB000239804024E8597E00000E78060363DA06F
:10ECC000034924004A8597000000E78020EB239742
:10ECD000A402834744004E85A388F402E38D0BFC15
:10ECE000E30B09FC97E00000E780202F97900000DD
:10ECF000E780007381460146D6855A8597E0FFFF7D
:10ED0000E7800058A167938797033EC42302010060
:10ED1000480002C697E0FFFFE780602E41011733ED
:10ED2000FFFF6700C33C8544A2862686D6855A85A8
:10ED300097E0FFFFE780C054A167938797033EC425
:10ED400023029100F1B7BD44C5B79144F1BF173319
:10ED5000FFFFE702233701111C08404D3EC2B707F1
:10ED60000F003EC41C083EC62A89AE8997C0FFFF2B
:10ED7000E78000D7585C1C5C6346B70E6394E500DF
:10ED800063E2A70E3385A740B3B7A700B305B7402A
:10ED90001306803E81469D8D97000100E78080B775
:10EDA00093140501C180A1659385C503480097B000
:10EDB000FFFFE780C0558145480097D0FFFFE780FF
:10EDC000603D83550404480097D0FFFFE780803EF4
:10EDD00083552404480097D0FFFFE780A03D81457C
:10EDE00089CCC167FD179305F00F6388F400268571
:10EDF00097500000E780E0E0AA85480097D0FFFF29
:10EE0000E780403903554404814501CDC167FD17B2
:10EE10009305F00F6307F50097500000E78060DE70
:10EE2000AA85480097D0FFFFE780C0368345640479
:10EE3000480097D0FFFFE780E03583457404480021
:10EE400097D0FFFFE7800035500001478146CE850F
:10EE50004A8597B0FFFFE780E07005611733FFFF39
:10EE600067008329814481B71733FFFFE702232717
:10EE700083C7950093F7F707A384F5009700000078
:10EE8000E78020ED1733FFFF6700A3271733FFFF4D
:10EE9000E702432383C795004111404D93F7F707DD
:10EEA000A384F5002A8A3285B284AE8997D0FFFF09
:10EEB000E780003E2A8B268597D0FFFFE780403D04
:10EEC0002A89268597D0FFFFE780603A93170B01C8
:10EED00063CA0702E177CA97C207C183116763E378
:10EEE000E70293070910C207C1831307B00F637BC2
:10EEF000F70093170901C187AA8A634AF000C54742
:10EF000063FE570141011733FFFF6700E31E97B00F
:10EF1000FFFFE7802025E31725FFD5B763080B0225
:10EF200063060902814463890A02B7077F00231040
:10EF30006405231124057CC0568597000000E780F6
:10EF4000E0C39304803EB304950239A0B7077F0065
:10EF5000232004047CC081440355240497E000006E
:10EF6000E780A0A3A1C497C0FFFFE78060B7269504
:10EF700093D7F44133379500AE97BA9708DC5CDC41
:10EF8000CE85528597000000E780A0DC99E023221F
:10EF90000404A1679387B70348003EC4230201001D
:10EFA00002C697E0FFFFE7808005A9BF81470148BF
:10EFB0001CDC232E0403E9B71733FFFFE7022312FB
:10EFC00097C0FFFFE7802034E1473305F502914504
:10EFD00097500000E78000C5E55711C59777FF1FE0
:10EFE00023ACA7D881473E851733FFFF6700631125
:10EFF00085471777FF1F2303F7D882801733FFFF5A
:10F00000E702E30D9777FF1F9387C7D680433DC084
:10F01000835704046390A70683572404639CB704B2
:10F020003689B28497C0FFFFE78080AB5C5C63C326
:10F03000B7046395B7001C5C63EEA70283476404C2
:10F0400063F3F400A6872303F4048347740463F393
:10F050009700A687A303F4048357440441677D17F0
:10F060006385E70085072312F4043C4481C7CA8501
:10F07000268582971733FFFF6700A3089777FF1F46
:10F08000938747CF9C43014599C303C5870082807E
:10F090001733FFFFE702A3040111B70707003EC6BD
:10F0A00083C79500584D0AC493F7F7070AC8A3848D
:10F0B000F5002A89AE8411CB1C4283C707002304C4
:10F0C000F70097900000E780003421649305540214
:10F0D000280097B0FFFFE780802397000000E780BB
:10F0E00020FAAA85280097D0FFFFE780A00A300009
:10F0F00001478146A6854A8597B0FFFFE780804695
:10F1000013044402480822CC230A010002CE97E0EF
:10F11000FFFFE780C0EE05611733FFFF670063FE66
:10F120001733FFFFE702A3FB01117C003ECAB707BC
:10F1300007003ECC7C003ECE83C795002E84AA8477
:10F1400093F7F707A384F500A16593855502480856
:10F1500097B0FFFFE780A01B97000000E78040F218
:10F16000AA85480897D0FFFFE780C00250080147F2
:10F170008146A285268597B0FFFFE780A03E056106
:10F180001733FFFF6700E3F79777FF1F938787BE6B
:10F190009C43094599C303C5970082809777FF1F59
:10F1A000938747BD9C43094599C303C5D700828017
:10F1B0009777FF1F938707BC9C43014599C303C5FD
:10F1C000A70082801733FFFFE702C3EF0111B707E3
:10F1D00008003EC683C79500404D0AC493F7F70761
:10F1E0000AC8A384F5002A89AE8429C4144285473D
:10F1F00003C7060063E0E70A834794000946814994
:10F200006380C702B307F740A304E400B339F000FA
:10F2100083C716002305F40097900000E780A01E26
:10F2200003572403058B19C76386090097D0000094
:10F23000E78000E9216493058402280097B0FFFF6E
:10F24000E780E00C97000000E78040F4AA852800E2
:10F2500097D0FFFFE78000F497000000E78080F57B
:10F26000AA85280097D0FFFFE780C0F201478146BA
:10F270003000A6854A8597B0FFFFE780A02E1304D3
:10F280007402480822CC230A010002CE97E0FFFF57
:10F29000E780E0D605611733FFFF6700E3E517332A
:10F2A000FFFFE702C3E301117C003ECAB707080075
:10F2B0003ECC7C003ECE83C795002E84AA8493F773
:10F2C000F707A384F500A16593858502480897B0E8
:10F2D000FFFFE780C00397000000E78020EBAA85CE
:10F2E000480897D0FFFFE780E0EA97000000E7803A
:10F2F00060ECAA85480897D0FFFFE780A0E9500896
:10F3000001478146A285268597B0FFFFE7808025CB
:10F3100005611733FFFF6700C3DE9777FF1F9387F1
:10F3200067A59C43014599C303C5B7008280173385
:10F33000FFFFE702C3DA0111B70707003EC683C724
:10F340009500404D0AC493F7F7070AC8A384F50057
:10F350002A89AE8405C81C42054783C70700636835
:10F36000F7060347B400630FF700A305F400979076
:10F370000000E78040098347B400B9CF97D0FFFF72
:10F38000E78040BE21649305B400280097B0FFFFDA
:10F39000E780E0F797000000E78060F8AA85280082
:10F3A00097D0FFFFE78000DF014781463000A68548
:10F3B0004A8597B0FFFFE780E01A2904480822CC6D
:10F3C000230A010002CE97E0FFFFE78040C30561FA
:10F3D0001733FFFF6700E3D297D0FFFFE78020BF1E
:10F3E00055B71733FFFFE70283CF01117C003ECAF8
:10F3F000B70707003ECC7C003ECE83C795002E8425
:10F40000AA8493F7F707A384F500A165AD05480822
:10F4100097B0FFFFE780A0EF97000000E78020F0A3
:10F42000AA85480897D0FFFFE780C0D6500801475B
:10F430008146A285268597B0FFFFE780A01205616F
:10F440001733FFFF6700E3CB9777FF1F9387879200
:10F450009C43094599C303C5C70082801733FFFF4A
:10F46000E702E3C701117C00AE843ECAA165B7077D
:10F4700007002A843ECCD1057C0048083ECE97B0D8
:10F48000FFFFE780C0E897000000E78020FCAA8526
:10F49000480897D0FFFFE780E0CF5008014781463A
:10F4A000A685228597B0FFFFE780C00B0561173363
:10F4B000FFFF670003C51733FFFFE70243C283C79F
:10F4C000950093F7F707A384F50097000000E78005
:10F4D00020F91733FFFF6700C3C21733FFFFE702AE
:10F4E00063BE83C795000329C501411193F7F70750
:10F4F000A384F5001C4283C90700854763E63707EC
:10F500009777FF1F938747DE9C432E84AA8485CF7D
:10F5100097000000E78080F389476306F5026304E3
:10F5200009028347C9006380370323063901979096
:10F530000000E78040ED83572903898B89C797D066
:10F540000000E780E0B72685A28597000000E780ED
:10F5500020F1A167CD0748003EC42302010002C686
:10F5600097E0FFFFE780A0A941011733FFFF670085
:10F57000A3B89767FF1F9387E77F9C431D4599C3F7
:10F5800003C5E70082801733FFFFE70243B501118F
:10F59000B70707003EC683C79500584D0AC493F7C6
:10F5A000F7070AC8A384F5002A89AE8415C71C4250
:10F5B00083C7070093968701E18663C406068546E4
:10F5C0006381D7068346E7006388F6002307F700C8
:10F5D00097900000E78020E321649305E400280071
:10F5E00097B0FFFFE780A0D297000000E780A0F867
:10F5F000AA85280097D0FFFFE780C0B90147814660
:10F600003000A6854A8597B0FFFFE780A0F5350456
:10F61000480822CC230A010002CE97E0FFFFE780D2
:10F62000009E05611733FFFF6700A3AD1733FFFF8F
:10F63000E702E3AA01117C003ECAB70707003ECCEF
:10F640007C003ECE83C795002E84AA8493F7F707EB
:10F65000A384F500A165B905480897B0FFFFE780CE
:10F6600000CB97000000E78000F1AA85480897D0FA
:10F67000FFFFE78020B2500801478146A28526851A
:10F6800097B0FFFFE78000EE05611733FFFF6700CB
:10F6900043A71733FFFFE702E3A2AA8401441769D7
:10F6A000FF1F1309696DE14997C0FFFFE780A0C5FF
:10F6B0006344A400014519A83305340383270900D6
:10F6C0003E95835725006397970011051733FFFF79
:10F6D000670083A20504C9BF032E8500630A0E12CA
:10F6E0001773FF1F1303038803230300631503002D
:10F6F00029436390061203234E01631503001D4343
:10F70000639907101733FFFFE702E39AC689428A1D
:10F710003E89BA8AB684328BAE8B2A84B5E1035512
:10F720004E0019E501431A851733FFFF6700239C3C
:10F73000A167A98F116763FBE70097000000E780CE
:10F7400080F5814597F0FFFFE780C0120844B707B6
:10F7500000E05841F98F18455CC1B707001FF98FC9
:10F760001CC55C4991C7610597E00000E780408BAC
:10F77000E38A09FA228597900000E78060C65DB7AA
:10F78000328597C00000E78040430D4349DD1C44AB
:10F79000116703D54700A167A98F63FBE7009700B6
:10F7A0000000E78040EF814597F0FFFFE780800C85
:10F7B0000323840093164B01D1828347B300035681
:10F7C00063008588FD8BA305F300FD777D8E558E44
:10F7D000FD76FD16B204F18E83274301C58E2312F8
:10F7E00073012313D3002304530123052301A3042E
:10F7F0004301BDDF228597B0FFFFE78080C9AA855E
:10F800000844B5D1610597D00000E780207F8DB70F
:10F810001D431A8582801733FFFFE702A38A05691B
:10F82000AA84AE89328A0144FD5A7D1997C0FFFF30
:10F83000E78020A26347A40001451733FFFF67005C
:10F84000A38BD84493171400BA9703D70700631FFC
:10F8500037032390570163070A002685979000001D
:10F86000E780A0809C449DC383D76700B3F727013E
:10F87000639E3701D288014881470147814601468E
:10F880008145268597000000E78040E5050479BFA3
:10F890001733FFFFE702038379711C103EC4B707DB
:10F8A0000F003EC61C103EC883C79500AA8A328549
:10F8B00093F7F707A384F5002E89328497D0FFFFD2
:10F8C000E780009D93170501C187635AF006AA8956
:10F8D000228597D0FFFFE780A09B2A8A4E85032BC5
:10F8E000040097B0FFFFE780609739ED835744002D
:10F8F00081440544F11793B71700A303F100834532
:10F900007100DA872287D2864E86280097E0FFFFB3
:10F91000E780E057014781463000CA85568597B099
:10F92000FFFFE78020C4A1679387F70348083ECC18
:10F93000230A810026CE97D0FFFFE780406C456107
:10F940001723FFFF6700437BA2851306710097E032
:10F95000FFFFE7806066AA84094455D1528597E08D
:10F96000FFFFE78060D40D4459D90546D28526852E
:10F9700097000000E78060EA2A8451B71723FFFF51
:10F98000E702E375835507000346270041112A84E7
:10F990002E8532C62EC497E0FFFFE780E0D001C974
:10F9A0003246A245228597000000E78000E741012A
:10F9B0001723FFFF6700E3741723FFFFE702A36F1E
:10F9C00083C795004111AA8A93F7F707A384F5002E
:10F9D0003285AE89328497D0FFFFE780608B931722
:10F9E0000501C1876357F00AC1452A8A228597C05D
:10F9F000FFFFE78080702A8D228597D0FFFFE78088
:10FA000020892A89228597D0FFFFE78040869307C7
:10FA100005F893F7F70F1307E007AA8B637BF70648
:10FA2000228597D0FFFFE78080842A8C228597D09B
:10FA3000FFFFE780C083AA8C5285032B040097B098
:10FA4000FFFFE780A08139E98357440023110100BB
:10FA50008144F11793B71700A300F1000544034751
:10FA6000110083562100938784005685DA88228806
:10FA70005286CE8597F0FFFFE78020A7A167E907B0
:10FA800048003EC42302810026C697D0FFFFE780CE
:10FA9000005741011723FFFF67006365130611003C
:10FAA000A28597E0FFFFE7802051AA8409E5231192
:10FAB000010009446DB7930521006A8597F0FFFFA7
:10FAC000E780A0F02A8441FD835521009356C900A8
:10FAD0001316490185486688E2875E87858A5182C8
:10FAE000268597000000E78060BF2A848DBF17231A
:10FAF000FFFFE702435C83C7950041112A8B93F710
:10FB0000F707A384F5003285AE89328497C0FFFFE2
:10FB1000E780007893170501C1876352F00A2A8AAB
:10FB2000228597C0FFFFE780A076AA8A228597C02A
:10FB3000FFFFE780E0752A89228597C0FFFFE780F5
:10FB40000073930705F893F7F70F1307E0072A8C64
:10FB50006377F706228597C0FFFFE7804071AA8C84
:10FB6000228597C0FFFFE78080702A8D5285832B06
:10FB7000040097A0FFFFE780606E39E583574400DB
:10FB800085440144F11793B71700A301F10003471F
:10FB90003100930784005A85DE882688D6865286EF
:10FBA000CE8597F0FFFFE78040948D4748003EC424
:10FBB0002302910022C697D0FFFFE7804044410115
:10FBC0001723FFFF6700A352A2851306310097E0B9
:10FBD000FFFFE780603E2A84894455D99356C900C7
:10FBE0001316490185486A88E6876287858A5182AB
:10FBF000D68597000000E78060AEAA8449BF17232E
:10FC0000FFFFE702234C2A8981440144617A916A0B
:10FC1000176BFF1F130B0B3597B0FFFFE780606476
:10FC200063C7A40022851723FFFF6700E34C8327E7
:10FC3000090093991400CE9703D5070033074501B7
:10FC4000420741836364570305C103270B0019C7AB
:10FC500085453E8597400000E78060E983270900DD
:10FC60000504CE972390070085047DB79700000018
:10FC7000E78060A2832709000504CE972390070040
:10FC800065D5814597F0FFFFE780C0BEF1BF172320
:10FC9000FFFFE702234383C7950041112A8A93F7A8
:10FCA000F707A384F50032852E89328497C0FFFFC1
:10FCB000E780005E93170501C187635AF004AA89A3
:10FCC000832A040097A0FFFFE780405931E583575E
:10FCD000440085440144F11793B71700A301F100D4
:10FCE00003483100D68752850147CE862686CA85CD
:10FCF00097D0FFFFE780806AA167F50748003EC400
:10FD00002302910022C697D0FFFFE780402F4101D8
:10FD10001723FFFF6700433EA2851306310097E0DB
:10FD2000FFFFE78060292A8489445DD99767FF1F18
:10FD3000938747239C4381CF044997B0FFFFE78017
:10FD40004052AA85268597400000E78040DA1305D7
:10FD5000040197000000E780C0EA22859780000038
:10FD6000E78000338144ADBF1723FFFFE702A334D0
:10FD700083C795004111AA8A93F7F707A384F5007A
:10FD80003285AE8932842311010097C0FFFFE780DE
:10FD9000205093170501C1876354F0062A8AC14594
:10FDA000228597C0FFFFE7804035AA8B5285032B41
:10FDB000040097A0FFFFE780604A21E983574400D1
:10FDC00085440144F11793B71700A300F1000348DD
:10FDD000110003572100DA875685D2862686CE8504
:10FDE00097D0FFFFE780805BA167938727024800D9
:10FDF0003EC42302910022C697D0FFFFE780202057
:10FE000041011723FFFF6700832EA285130611000F
:10FE100097E0FFFFE780401A2A8489444DD997670D
:10FE2000FF1F9387271498433E8901CF044997B059
:10FE3000FFFFE7800043AA85268597400000E78002
:10FE400000CB1305040197000000E78080DB97B02A
:10FE5000FFFFE780004195443DD9930521005E8571
:10FE600097F0FFFFE78060B6AA8435F11C4803577E
:10FE7000210022852390E70097800000E780402141
:10FE800083270900A9D70355210097400000E78088
:10FE9000A0BD35BF1723FFFFE702E32183C795000D
:10FEA0004111AA8A93F7F707A384F5003285AE893A
:10FEB000328497C0FFFFE780A03D93170501C187FB
:10FEC0006351F0062A8A228597C0FFFFE780403CF5
:10FED0002A895285032B040097A0FFFFE780003892
:10FEE00031E58357440085440144F11793B7170067
:10FEF000A301F10003483100DA8756854A87D2868C
:10FF00002686CE8597D0FFFFE7804049A167F90795
:10FF100048003EC42302910022C697D0FFFFE7802D
:10FF2000000E41011723FFFF6700631CA285130623
:10FF3000310097E0FFFFE78020082A8489445DD9DB
:10FF40009167CA97C2071167C1831307F7EF85440A
:10FF5000E362F7FA9767FF1F9387C7009843BE8B4A
:10FF600001CF044997B0FFFFE780A02FAA8526851F
:10FF700097400000E780A0B7130504019700000038
:10FF8000E78020C897B0FFFFE780A02D95443DD1C2
:10FF90001C48228581442390270197800000E78038
:10FFA000200F83A70B00B9D74A8597400000E78050
:10FFB000A0AB89B71723FFFFE70263122A8441052C
:10FFC000B28497000000E780C0C311C522859780E6
:10FFD0000000E780E00B81460146A68522859780D8
:10FFE0000000E780C04E1C4C89C7DC4799C32285BE
:10FFF00082971723FFFF6700C3109767FF1F938740
:020000040001F9
:1000000067D79C43014599C3138507018280976791
:10001000FF1F938727D6884382801723FFFFE702BD
:10002000030C9317C600DD8DC2054111C1812A84DE
:1000300032C697C0FFFFE780E01732462285118263
:100040009375F60F97C0FFFFE780C0144101172397
:10005000FFFF6700030B1723FFFFE702A306797179
:100060003C083ED2B7070C003ED43C083ED683C7BE
:100070009500AE842A8993F7F707A384F500A1655C
:1000800093853504481097A0FFFFE7804028C1659D
:10009000FD150144176AFF1F130A4AEE930A400E2A
:1000A000AE892E8B2EC697B0FFFFE780801E4205DB
:1000B000931704014181C183B24563E9A702C16777
:1000C000FD176387F500481097C0FFFFE780800E9B
:1000D000501001478146A6854A8597A0FFFFE7801B
:1000E000604845611723FFFF67000301330754038E
:1000F00083270A0BBA9703D6C701630A3601638ABE
:100100003501481097000000E78060F1DA850504AA
:1001100051BFB285EDBF1723FFFFE702C3F9797125
:100120007C083EC8B70711003ECA7C083ECC83C796
:100130009500AA89328593F7F707A384F5002E89E5
:1001400097C0FFFFE780C01485676378F504A16559
:10015000AA848905080897A0FFFFE780401B268531
:1001600097400000E78060ED133415000A04A28573
:10017000080897C0FFFFE780E001A685080897C040
:10018000FFFFE780200325CC014781461008CA8580
:100190004E8597A0FFFFE780E03C45611723FFFFF6
:1001A0006700E3F4B30754030327CA0ABA9703D7D7
:1001B0000700631C970003D62700638065050808C5
:1001C00097000000E780A0E5DE8505042EC697B005
:1001D000FFFFE780000D4205931704014181C183B1
:1001E000B245E3E1A7FCC167FD17E38FF5F8080806
:1001F00097C0FFFFE78000FC41BFB285F9B7C1653A
:10020000FD150144176AFF1F130A4AD7930A80029B
:100210002E8BAE8B65BF1723FFFFE70243EC18411F
:100220008347170083460700A207D58FD207D183E3
:100230002390F50083472700034717008D45A20749
:10024000D98F91832310F60097C0FFFFE780A0E9C4
:100250001723FFFF6700E3EA1723FFFFE70283E6A8
:10026000C16401441769FF1F130949D19309800232
:10027000FD1497B0FFFFE780C0026347A40001456B
:100280001723FFFF670043E7330534038327C90AB9
:100290003E9583570500E38597FE0504D9BF1723D4
:1002A000FFFFE70223E22A8AAE89B284B68A97402A
:1002B0000000E78080D819E591473E851723FFFFAE
:1002C000670083E32A894E8597C00000E780E08EAF
:1002D0002A84638E0A048D476DD103570500C547F4
:1002E000E31D47FD0347F9018546AD47E317D7FCFA
:1002F0008347450081CF4146A6855D0597F0000004
:10030000E780C09E814755D9AD4745BF13096501B8
:100310002302E500CA85268597100000E780606209
:1003200031C1A547E38B0AF82302040079B705C160
:1003300083570500E39247F94146A685190597F0D2
:100340000000E780A09A81472DD99947BDB74E8517
:1003500097000000E78080F02A84954739DD130973
:1003600055004DBF4146A685231044012311340199
:100370001305190097F00000E780A0992285978067
:100380000000E780A0EA81470DBF1723FFFFE702C7
:1003900003D579717C003ECCB7070A003ECE7C00C5
:1003A0003ED083C79500B2842E8493F7F707A384C9
:1003B000F5001306A1002A892C002685970000006D
:1003C000E780A0E5A16528088D0597A0FFFFE780DD
:1003D00000F490408355A1000355810085469700A5
:1003E0000000E78000ECAA84AA85280897C0FFFFD8
:1003F000E78040DA0356A100835581002808970062
:100400000000E780C0C1300801478146A2854A85C7
:1004100097A0FFFFE7800015854748103ED42302D0
:10042000910202D697D0FFFFE78060BD4561172398
:10043000FFFF670003CD1723FFFFE70243CA79716F
:100440007C003ECCB7070A003ECE7C003ED083C77E
:100450009500B2842E8493F7F707A384F500130662
:10046000A1002A892C00268597000000E780E0DAA9
:10047000A16528088D0597A0FFFFE78040E990401F
:100480008355A10003558100814697000000E78055
:1004900040E1AA84AA85280897C0FFFFE78080CFA3
:1004A0000356A10083558100280897000000E780CB
:1004B00000B7300801478146A2854A8597A0FFFF13
:1004C000E780400A48102302910202D402D697D056
:1004D000FFFFE780C0B245611723FFFF670063C2DB
:1004E0001723FFFFE702A3BF97000000E78060DB50
:1004F0001723FFFF6700E3C09767FF1F9387C78736
:10050000884382801723FFFFE70263BD83572500DE
:100510004111AE842A842307B10017F5FFFF1305AC
:1005200025466C002316F10097A0FFFFE780804569
:1005300091C4228597800000E780E0D6FD57231004
:10054000F400130620028145130554009720FFFF95
:10055000E780E0BB41011723FFFF670083BA172341
:10056000FFFFE70223B679717C003ECCB7070A0093
:100570003ECE7C003ED083C79500AA89AE8493F717
:10058000F7073285A384F5001306A1002C0097001D
:100590000000E78080C803558100114497400000A7
:1005A000E780A0A915C50355A100014497B000003C
:1005B000E780A06011CD03570500835781004544B3
:1005C0006318F700854597000000E780E0F30144D9
:1005D000216993053900280897A0FFFFE78020D301
:1005E000A285280897C0FFFFE780C0BA0356A10084
:1005F00083558100280897000000E78040A230085A
:1006000001478146A6854E8597A0FFFFE78080F5CC
:1006100048104AD42302810202D697D0FFFFE78018
:10062000009E45611723FFFF670003AD1723FFFFFF
:10063000E70243A99757FF1F9387C7732A8488430C
:100640002E8915C5035745038357C4016311F7026B
:100650002326050223180502410597D00000E780F4
:10066000209C6306090097800000E78060DB8144DE
:100670009769FF1F93898990130A800297B0FFFF43
:10068000E78020C263C4A4049757FF1F938747776E
:100690009C4399C70355C40197200000E780C0BD63
:1006A00063070900228597800000E780C0A0130639
:1006B000400E814522859720FFFFE78040A5FD572A
:1006C000231EF4001723FFFF670003A333854403B1
:1006D00083A7C90A3E95035705008357C4016317D2
:1006E000F700CA8597000000E78000E2850479B72B
:1006F0001723FFFFE702039D83C795004111AA89D5
:1007000093F7F707A384F5003285AE8497C0FFFF07
:10071000E78000B885676378F5042A899740000070
:10072000E780A091014401CD83D704003144638860
:100730002701854597000000E78080EF01444E8542
:10074000A2864A86A68597D0FFFFE780A09CA16776
:100750009387170448003EC42302810002C697D045
:10076000FFFFE780C08941011723FFFF6700C3989F
:100770001723FFFFE70203959757FF1F9387875FB4
:10078000804329C4014597C00000E78000218147CC
:100790000148C1641CDC232E0403232004041759E0
:1007A000FF1F1309A97D01449309400EFD1497B062
:1007B000FFFFE78000AE634FA400814517F5FFFF00
:1007C0001305857F97A0FFFFE780C01B1723FFFF5E
:1007D00067008392330534038327090B3E958357C3
:1007E000C50163879700854597000000E78040E4D6
:1007F000050475BF9357050113D78700A380F50043
:1008000093170501C183A1832380E5002381F500AF
:10081000A381A50082801723FFFFE702438C2300FA
:10082000050083C71500A300F50083C72500230139
:10083000F50083C73500A301F50083C745002302F7
:10084000F50083C75500A302F50083C76500930533
:100850009500A30305002303F5002304050032855A
:1008600097000000E78040F91723FFFF67006389C6
:100870001723FFFFE70203854111E9540DCD85CD14
:1008800093F9C5FF2E842A89AA84338AA900B7EA7E
:10089000040063189A020D88854411CCB7E7040060
:1008A0009C5F82972AC622866C003305390197E047
:1008B0000000E7800046268541011723FFFF6700FF
:1008C000A38383A78A039104829793170501C183A9
:1008D000A183A38EF4FE93570501238FF4FEA18319
:1008E000238EA4FEA38FF4FE6DB763E6D502171323
:1008F000FFFFE702C37EB28741113686BE8536C64A
:1009000097E00000E780E040B246410136851713CA
:10091000FFFF6700037F814636858280838705005D
:100920001387F5003D05FD8793F777088346070099
:100930007D158606B58FA300F5006307B7007D1708
:10094000834717009D83DDB782801713FFFFE702FF
:100950000379B7E7040083A7070932872A863A8517
:100960008297133515001713FFFF6700837915C1B0
:1009700081478DC11713FFFFE7026376414697E079
:100980000000E780003985473E851713FFFF6700A9
:10099000437781473E8582801DCD1713FFFFE70215
:1009A0000374414681452A849710FFFFE780207633
:1009B00041468145130504039710FFFFE78020752A
:1009C0000147C1672322040438C87CC805451713B2
:1009D000FFFF670003730145828081473DCDB5CDA0
:1009E0001713FFFFE702A36FB2842E891306800559
:1009F00081452A849710FFFFE7806071CA8524C46F
:100A0000268597000000E780C0F641468145228593
:100A10009710FFFFE780A06F3044A28522859700E2
:100A20000000E780C0F293040401A28526859700A8
:100A30000000E780E0EEA6851305040297000000A1
:100A4000E78000EE228597000000E78020F58547CB
:100A50003E851713FFFF6700C36A3E858280171328
:100A6000FFFFE70223664111E9540DCD85CD93F9CF
:100A7000C5FF2E842A89AA84338AA900B7EA040014
:100A8000639844030D88814411CCB7E704009C5F50
:100A900082972AC622866C003305390197E0000050
:100AA000E7802027268541011713FFFF6700C364F5
:100AB00083A78A039104829793170501C183A183B9
:100AC000A38EF4FE93570501238FF4FEA183238E9A
:100AD000A4FEA38FF4FE6DB765CD1713FFFFE702E9
:100AE000635EB28411E605451713FFFF6700C3601C
:100AF0002A842E890145EDD93C487848B3E6E700C1
:100B0000E5D69386F7FFB3B7F6007D17032A4404B2
:100B1000BA9734C87CC863050A06C14913050A039D
:100B2000B38949412295637D3601B2862E86A6851A
:100B300097000000E780A0DB7C40BE9464C065B7EE
:100B4000CE862E86CE8597000000E78040DAC1145D
:100B5000D2944E9923220404A2879306040103C76A
:100B6000070003C607038507318FA38FE7FEE398CD
:100B7000F6FE3044A285228597000000E78020DD44
:100B80002699C1493306994063EC9900A9DCA686F1
:100B9000A6851305040397000000E78040D579BFC0
:100BA0008147B306F4003307F6000347070083C507
:100BB000060085072D8F2380E600E39437FF30443D
:100BC000A285228597000000E78060D8C1145DBF30
:100BD000014582800DC11713FFFFE7024350130642
:100BE000800581459710FFFFE78060520545171388
:100BF000FFFF6700035101458280814749C5C1C598
:100C00001713FFFFE702A34DFC4141462E84AA843F
:100C10006399C70413860501A2878146C14503C7AE
:100C2000070003C507038507298F3305D600034551
:100C300005008506298FA38FE7FEE392B6FE3044B8
:100C4000A285268597000000E78060D02285970066
:100C50000000E78060F885473E851713FFFF6700B7
:100C6000434A138507031D8E814522959710FFFF88
:100C7000E780E0497C40130700F813060402A297BE
:100C80002388E70251BF3E8582801713FFFFE702EA
:100C900003456D712E84B284AA8590102800368990
:100CA00097000000E780A0D309EDD55725A050405C
:100CB0000C40280097000000E78040E27DD5FD143D
:100CC0002104F5F42C004A8597000000E78020F30A
:100CD000814761DD3E8551611713FFFF6700634265
:100CE0001713FFFFE702A33F41112EC432C62C00A9
:100CF000054697000000E78080F941011713FFFFC8
:100D0000670023401713FFFFE702633D01112A84A8
:100D10002EC602C802CA02CC02CE97E00000E780CD
:100D2000C023B2462A86A285080897000000E78003
:100D300060FB1375F50F05611713FFFF6700633C38
:100D40001713FFFFE702A3397971B2872A8421467E
:100D50002308B10013051101BE853AC436C697E0D9
:100D60000000E78000FBB2469305910136859700AD
:100D70000000E78060A82285141035460C08970013
:100D80000000E78020F62A84224701E921460C1062
:100D90003A8597E00000E780C0F722854561171388
:100DA000FFFF670003361713FFFFE702433371713C
:100DB000AE84AA850A85328497000000E78060BB74
:100DC00011C90A86A685228597000000E78020B811
:100DD000814711E1C5473E854D611713FFFF67004D
:100DE00043321713FFFFE702832C1D712A8AB28951
:100DF000BE8435468547130511012E8CB68A3A8B81
:100E0000C28C468D2308F10097E00000E78060F077
:100E100010100C085285231F010097000000E78086
:100E2000C0F82A843DEDA1476313FD0893079005A0
:100E300091E0E5473546E2851305110113990A0152
:100E40002308F1001359090197E00000E78060ECE6
:100E50001357890093978A00D98F90080C08528500
:100E6000231FF10097000000E78020F42A8415E991
:100E7000A1E49387FA0091831379F9003EC66313C6
:100E800009004149668B8144C14B854DB247639F40
:100E9000970C6A868C0033855C0197E00000E78040
:100EA00040E7228525611713FFFF6700032493079E
:100EB0009004C9F0A547BDBF834701050947C14B51
:100EC0002308F10083471105A58FA308F10093873C
:100ED0002400814463E1FB04014714083386E600E3
:100EE0008C08B386E400BA95DA9683C6060083C5FB
:100EF00005000507AD8E2300D600E390E7FE4147CD
:100F0000639CE70490080C08528597000000E78076
:100F1000C0E925D181A0B3069B00BA871008B305AC
:100F2000F60090083E9603C50600034606008507B6
:100F30008506298E2380C500E39277FF998F90085C
:100F40000C085285BE9497000000E78000E68947B0
:100F5000014749D12A84B1B790083E96034606005E
:100F60001408BE962380C600850759BFB247850482
:100F70006387971481471808B306F70098083E97CF
:100F80003386F90003470700034606008507318FC3
:100F90002380E600E39177FF90080C0852859700C4
:100FA0000000E78080E05DF53546E285130511011C
:100FB0002308B10197E00000E780A0D51397040152
:100FC0004183939784002183D98F10180C08528590
:100FD000231FF10097000000E78020DD25FD8147F9
:100FE00010183387F9003E960347070003460600B2
:100FF000B306FB008507318F2380E600E39277FF7D
:1010000065A81808B306F70098083E973386F900DC
:1010100003470700034606008507318F2380E6005B
:10102000E3E127FFCA87639E770990080C08528581
:1010300097000000E78060D711FD81479800B30654
:10104000F700900818103E973E96034707000346A6
:1010500006008507318F2380E600E39177FF354650
:10106000E285130511012308B10197E00000E78034
:1010700040CA139704014183939784002183D98F39
:1010800010180C085285231FF10097000000E7801C
:10109000C0D1E31105EC814710183387F9003E9663
:1010A0000347070003460600B306FB008507318FA0
:1010B0002380E600E3E227FFC109410BC1BB814762
:1010C00085B79408BE9683C6060018083E9723008D
:1010D000D700850789BF638006321713FFFFE70239
:1010E00003FD59712A84BE89B28B854735461305A5
:1010F00011022E8B468C4289BA8A368A2300F1026D
:1011000097E00000E780E0C010180C10228523173C
:10111000010297000000E78040C963180512A1474B
:10112000631FFC069307900563930900E547354666
:10113000DA851305110293140A012300F102C1801C
:1011400097E00000E780E0BC93178A0013D7840083
:10115000D98F90080C1022852317F1029700000008
:10116000E780A0C47DE1639209049307FA00BD887B
:10117000918391E0C144C207C183DE8C814A3EC69F
:10118000414DB24763E2FA0E6286B3854B01881087
:1011900097E00000E78080B54DC93D557DA09307DD
:1011A0009004E39609F8A54759B783470105094715
:1011B000C14C2300F10283471105B3C7F900A30016
:1011C000F10293872900814963E1FC0481461810EC
:1011D0003306D7008C083387D900B6955697034756
:1011E000070083C5050085062D8F2300E600E390E8
:1011F000D7FE41476390E70690080C1022859700C0
:101200000000E78080BA35D189A0B3863A01BA8759
:101210001010B305F60090083E9603C5060003467D
:10122000060085078506298E2380C500E39297FF77
:101230003387EC4090080C102285BA999700000083
:10124000E780A0B68947014741D165611713FFFFC9
:101250006700A3E990083E96034606001410BE9668
:101260002380C600850779B7B247850A93990A019A
:10127000939D8A0093D909016391570F854735469D
:10128000DA85130511022300F10293D9890097E052
:101290000000E78000A8B3ED3D0190000C1022850E
:1012A0002317B10397000000E78020B059FD814764
:1012B000A68963EA970626860C084A8597E000000F
:1012C000E78020A581471810B306F700100898089A
:1012D0003E973E9603470700034606008507318F79
:1012E0002380E600E3E197FE639FA90590080C10B8
:1012F000228597000000E78040AB21F981479810D4
:10130000B306F700900818183E973E96034707006B
:10131000034606008507318F2380E600E391A7FF8F
:101320004109C10CB9BD18089000B306F7003E96FC
:101330003387FC0003470700034606008507318F0B
:101340002380E600B5B798084E97034707001C10A6
:10135000CE972380E700850941BF85473546DA856A
:10136000130511022300F10293D9890097E00000D0
:10137000E780209AB3ED3D0190000C1022852317E1
:10138000B10397000000E78040A2E31005EC81471D
:1013900018089000B306F7003E963387FC00034719
:1013A0000700034606008507318F2380E600E3919E
:1013B000A7FF41460C084A8597E00000E78060954A
:1013C00081471810B306F700100898083E973E961C
:1013D00003470700034606008507318F2380E60098
:1013E000E391A7FF90080C10228597000000E7808A
:1013F000C09B1DD599BD7D5582801713FFFFE70265
:1014000003CE01112A842E8593055100328902C032
:1014100002C202C402C69304740097F0FFFFE78083
:10142000A03D1D46A6851305910097E00000E780CA
:10143000408E10088A854A8597000000E780E09674
:1014400019ED93071400180883C607000346070028
:1014500085070507B18EA38FD7FEE397F4FE0561DC
:101460001713FFFF6700E3C91713FFFFE70283C5E8
:101470002E848C414111AA898387150032899144B9
:1014800063D30700A1449757FF1F9387E7E59C4369
:10149000A1C7C1CA8D472310F10083C725004A8523
:1014A0002301F10083C73500A301F10083C7450084
:1014B0002302F10083C75500A302F10083C7650032
:1014C00093059100A30301002303F100230401000D
:1014D00097F0FFFFE78040320C404A860A8597F07C
:1014E000FFFFE78080330328040083564400A6886A
:1014F0001D0881470147E51642868A854E8597007B
:101500000000E780408E2A8919E5A685228597B0DC
:10151000FFFFE780E0C14A8541011713FFFF670025
:10152000A3BD4A860A8597F0FFFFE780002F6DB7BD
:101530001713FFFFE70203B92E848C414111AA89DA
:10154000838715003289914463D30700A1449757DC
:10155000FF1F938767D99C43A1C7C1C68D4723103E
:10156000F10083C725004A852301F10083C73500B8
:10157000A301F10083C745002302F10083C7550092
:10158000A302F10083C7650093059100A303010046
:101590002303F1002304010097F0FFFFE780C0253B
:1015A0000C404A860A8597F0FFFFE78000278356A4
:1015B0004400032804008A85858EC2061D08C18266
:1015C0002312D400A68881470147E51642864E853E
:1015D00097000000E78060B041011713FFFF67002C
:1015E000A3B14A860A8597F0FFFFE78000234DBF2D
:1015F0001713FFFFE702A3AEB335B0000111850555
:101600002A891315F601336515012308B1009305E6
:10161000110136843AC632C03EC442C297F0FFFF81
:10162000E780801DA2471248425593D68700230BBE
:10163000F1009305910193578800A30AD100A30BF1
:10164000F100230C010197F0FFFFE780E01A324719
:10165000024603280400B337E00083564400920793
:10166000914411C2A1444A85A68842860C0897F08D
:10167000FFFFE78040772A8919E5A685228597B084
:10168000FFFFE780E0AA4A8505611713FFFF6700A7
:1016900043A71713FFFFE702E3A201113EC68647E7
:1016A000B335B0008505AA891315F6015D8D2308B1
:1016B000B1009305110136843A89B28442C446C20E
:1016C00097F0FFFFE7804013224892481645935752
:1016D0008800A30AF1009305910193D78800230B9A
:1016E0000101A30BF100230C110197F0FFFFE7802C
:1016F000A0103247104083564400B337E0009207F1
:1017000003280900914891C0A1480C084E85970014
:101710000000E780809CAA8401E9835544004A8543
:1017200097B0FFFFE780C0A0268505611713FFFF74
:101730006700839CAA959307F00F17070100130712
:10174000A7676317B50013C5F7FF1375F50F828000
:1017500005058346F5FFB58FBA9783C70700D5B750
:101760000357450014419307F00F170601001306B5
:10177000A664369742074183139506014181631B96
:10178000E500AD8FB29703C50700130515F31335B8
:1017900015008280850603C5F6FFA98FB29783C71F
:1017A0000700D9BF1713FFFFE7026393B2873684A0
:1017B0002E86BA86AA853E85BA8497F0FFFFE78019
:1017C0006052634F0500228597D00000E780E078E3
:1017D0002A86A686A285268597F0FFFFE78080509F
:1017E0001713FFFF6700E3911713FFFFE702838DD5
:1017F0005D712A8BAE8A17050100130565592C000F
:10180000B284368ABA893E8997F0FFFFE780C04FDD
:101810002A845DE134104146DA85280097F0FFFF05
:10182000E780404C2A8449E98547A303F100A6C21A
:10183000930771002408BEC4A68685470D462C1860
:10184000281002DC02DED6C0BEC697F0FFFFE7809C
:1018500000442A8435E183477102A6860D4693F73A
:10186000F7072300FA00C1473EDE2C1889472810ED
:1018700026DCA303F10097F0FFFFE78040412A84B4
:1018800005ED4146A6854E8597D00000E78060486B
:101890008D47A6860D462C182810A303F10097F05B
:1018A000FFFFE780C03E2A8401E94146A6854A85BC
:1018B00097D00000E780E045228561611713FFFFA4
:1018C000670083831713FFFFE702638197F7000028
:1018D0009387C7A0984383C7470079712A89AE844C
:1018E000170501001305454B0C083AC42306F10007
:1018F00097F0FFFFE78040412A8405ED1410414630
:10190000CA85080897F0FFFFE780C03D2A8415E1EB
:10191000140815462C00081097F0FFFFE780803C64
:101920002A8401E921462C08268597D00000E7800B
:10193000403E228545611703FFFF6700837C170344
:10194000FFFFE702C37997F70000938727999C4729
:101950007971AA842E8417050100130565440C08CB
:101960003EC697F0FFFFE780203A0DE9141041468C
:10197000A685080897F0FFFFE780C03605E1140848
:1019800011466C00081097F0FFFFE780A03519E5BD
:101990008347F10193F7F7032300F4004561170330
:1019A000FFFF670003761703FFFFE70243733688E4
:1019B000A14881470147E54697F0FFFFE780A04235
:1019C0001703FFFF6700E3731703FFFFE7022371AD
:1019D0003688A14881470147E54697F0FFFFE78039
:1019E000C06F1703FFFF6700C3711703FFFFE70214
:1019F000036F01112A842E850C0832C697F0FFFF71
:101A0000E780803009ED3247970601009386C6379C
:101A10001008C145228597000000E780E0D80561E5
:101A20001703FFFF6700E36D1703FFFFE702236B58
:101A30004111C1472EC032C48A8509463EC23EC606
:101A400097F0FFFFE780A02441011703FFFF670025
:101A5000436B1703FFFFE70283684111AE8613064D
:101A60001009AA850A8502C002C202C402C697F004
:101A7000FFFFE780202741011703FFFF670063682E
:101A80001703FFFFE702A3653287970601009386DD
:101A9000A6312E869305000297000000E780C0D093
:101AA0001703FFFF6700E3651703FFFFE7022363E8
:101AB0007971C1472ACC2ED032D42C080D4628008B
:101AC0003ECE3ED23ED602C402C602C802CA97F03B
:101AD000FFFFE780C01B45611703FFFF67006362DC
:101AE0001703FFFFE702A35F0111AA842E841705E5
:101AF00001001305E52B8A8597F0FFFFE780C020E2
:101B000015E514084146A6850A8597F0FFFFE78092
:101B1000601D09ED8347E1010347F101A207D98F59
:101B2000CA07C9836177D98F2310F40005611703B1
:101B3000FFFF6700035D15CD1703FFFFE702235A80
:101B40009747FF1F9387C72790439745FF1F9385AC
:101B500065271745FF1F1305A52297D00000E780D2
:101B600000C51745FF1F1305A5211703FFFF6700D9
:101B700043591745FF1F1305A52082808DCD1703FC
:101B8000FFFFE702C3559747FF1F938767239443DF
:101B900001112E840A869745FF1F9385A52297D0B1
:101BA0000000E78040C60A850294014505611703DD
:101BB000FFFF670003557D5582801703FFFFE70293
:101BC000035297D00000E78080D19747FF1F23A9D9
:101BD000A71E17F5FFFF1305E5C997B00000E780C2
:101BE000C0741703FFFF6700C3511747FF1F130798
:101BF000671F9317150008433E95FD572310F50006
:101C000082801703FFFFE702834D2A84084009E51D
:101C10001703FFFF6700E34E1C4158401CC06313CD
:101C2000E5005CC08347550023200500F99BA30213
:101C3000F50097A0FFFFE780207CC9BF1703FFFFD7
:101C4000E70243489747FF1F9387C71B98432A849F
:101C500011CB8347350093F7070289C70355050069
:101C6000894502971305440197B00000E780403B87
:101C7000835504000355E40097300000E780A00C72
:101C8000485819C597A0FFFFE7800077232A040270
:101C90001305840397000000E780E0F68144B14912
:101CA0009790FFFFE780206A63CBA402834734004C
:101CB0002320040493F727FCA301F4000048979025
:101CC000FFFFE780406913161500814522859700C4
:101CD000FFFFE780C0431703FFFF6700E341B387BF
:101CE00034030329040385043E994A8597000000C4
:101CF000E78060F12304090065B78347350093F757
:101D0000070299E3014582808357E500E39CB7FE13
:101D1000C167FD176316F60005458280054599A841
:101D20001703FFFFE702A33B93170601C187B284A5
:101D30002A8401496359F002835705009DCB014570
:101D40006367F600034584003E953325A6001375AE
:101D5000F50F0DA01C4813171900BA9783D7070079
:101D6000E38E97FA05099790FFFFE780C05EE34393
:101D7000A9FE01451703FFFF6700A3381703FFFF04
:101D8000E7024334AE89AA849790FFFFE780605250
:101D90002A8497D0FFFFE780A02EAA86014713066A
:101DA000840197050000938585E41745FF1F1305FF
:101DB000A5039790FFFFE780E0182A8925C98C4486
:101DC0001304C50022859E0593F5050897A0FFFF23
:101DD000E780403CCC4083877400E18163DD0704E9
:101DE00093E50508228597A0FFFFE780A03A0D46FE
:101DF00093854400228597A0FFFFE780C03683D5F6
:101E00000400228597A0FFFFE780E03D83D52400F2
:101E1000228597A0FFFFE780003D03D6490083A5F8
:101E20000900228597A0FFFFE780E0334A8517036A
:101E3000FFFF6700632C93F5F5076DB71703FFFFEE
:101E4000E702E32901112A84328532C697A0FFFFF9
:101E5000E780E0279780FFFFE780C03083570400CA
:101E60001747FF1F130787113246231BF100930703
:101E700000F8A30DF1001C471843231AA100898321
:101E8000858BB307F740B28548083ECE231C01007E
:101E9000230D010097000000E78080EE0561170325
:101EA000FFFF670003261703FFFFE702A32100419E
:101EB00001453DC49304C40026853289AE8997A0AC
:101EC000FFFFE780C02495452A8A2685035B04012D
:101ED00097A0FFFFE7802021268597A0FFFFE780DE
:101EE000603E8D45AA8A268597A0FFFFE780A01F48
:101EF000268597A0FFFFE780E03C5C48420A135A22
:101F00000A01D2975CC423186401814763983A019F
:101F100046054D81330625419337160013F5F70F1B
:101F20001703FFFF6700431D1703FFFFE702A31816
:101F300089692A8BAE8B328AB68A81440144314C3E
:101F4000FD199790FFFFE780004063CDA4009790B4
:101F5000FFFFE7804042018D33B5AA001703FFFF62
:101F60006700E3183389840383270B003E996317C6
:101F70000A008347890085043E94E1B703560A00AE
:101F8000DE854A8533F6C90097000000E780E0F15E
:101F90006DD10545E1B71703FFFFE70243140111B7
:101FA0002A847C000355E5003ECAB70707003ECCF3
:101FB0007C003ECE97200000E78020082A898545D6
:101FC000480897A0FFFFE78020399945480897A067
:101FD000FFFFE780E015AA844A8597200000E7808C
:101FE000A0082380A4009747FF1F938727F99C43ED
:101FF0004166130606F09396870113D78701558F24
:1020000093D68700F18E558FA207B706FF00F58F94
:10201000D98F11462C00138514003EC497D00000C0
:10202000E78020CF5008A3820400894522859700CD
:102030000000E780E0E019C9AA851305840397A092
:10204000FFFFE780E0313C4085073CC00561170396
:10205000FFFF6700030B1703FFFFE702430897909A
:10206000FFFFE78040312A8405049790FFFFE78057
:10207000802F3305A402F14791453305F5029720DF
:102080000000E78020BA11E565551703FFFF6700E0
:1020900043079747FF1F23AFA7D49790FFFFE78021
:1020A000802D2A8405049790FFFFE780C02B33051D
:1020B000A4028945060597200000E780A0B669D5EF
:1020C0009747FF1F23A0A7D29790FFFFE780A02A82
:1020D0002A8405049790FFFFE780E0283304A402D8
:1020E0009747FF1F239287D09790FFFFE780A02894
:1020F0002A849790FFFFE780002793071400338519
:10210000A7029747FF1F2392A7CE97070100938747
:10211000E78D1747FF1F232DF7CC0145BDB71703E8
:10212000FFFFE70223FAAA842E8901449749FF1F83
:102130009389C9E4130A80069790FFFFE780A022E5
:102140006347A40001451703FFFF6700E3FA330567
:10215000440383A709024A86A6853E95970000009E
:10216000E780E0B919E10504C1BF0545E9BF1703E0
:10217000FFFFE70243F4AA8A2E8BB28B368C3A8A91
:10218000814401448149974CFF1F938C2CDF130D30
:1021900080069790FFFFE780001D63C9A40011E04F
:1021A00085494E851703FFFF670063F43389A40355
:1021B00083A70C025E86D6853E994A85970000006B
:1021C000E780E0B31DC19790FFFFE780C01A054488
:1021D000636D4501D2866286DA851305090397008F
:1021E0000000E780A0D411C1854985045DB71703BD
:1021F000FFFFE70223EDC16441112A890144974999
:10220000FF1F9389A9D7130A8006FD1436C632C46E
:102210002EC29790FFFFE780001592452246B246F6
:102220006348A400014541011703FFFF6700C3ECA9
:102230003305440383A709023E9509C68347350049
:10224000C18B9DC791C68347350093F707028DC3A5
:10225000630699008357E500639C27010357050037
:1022600001CB63E7E50083478500BA97E3CDF5FA34
:10227000050469BF1703FFFFE702C3E4C1642A89AD
:1022800001449749FF1F938969CF130A8006FD1403
:102290009790FFFFE780200D6346A4001703FFFF20
:1022A000670083E53305440383A709023E958357FE
:1022B000E500638A970063049900639627019700FD
:1022C0000000E780E0970504E1B71703FFFFE7028E
:1022D00003DE89692A8AAE8A328BB68B8144174C19
:1022E000FF1F130CACC9930C8006314DFD1997905C
:1022F000FFFFE780400763C6A4001703FFFF6700E6
:10230000C3DE3389940383270C028355CA015A869E
:102310003E994A8597000000E780609E31C1814D5B
:1023200015A03384AD038327090303D60B00D6859C
:1023300033F6C9003E94228597000000E780E0B69E
:1023400009E9850D9790FFFFE780E0FFE3CBADFC47
:1023500001A8228597000000E780E08A230404009A
:10236000850471B71703FFFFE702E3D44169AA8A26
:10237000014A174BFF1F130B6BC07D19C14B054C56
:102380009790FFFFE78020FE6346AA001703FFFF38
:102390006700E3D593098006B3073A0383290B024C
:1023A000BE9983D7E900638E270163842A01639A6B
:1023B000570103A4890301E84E8597000000E780D8
:1023C000C0BD050A75BF835704016399770993045B
:1023D000C400268597A0FFFFE78060D385452A8D3E
:1023E0002685835C040197A0FFFFE780C0CF268588
:1023F00097A0FFFFE780A0E76205618563590504A8
:102400008D45268597A0FFFFE780E0CD894526858D
:1024100097A0FFFFE78020CD8945268597A0FFFF85
:10242000E78060CC8545268597A0FFFFE780E0CC5C
:1024300083470500094793F7F707639AE700994533
:10244000268597A0FFFFE78040CBA302850148487F
:10245000337D2D01231894016A9548C40040A1BF23
:102460001703FFFFE702A3C737E404008327041D17
:1024700082979747FF1F83C7679D1715FF1F130597
:10248000E50CA300F5008327441C82978327841C56
:1024900081461306F00F8145014582971703FFFF20
:1024A000670023C61747FF1F1307478A184397453E
:1024B000FF1F83C5A5999747FF1F9387A79783465B
:1024C0008703034697036397D5009747FF1F238F22
:1024D000C796828083C587010347A7036317B600A9
:1024E0009747FF1F2384E796828003C687016317FF
:1024F000C7009747FF1F238BD794828083C687012D
:10250000130750026319D700930760021747FF1F94
:10251000230EF792828083C687011306600263153B
:10252000D60093077002DDB783C7870155BF974771
:10253000FF1F93872790D44B0947638DE608170345
:10254000FFFFE702C3B91749FF1F1309E98B3E8458
:1025500083470900918B9DCFB7E4040083A7041D36
:10256000829783A7441C1745FF1F1305658A82972E
:1025700083A7841C81461746FF1F0346668B81454F
:102580000145829721C583470900ED9B1747FF1F2F
:10259000230CF7868347040093F7F70F85CB914709
:1025A0001747FF1F2322F78A97000000E78080EB80
:1025B00097000000E78040EFB7E70400BC4F4146BA
:1025C00091451745FF1F0345658782971703FFFF56
:1025D000670023B382801703FFFFE70243B08D47F4
:1025E00041116306F504C5476308F502854763108A
:1025F000F5029747FF1F238DA784B7E70400BC4B64
:10260000930500101745FF1F03454583829741013D
:102610001703FFFF6700E3AE85471747FF1F230936
:10262000F782B7E70400BC4B93050020E1BF974752
:10263000FF1F93872780D44B1147638DE600B7E7D0
:10264000040083A7071D8297B7E70400BC4B9305DE
:1026500000044DBF05491737FF1F2327277F83C776
:10266000070032C62E8493F7F70FD5D3B7E40400E2
:1026700083A7041D7D141374F40F8297E37689FCFD
:10268000B245994703C61500E3F0C7FCFC440906B0
:102690001735FF1F1305057C8297BC48930500087A
:1026A0001735FF1F03458579829779BF1703FFFF11
:1026B000E702E3A21737FF1F1307C7774047184BFE
:1026C0001C409736FF1F23ADF6766316E4001737DC
:1026D000FF1F2329F776130584FE9790FFFFE780FD
:1026E00060A6035564FF9780FFFFE780E06E97A028
:1026F000FFFFE78060D01703FFFF670083A0170389
:10270000FFFFE702C39D9737FF1F9387A772D84B40
:10271000DC4789C797000000E78080F985471737B5
:10272000FF1F2323F7729737FF1F938727629C436E
:10273000930500021735FF1F0345457083C78703C4
:102740001737FF1F2304F770B7E70400BC4B8297CD
:102750001703FFFF6700E39A9737FF1F23AEA76CAD
:1027600082801703FFFFE702E39537E404007C4C07
:10277000A1451735FF1F0345656C82977C48A1452D
:102780001735FF1F0345856B9734FF1F9384846AB9
:102790008297DC4489EB97000000E78080D917031B
:1027A000FFFF6700639503D567FF9780FFFFE78012
:1027B000A062AA896DD1D84891476310F7027C4C7A
:1027C00091451735FF1F0345656782977C48914502
:1027D0001735FF1F03458566829703A9490103D476
:1027E00009018947B7E904001737FF1F232EF76453
:1027F00083A7091D21044204829783C7840117150A
:10280000FF1F1305A5D461191717FF1FA300F7D4E5
:1028100083A7491C418082979737FF1F238A07624D
:1028200083A7C91C814609469375F40F4A85829790
:1028300011E99737FF1F83C7E77189C79700FF1F0B
:10284000E780403BB7E70400BC4F2146A145173560
:10285000FF1F0345A55E829799B71703FFFFE702A5
:10286000038893F7052001112E8481CF9700000083
:10287000E78020E91345042005611703FFFF670087
:10288000438893F70510A9CF9734FF1F9384845A88
:10289000DC4897000000E78020C11737FF1F1307AF
:1028A000E74A184383C78401034787036318F70087
:1028B000DC4489C797000000E78080DF8547173731
:1028C000FF1F2323F758B7E70400BC4B9305000212
:1028D0001735FF1F0345855682971345041069BFBE
:1028E00093F70508BDC79737FF1F83C7B756E9178A
:1028F00019469735FF1F938505561305D10093F4AC
:10290000F70F1739FF1F0349E95497C00000E7800C
:10291000404093970401C1831737FF1F13070754E3
:10292000231DF100231CF1009737FF1F9387875069
:102930003ACE3ACAD8432306010009CBDC439315AB
:10294000890154080D46E185680082971345040803
:1029500025B793F72500A5C39737FF1F9387874DAA
:10296000D84B89476306F7029737FF1F83C7C749CC
:1029700013F7270011EF918B99CFB7E70400BC4FF5
:102980001306000A89451735FF1F0345254B82971B
:1029900013452400D5B59737FF1F9387273B9C43EA
:1029A00083C787031737FF1F2302F74A97000000EA
:1029B000E78060DBF1BF93F7050281CB9700000051
:1029C000E78060DA1345040245BD93F7850081CBAB
:1029D00097000000E780E0D21345840071BD93F7B3
:1029E000150081CB97000000E780A0B413451400C8
:1029F00061B593F7450081CB97000000E78060B395
:102A00001345440095BD93F7050495C39737FF1F01
:102A100083C7474291CB97000000E780A0A491476D
:102A20001737FF1F2322F74213450404B1B593F76C
:102A300005010145E38207E49737FF1F9387873F2E
:102A4000D84B91476310F7049737FF1F9387C73B15
:102A50009C4313D727008583D98F858B91E7B7E7F0
:102A6000040083A7071D8297B7E70400FC4F914538
:102A70001735FF1F0345853C829785471737FF1F92
:102A80002324F73C13450401C5BB9737FF1F23835D
:102A9000A74C828017F3FEFFE70263649737FF1F9E
:102AA00023A0073A9737FF1F23AE0738854717340F
:102AB000FF1F1304A4291737FF1F2327F7381C40D3
:102AC00083C787031737FF1F2302F7389790FFFF4D
:102AD000E780A08F29C59717FF1F23ADA7A61C402D
:102AE000170500001305A5D783C787031737FF1FF6
:102AF000230EF7341717FF1FA30AF7A49737FF1FFA
:102B0000A38A0732B7E7040083A70708829797379D
:102B1000FF1F2385A73217F3FEFF6700835EB7C749
:102B2000898E938767ED1717FF1F2325F7A245BFEF
:102B30001737FF1F03470730795555E79737FF1FB2
:102B40009387472F03C7170005079736FF1FA383F7
:102B5000E62E03C717008D463377D7029736FF1F3F
:102B6000A38AE62C83C617001737FF1F1307071E1B
:102B7000184393F6F60FA9EE834787031737FF1F15
:102B80002306F72C85471737FF1F2305F72A9737AA
:102B9000FF1F938767279C430145998BA9E717F38C
:102BA000FEFFE702C35337E404007C48C1451735F4
:102BB000FF1F0345A52882973C4885451735FF1F11
:102BC0000345C5278297014517F3FEFF670063534E
:102BD00083C7170085466395F6008347970379BF3F
:102BE0008347A70361BF82809737FF1F83C787246E
:102BF000A1CF17F3FEFFE702834E37E404009737B7
